:020000040800F2
:10000000B804002045010008314E0008F908000836
:100010002D4E0008DF0300081957000800000000FB
:10002000000000000000000000000000F54F000884
:10003000A905000800000000BD4E0008DD500008C2
:100040005F0100085F0100085F0100085F01000810
:100050005F0100085F0100085F0100085F01000800
:100060005F0100085F0100085F0100085F010008F0
:100070005F0100085F0100085F0100085F010008E0
:100080005F0100085F0100085F0100085F010008D0
:100090005F0100085F0100085F0100085F010008C0
:1000A0005F0100085F0100085F0100085F010008B0
:1000B0005F010008415100085F0100085F0100086E
:1000C0005F0100085F0100085F0100085F01000890
:1000D0005F0100080154000861540008BD54000885
:1000E0005F0100085F0100085F0100085F01000870
:1000F0005F0100085F0100085F0100085F01000860
:100100005F0100085F0100085F0100085F0100084F
:100110005F0100085F0100085F0100085F0100083F
:100120005F0100085F0100085F0100085F0100082F
:10013000DFF80CD000F032F900480047A95F000852
:10014000B80400200648804706480047FEE7FEE75F
:10015000FEE7FEE7FEE7FEE7FEE7FEE7FEE7FEE777
:10016000E150000831010008D2B201E000F8012B93
:10017000491EFBD270470022F6E710B513460A4627
:1001800004461946FFF7F0FF204610BD2DE9FE4F4B
:1001900081EA030404F0004421F0004100944FF090
:1001A000000B23F0004350EA010402D052EA03049A
:1001B00004D10020014603B0BDE8F08FC3F30A5418
:1001C000C1F30A552C44A4F2F3340194A0FB025469
:1001D000C1F3130141F48011C3F3130343F48013FB
:1001E00001FB024400FB034E840A970A44EA81544F
:1001F00047EA8357A4FB076802958D0A05FB07852C
:100200004FEA932C04FB0C542705029D4FEA065835
:1002100047EA1637B5EB08056EEB070C870E920E12
:1002200047EA811742EA8312A7FB0201B6EB0B01F2
:1002300064EB00042B0D43EA0C335E1844EB1C50B6
:10024000DA465146E7FB0201C5F313044FEA0B33CC
:1002500043EA14534FEA0432019C43EA0603A4F133
:100260000C040294009CCDE900B400F044F8A2E72D
:100270000EB540F2334102910021CDE900110A464A
:100280000B4600F038F803B000BDC1F30A5210B5B8
:10029000C1F3130140F2FF3341F480119A4201DAB5
:1002A000002010BD40F233439A42A2F2334203DCF5
:1002B000524200F003F810BD904010BD202A04DB2C
:1002C000203A21FA02F00021704721FA02F3D040CF
:1002D000C2F12002914008431946704710B5002B27
:1002E00008DA401C41F1000192185B411A4301D128
:1002F00020F0010010BD2DE9F04D92469B4611B152
:10030000B1FA81F202E0B0FA80F22032904600F0B9
:1003100057F804460F4640EA0A0041EA0B015346EB
:100320005A46084303D120463946BDE8F08D1146B0
:1003300053EA010015D0C8F140025046FFF7BEFF56
:1003400005460E4650465946424600F039F80843E5
:1003500001D0012000E00020054346EAE0762C436E
:1003600037430A984FEA4453A0EB08004FEAD424DD
:100370000A304FF0000244EA47544FEAD72502D52D
:1003800000200146D1E7010510196941DDE9084562
:1003900000196941BDE8F04DA0E70000064C074D8B
:1003A00006E0E06840F0010394E807009847103445
:1003B000AC42F6D3FFF7C0FE04200608242006084E
:1003C000202A04DB203A00FA02F100207047914015
:1003D000C2F1200320FA03F319439040704700BF95
:1003E000FEE7000010B5002400F024F804E0601CD3
:1003F000C4B2012005F0E7FA0D48006808B1642C8A
:10040000F5DB642C01DB012010BD002404E0601C3E
:10041000C4B2012005F0D7FA0548006808B9642C79
:10042000F5DB642C01DB0120EEE70020ECE70000A7
:100430002401224208B54FF40070ADF800004820B6
:100440008DF803006946024800F04DF908BD000030
:100450000010014008B54FF40070ADF80000102006
:100460008DF8030003208DF802006946014800F072
:100470003AF908BD0010014008B50121102004F030
:100480003FFD4FF40070ADF8000010208DF8030020
:1004900003208DF802006946064800F024F94FF465
:1004A0000071044800F0AAF900F068F8FFF79AFF1D
:1004B00008BD00000010014010B5002404E0601CDD
:1004C000C4B2012005F07FFA0D48006808B1642C21
:1004D000F5DB002404E0601CC4B2012005F073FACF
:1004E0000748006808B9642CF5DB282005F06BFA92
:1004F0000348006808B1012010BD0020FCE700009F
:100500002401224270B50024002506E06006040E96
:10051000FFF7D2FF0443681CC5B2082DF6DB204666
:1005200070BD7CB505460E4600F028F8FFF75AFF6F
:10053000F8B9002405E0FFF7E5FF0DF80400601CA2
:10054000C4B2052CF7DB9DF800009DF801100844AB
:100550009DF8021008449DF8031008449DF804100B
:10056000884208D19DF8000030709DF80200287084
:1005700001E001207CBD0020FCE7000010B5FFF782
:1005800069FF0020064908604FF0140005F000FAEA
:1005900001200449C1F8A4011E2005F014FA10BD81
:1005A000A4012242000022427047000051B14FF0E6
:1005B000204252F8202042F001024FF0204343F83D
:1005C000202009E04FF0204252F82020034B1A402F
:1005D0004FF0204343F8202070470000FEFF0F003B
:1005E000D0E901121143C268114302691143426903
:1005F000114382691143C2691143026A1143426A7D
:100600001143826A1143C26A1143026B11434FF0D6
:100610002043026843F822108168082908D11A464D
:10062000016852F8211041F04001026843F822109D
:10063000416B0968426B526841EA0211426B926851
:1006400041EA0221426B928941EA0241426B128ADD
:1006500041EA0251426B127D41EA0261426B9269AA
:1006600011430268521C4FF0204343F82210C16A24
:10067000B1F5804F1AD1816B0968826B526841EAEB
:100680000211826B926841EA0221826B128A41EA6E
:100690000251826B127D41EA0261826B92691143C1
:1006A000026803EB8202C2F8041108E06FF07041A7
:1006B0004FF02043026803EB8202C2F80411704736
:1006C00010B502460020521C002305E014780444B3
:1006D000E0B2521C5C1CE3B28C1E9C42F6DCC443AC
:1006E000641CE0B210BD2DE9F04102460025002651
:1006F000002000230024002791F803C00CF00F0510
:1007000091F803C01CF0100F03D091F802C04CEA1E
:10071000050591F800C0BCF1000F31D0146800202D
:100720002BE04FF0010C0CFA00F3B1F800C00CEA1A
:1007300003069E4220D183004FF00F0C0CFA03F702
:10074000BC4305FA03FC4CEA040491F803C0BCF175
:10075000280F06D14FF0010C0CFA00FCC2F814C0AF
:100760000AE091F803C0BCF1480F05D14FF0010C2D
:100770000CFA00FCC2F810C0401C0828D1D3146049
:10078000B1F800C0BCF1FF0F34DD546800202EE04A
:1007900000F1080C4FF0010808FA0CF3B1F800C0A2
:1007A0000CEA03069E4221D183004FF00F0C0CFA95
:1007B00003F7BC4305FA03FC4CEA040491F803C0B8
:1007C000BCF1280F05D100F1080C08FA0CF8C2F8AA
:1007D000148091F803C0BCF1480F07D100F1080C58
:1007E0004FF0010808FA0CF8C2F81080401C0828E5
:1007F000CED35460BDE8F08141617047016170471C
:100800002DE9FF4F82B0834691469A460024002589
:100810000020019000905F46DDF80C80002661E02A
:10082000012000EB460019F80000A13819F8161055
:10083000A1395E2202FB010080B2009000244AE050
:1008400000251EE00098400100EB44002949085CA7
:1008500001900198A84010F0800F08D008EB040226
:1008600091B27A1990B20F9A00F0C8F907E008EB3C
:10087000040291B27A1990B2109A00F0BFF9681C84
:1008800085B2082DDEDB002521E00098400100EB59
:100890004400401C1749085C01900198A84010F0E2
:1008A000800F09D008EB040291B27A19083290B295
:1008B0000F9A00F0A3F908E008EB040291B27A194C
:1008C000083290B2109A00F099F9681C85B2082D90
:1008D000DBDB601C84B2102CB2DB07F1110087B2A5
:1008E000701C86B20AEBDA71B6EB610F98DB06B0CA
:1008F000BDE8F08F84CF010800BFFEE770B5044665
:100900000026174805884088454315488088A0F58B
:10091000D041043916D112488079012812D1002023
:100920000F4988712A2048812B20888100210846A0
:1009300003F0EEFF01200A4988712B2048812A200C
:10094000888103E00021084603F0E2FF04F03EFA4C
:10095000002602E003480480761CAE42FAD370BD44
:10096000A60000200008006C10B50446002C66D1DB
:100970006C498871F02008804FF4A07048800846C8
:100980008088A0F5134141390BD066488088A0F5D6
:10099000D041043905D063488088A0F5A6411039BC
:1009A0001AD12C205F4908812A2048812B20888178
:1009B00008468088A0F5D041043905D05948808880
:1009C000A0F5A641103906D14FF4A0705549088012
:1009D0004FF4F0704880A1E052488088A0F5AA4109
:1009E000103910D14FF430504E4908814FF428503F
:1009F00048814FF42C5088814FF4F07008804FF4F8
:100A0000487048808AE047488088A0F5C85163391B
:100A10000DD12C20434908812B2048812A20888130
:100A20004FF4F07008804FF44870488076E0222040
:100A30003C49088120204881212088816EE00120E6
:100A4000384988714FF4A0700880F020488008462B
:100A50008088A0F51341413905D032488088A0F53F
:100A6000A641103907D12C202E4908812A2048811F
:100A70002B2088813FE02B488088A0F5D0410439A5
:100A800007D12C20274908812B2048812A208881E2
:100A900031E024488088A0F5AA41103910D14FF4E4
:100AA0003050204908814FF4285048814FF42C5091
:100AB00088814FF4487008804FF4F07048801AE045
:100AC00018488088A0F5C85163390DD12C201549EC
:100AD00008812A2048812B2088814FF448700880A3
:100AE0004FF4F070488006E022200E490881212052
:100AF0004881202088810B488088A0F5D0410439A6
:100B000005D008488088A0F5A641103906D14FF4D9
:100B1000F070044908804FF4A0704880002003F072
:100B200081FD10BDA60000202DE9FF4F84B0814655
:100B30008A460020039002900698A0EB09050798CA
:100B4000A0EB0A06CDF80490CDF800A0002D01DD41
:100B5000012705E00DB9002702E04FF0FF376D4295
:100B6000002E02DD4FF0010806E016B94FF0000834
:100B700002E04FF0FF387642B54201DD2C4600E03E
:100B800034464FF0000B21E0009A91B2019A90B2E6
:100B900000F022F803982844039002983044029011
:100BA0000398A04205DD0398001B03900198384488
:100BB00001900298A04205DD0298001B0290009867
:100BC000404400900BF101001FFA80FB601C83453C
:100BD000DADD08B0BDE8F08F30B504460D46294691
:100BE000204603F095FE04F0F1F80248008802491F
:100BF000088030BD180000200008006C30B50346A6
:100C00000C4615465A488088A0F51341413905D055
:100C100057488088A0F5A641103914D15449488915
:100C200004F0CEF8181204F0C5F8D8B204F0C2F8F7
:100C30004F49888904F0C4F8201204F0BBF8E0B2F0
:100C400004F0B8F88CE04A488088A0F5AA41103931
:100C500020D14749488904F0B3F8181204F0AAF8E3
:100C600043494989491C88B204F0AAF8D8B204F073
:100C7000A1F83F49888904F0A3F8201204F09AF8FB
:100C80003B498989491C88B204F09AF8E0B204F023
:100C900091F865E036488088A0F5C851633928D1BD
:100CA0003348807920B932480088401EC01A83B288
:100CB0002F49488904F084F8181204F07BF8D8B260
:100CC00004F078F8181204F075F8D8B204F072F84D
:100CD0002749888904F074F8201204F06BF8E0B218
:100CE00004F068F8201204F065F8E0B204F062F84D
:100CF00036E01F488088A0F5D04104391DD11C483A
:100D00008079012804D11A480088401EC01A83B295
:100D10001749488904F054F8181204F04BF8D8B277
:100D200004F048F81249888904F04AF8201204F0C7
:100D300041F8E0B204F03EF812E00D488079012855
:100D400004D10B480088401EC01A83B20849488964
:100D5000194604F045F806498889214604F040F810
:100D60000348008903490880881C058030BD0000C5
:100D7000A6000020FE07006C2DE9FC4F05460E463C
:100D800017469846DDF82C9000200190274880886F
:100D9000A0F5D041043929D124488079012825D1F2
:100DA000AB46354621480088C01B401E86B24746E8
:100DB0001E480088A0EB0B00401E1FFA80F80020A0
:100DC0001A4988712A2048812B20888143463A4657
:100DD00031462846CDF80090FFF7CEFF0120134999
:100DE00088712B2048812A2088811CE0781B401CB8
:100DF00080B20190344614E02146284603F088FD75
:100E000003F0E4FF4FF0000A06E00948A0F8009064
:100E10000AF101001FFA80FA01988245F5DB601C97
:100E200084B24445E8DDBDE8FC8F0000A600002048
:100E30000008006C00B59FB00121080204F040F8E2
:100E400001214FF4B47004F05BF80320ADF8780092
:100E500010208DF87B0003208DF87A001EA9FE4833
:100E6000FFF741FC4CF23370ADF8780018208DF894
:100E70007B0003208DF87A001EA9F848FFF733FCA9
:100E80004FF68070ADF8780018208DF87B000320B5
:100E90008DF87A001EA9F248FFF725FC41F2010007
:100EA000ADF8780018208DF87B0003208DF87A00CB
:100EB0001EA9EC48FFF717FC0221E748FFF79EFC4C
:100EC00001200890002009900F200A9000200B902C
:100ED0000C900D900E900190029003200390002042
:100EE000049005900690079006200F900020109027
:100EF00011901020129000201390159014901690CD
:100F000017904FF480501890002019904FF48040B3
:100F10001A9000201B9008A81C9001A81D900FA8F3
:100F2000FFF75EFB01210620FFF740FB322004F0B3
:100F30002FFD002003F040FBCB49888008468088C5
:100F4000FF280ADB08468088A0F57F41FF3904D0DE
:100F5000C5488088B0F5134F7ED1D32003F030FF11
:100F600003F020FBC049888003F01CFBBE49888049
:100F700003F018FBBC498880084680884FF6FF7153
:100F800001EA0020B849888003F00CFBB649898843
:100F90000843B549888008468088A0F51341413947
:100FA0005AD0BF2003F00CFF03F0FCFAAE49888052
:100FB00003F0F8FAAC49888003F0F4FAAA49888073
:100FC00003F0F0FAA8498880084680884FF6FF7140
:100FD00001EA0020A449888003F0E4FAA249898844
:100FE0000843A149888008468088A0F5D04104398B
:100FF0007AD0D42003F0E4FE03F0D4FA9A49888032
:1010000003F0D0FA9849888003F0CCFA964988809A
:10101000084680884FF6FF7101EA002092498880D7
:1010200003F0C0FA9049898808438F4988800846B0
:101030008088A0F5A641103956D04FF45A4003F0ED
:10104000BFFE03F0AFFA884988804FF45B4003F09D
:10105000B7FE03F0A7FA00E046E08349888008461F
:1010600080884FF6FF7101EA00207F4988804FF4A5
:101070005C4003F0A5FE03F095FA7B49898808439C
:101080007949888008468088B0F5004F02D145F242
:101090001050888074488088A0F5AA41103923D068
:1010A000A12003F08DFE03F07DFA6F49888003F0E4
:1010B00079FA6D498880084680884FF6FF7101EA09
:1010C00000206949888003F06DFA674989880843E0
:1010D0006549888008468088A0F5AE41613903D112
:1010E00041F66310604988805F488088A0F513410D
:1010F00041397CD1CF2003F063FE002003F05AFE7B
:10110000C12003F057FE302003F054FEED2003F021
:1011100057FE642003F04EFE032003F04BFE122026
:1011200003F048FE812003F045FEE82003F048FE6E
:10113000852003F03FFE102003F03CFE7A2003F0F0
:1011400039FECB2003F03CFE392003F033FE2C2087
:1011500003F030FE002003F02DFE342003F02AFEC1
:10116000022003F027FEF72003F02AFE202003F0E0
:1011700021FEEA2003F024FE002003F01BFE0020E5
:1011800003F018FEC02003F01BFE1B2003F012FE2C
:10119000C12003F015FE012003F00CFEC52003F072
:1011A0000FFE302003F006FE302003F003FEC720C0
:1011B00003F006FEB72003F0FDFD362003F000FE2D
:1011C000482003F0F7FD3A2003F0FAFD552003F024
:1011D000F1FDB12003F0F4FD002003F0EBFD1A2037
:1011E00003F0E8FDB62003F0EBFD0A2000E0A4E0E8
:1011F00003F0E0FDA22003F0DDFDF22003F0E0FDAE
:10120000002003F0D7FD262003F0DAFD012003F0D3
:10121000D1FDE02003F0D4FD0F2003F0CBFD2A2008
:1012200003F0C8FD282003F0C5FD082003F0C2FD2F
:101230000E2003F0BFFD082003F0BCFD542003F096
:10124000B9FDA92003F0B6FD432003F0B3FD0A2049
:1012500003F0B0FD0F2009E0000C01400014014034
:101260000018014000200140A600002003F0A2FD6C
:10127000002003F09FFD002003F09CFD002003F000
:1012800099FD002003F096FDE12003F099FD002078
:1012900003F090FD152003F08DFD172003F08AFD6B
:1012A000072003F087FD112003F084FD062003F0E2
:1012B00081FD2B2003F07EFD562003F07BFD3C20BA
:1012C00003F078FD052003F075FD102003F072FD9A
:1012D0000F2003F06FFD3F2003F06CFD3F2003F073
:1012E00069FD0F2003F066FD2B2003F069FD00204F
:1012F00003F060FD002003F05DFD012003F05AFDC6
:101300003F2003F057FD2A2003F05AFD002003F090
:1013100051FD002003F04EFD002003F04BFDEF20B7
:1013200003F048FD112003F04BFD782004F030FB62
:10133000292003F045FD03F019B9FE488088A0F587
:10134000D04104397ED1112003F03AFD142004F07D
:101350001FFBD02003F034FD072003F02BFD4220BB
:1013600003F028FD1D2003F025FDD12003F028FD0A
:10137000002003F01FFD1A2003F01CFD092003F0DC
:1013800019FDD22003F01CFD012003F013FD2220E3
:1013900003F010FDC02003F013FD102003F00AFD40
:1013A0003B2003F007FD002003F004FD022003F0C2
:1013B00001FD112003F0FEFCC52003F001FD032018
:1013C00003F0F8FCC82003F0FBFC002003F0F2FC63
:1013D000252003F0EFFC212003F0ECFC052003F0B6
:1013E000E9FC002003F0E6FC0A2003F0E3FC6520A2
:1013F00003F0E0FC252003F0DDFC772003F0DAFCAD
:10140000502003F0D7FC0F2003F0D4FC002003F0A1
:10141000D1FCF82003F0D4FC012003F0CBFCFE202B
:1014200003F0CEFC002003F0C5FC022003F0C2FC58
:10143000202003F0C5FC362003F0C2FC082003F096
:10144000B9FC00E02AE03A2003F0BAFC552003F092
:10145000B1FC2B2003F0B4FC002003F0ABFC002017
:1014600003F0A8FC012003F0A5FC3F2003F0A2FC40
:101470002A2003F0A5FC002003F09CFC002003F0D0
:1014800099FC012003F096FCDF2003F093FC782008
:1014900004F07EFA292003F093FC4CE7A5488088ED
:1014A000A0F5A641103940F07C87ED2003F088FCC0
:1014B000012003F07FFCFE2003F07CFCEE2003F013
:1014C0007FFCDE2003F076FC212003F073FCF1208A
:1014D00003F076FC012003F06DFCDF2003F070FCCC
:1014E000102003F067FCC42003F06AFC8F2003F097
:1014F00061FCC62003F064FC002003F05BFCE220EA
:1015000003F058FCE22003F055FCE22003F052FC0B
:10151000BF2003F055FCAA2003F04CFCB02003F0E0
:101520004FFC0D2003F046FC002003F043FC0D208F
:1015300003F040FC002003F03DFC112003F03AFCD6
:10154000002003F037FC192003F034FC002003F0E6
:1015500031FC212003F02EFC002003F02BFC2D2079
:1015600003F028FC002003F025FC3D2003F022FCC2
:10157000002003F01FFC5D2003F01CFC002003F0A2
:1015800019FC5D2003F016FC002003F013FCB120D1
:1015900003F016FC802003F00DFC002003F00AFC91
:1015A0008B2003F007FC002003F004FC962003F0DE
:1015B00001FC002003F0FEFBB22003F001FC002040
:1015C00003F0F8FB002003F0F5FB022003F0F2FB30
:1015D000002003F0EFFB032003F0ECFB002003F0FE
:1015E000E9FBB32003F0ECFB002003F0E3FB002059
:1015F00003F0E0FB002003F0DDFB002003F0DAFB4A
:10160000002003F0D7FB002003F0D4FB002003F000
:10161000D1FB002003F0CEFB002003F0CBFB002029
:1016200003F0C8FB002003F0C5FB002003F0C2FB61
:10163000002003F0BFFB002003F0BCFB002003F000
:10164000B9FB002003F0B6FB002003F0B3FB002041
:1016500003F0B0FB002003F0ADFB002003F0AAFB79
:10166000002003F0A7FB002003F0A4FB002003F000
:10167000A1FB002003F09EFBB42003F0A1FB8B2014
:1016800003F098FB002003F095FB962003F092FBFB
:10169000002003F08FFBA12003F08CFB002003F05F
:1016A00089FBB52003F08CFB022003F083FB0020B4
:1016B00003F080FB032003F07DFB002003F07AFBA6
:1016C000042003F077FB002003F074FBB62003F046
:1016D00077FB002003F06EFB002003F06BFBB720CC
:1016E00003F06EFB002003F065FB002003F062FBBB
:1016F0003F2003F05FFB002003F05CFB5E2003F063
:1017000059FB002003F056FB642003F053FB00203C
:1017100003F050FB8C2003F04DFB002003F04AFB4C
:10172000AC2003F047FB002003F044FBDC2003F077
:1017300041FB01E0A6000020002003F03BFB7020ED
:1017400003F038FB002003F035FB902003F032FB60
:10175000002003F02FFBEB2003F02CFB002003F014
:1017600029FBDC2003F026FB002003F023FBB8203C
:1017700003F026FB002003F01DFB002003F01AFB02
:10178000002003F017FB002003F014FB002003F0FF
:1017900011FB002003F00EFB002003F00BFB0020E8
:1017A00003F008FBBA2003F00BFB242003F002FB3C
:1017B000002003F0FFFA002003F0FCFA002003F001
:1017C000F9FAC12003F0FCFA202003F0F3FA00201C
:1017D00003F0F0FA542003F0EDFA002003F0EAFAE7
:1017E000FF2003F0E7FA002003F0E4FAC22003F040
:1017F000E7FA0A2003F0DEFA002003F0DBFA042007
:1018000003F0D8FA002003F0D5FAC32003F0D8FA89
:101810003C2003F0CFFA002003F0CCFA3A2003F08A
:10182000C9FA002003F0C6FA392003F0C3FA0020F9
:1018300003F0C0FA372003F0BDFA002003F0BAFA33
:101840003C2003F0B7FA002003F0B4FA362003F08E
:10185000B1FA002003F0AEFA322003F0ABFA002018
:1018600003F0A8FA2F2003F0A5FA002003F0A2FA53
:101870002C2003F09FFA002003F09CFA292003F0AB
:1018800099FA002003F096FA262003F093FA00203C
:1018900003F090FA242003F08DFA002003F08AFA76
:1018A000242003F087FA002003F084FA232003F0B9
:1018B00081FA002003F07EFA3C2003F07BFA00203E
:1018C00003F078FA362003F075FA002003F072FA7C
:1018D000322003F06FFA002003F06CFA2F2003F09F
:1018E00069FA002003F066FA2C2003F063FA002066
:1018F00003F060FA292003F05DFA002003F05AFAA1
:10190000262003F057FA002003F054FA242003F0B5
:1019100051FA002003F04EFA242003F04BFA002085
:1019200003F048FA232003F045FA002003F042FABE
:10193000C42003F045FA622003F03CFA002003F0D3
:1019400039FA052003F036FA002003F033FA842038
:1019500003F030FA002003F02DFAF02003F02AFA09
:10196000002003F027FA182003F024FA002003F0E7
:1019700021FAA42003F01EFA002003F01BFA18201D
:1019800003F018FA002003F015FA502003F012FAC1
:10199000002003F00FFA0C2003F00CFA002003F0F3
:1019A00009FA172003F006FA002003F003FA952045
:1019B00003F000FA002003F0FDF9F32003F0FAF938
:1019C000002003F0F7F9E62003F0F4F9002003F01B
:1019D000F1F9C52003F0F4F9322003F0EBF900200F
:1019E00003F0E8F9442003F0E5F9002003F0E2F900
:1019F000652003F0DFF9002003F0DCF9762003F026
:101A0000D9F9002003F0D6F9882003F0D3F900209B
:101A100003F0D0F9C62003F0D3F9202003F0CAF96F
:101A2000002003F0C7F9172003F0C4F9002003F0E9
:101A3000C1F9012003F0BEF9002003F0BBF9C72073
:101A400003F0BEF9002003F0B5F9002003F0B2F96D
:101A5000002003F0AFF9002003F0ACF9C82003F038
:101A6000AFF9002003F0A6F9002003F0A3F900204D
:101A700003F0A0F9002003F09DF9C92003F0A0F9BC
:101A8000002003F097F9002003F094F9002003F000
:101A900091F9002003F08EF9002003F08BF900206B
:101AA00003F088F9002003F085F9002003F082F9A3
:101AB000002003F07FF9002003F07CF9002003F000
:101AC00079F9002003F076F9002003F073F9002083
:101AD00003F070F9002003F06DF9002003F06AF9BB
:101AE000E02003F06DF9162003F064F9002003F004
:101AF00061F91C2003F05EF9002003F05BF921205E
:101B000003F058F9002003F055F9362003F052F99C
:101B1000002003F04FF9462003F04CF9002003F0B9
:101B200049F9522003F046F9002003F043F96420FC
:101B300003F040F9002003F03DF97A2003F03AF970
:101B4000002003F037F98B2003F034F9002003F074
:101B500031F9992003F02EF9002003F02BF9A82089
:101B600003F028F9002003F025F9B92003F022F949
:101B7000002003F01FF9C42003F01CF9002003F03B
:101B800019F9CA2003F016F9002003F013F9D22046
:101B900003F010F9002003F00DF9D92003F00AF941
:101BA000002003F007F9E02003F004F9002003F01F
:101BB00001F9F32003F0FEF8002003F0FBF8E12028
:101BC00003F0FEF8162003F0F5F8002003F0F2F819
:101BD0001C2003F0EFF8002003F0ECF8222003F0C3
:101BE000E9F8002003F0E6F8362003F0E3F80020DF
:101BF00003F0E0F8452003F0DDF8002003F0DAF808
:101C0000522003F0D7F8002003F0D4F8642003F04A
:101C1000D1F8002003F0CEF87A2003F0CBF80020B2
:101C200003F0C8F88B2003F0C5F8002003F0C2F8D9
:101C3000992003F0BFF8002003F0BCF8A82003F0BF
:101C4000B9F8002003F0B6F8B92003F0B3F800208B
:101C500003F0B0F8C42003F0ADF8002003F0AAF8B8
:101C6000CA2003F0A7F8002003F0A4F8D22003F064
:101C7000A1F8002003F09EF8D82003F09BF8002084
:101C800003F098F8E02003F095F8002003F092F8B4
:101C9000F32003F08FF8002003F08CF8E22003F02B
:101CA0008FF8052003F086F8002003F083F80B205E
:101CB00003F080F8002003F07DF81B2003F07AF891
:101CC000002003F077F8342003F074F8002003F0CC
:101CD00071F8442003F06EF8002003F06BF84F20F9
:101CE00003F068F8002003F065F8612003F062F863
:101CF000002003F05FF8792003F05CF8002003F087
:101D000059F8882003F056F8002003F053F8972084
:101D100003F050F8002003F04DF8A62003F04AF835
:101D2000002003F047F8B72003F044F8002003F048
:101D300041F8C22003F03EF8002003F03BF8C72032
:101D400003F038F8002003F035F8D12003F032F822
:101D5000002003F02FF8D62003F02CF8002003F029
:101D600029F8DD2003F026F8002003F023F8F32003
:101D700003F020F8002003F01DF8E32003F020F822
:101D8000052003F017F8002003F014F80A2003F0F0
:101D900011F8002003F00EF81C2003F00BF80020CF
:101DA00003F008F8332003F005F8002003F002F8F0
:101DB000442002F0FFFF002002F0FCFF502002F060
:101DC000F9FF002002F0F6FF622002F0F3FF00208E
:101DD00002F0F0FF782002F0EDFF002002F0EAFFB1
:101DE000882002F0E7FF002002F0E4FF972002F0D5
:101DF000E1FF002002F0DEFFA62002F0DBFF002062
:101E000002F0D8FFB72002F0D5FF002002F0D2FF89
:101E1000C22002F0CFFF002002F0CCFFC72002F06A
:101E2000C9FF002002F0C6FFD12002F0C3FF00204E
:101E300002F0C0FFD52002F0BDFF002002F0BAFF83
:101E4000DD2002F0B7FF002002F0B4FFF32002F023
:101E5000B1FF002002F0AEFFE42002F0B1FF01204C
:101E600002F0A8FF002002F0A5FF012002F0A2FF6F
:101E7000002002F09FFF022002F09CFF002002F0F1
:101E800099FF2A2002F096FF002002F093FF3C20E9
:101E900002F090FF002002F08DFF4B2002F08AFF3D
:101EA000002002F087FF5D2002F084FF002002F096
:101EB00081FF742002F07EFF002002F07BFF84206F
:101EC00002F078FF002002F075FF932002F072FF0D
:101ED000002002F06FFFA22002F06CFF002002F051
:101EE00069FFB32002F066FF002002F063FFBE200E
:101EF00002F060FF002002F05DFFC42002F05AFFF4
:101F0000002002F057FFCD2002F054FF002002F025
:101F100051FFD32002F04EFF002002F04BFFDD20E6
:101F200002F048FF002002F045FFF32002F042FFDC
:101F3000002002F03FFFE52002F042FF002002F007
:101F400039FF002002F036FF002002F033FF0020AE
:101F500002F030FF022002F02DFF002002F02AFFE5
:101F6000292002F027FF002002F024FF3C2002F08D
:101F700021FF002002F01EFF4B2002F01BFF00207B
:101F800002F018FF5D2002F015FF002002F012FFA2
:101F9000742002F00FFF002002F00CFF842002F0FA
:101FA00009FF002002F006FF932002F003FF00204B
:101FB00002F000FFA22002F0FDFE002002F0FAFE77
:101FC000B32002F0F7FE002002F0F4FEBE2002F083
:101FD000F1FE002002F0EEFEC42002F0EBFE002035
:101FE00002F0E8FECD2002F0E5FE002002F0E2FE65
:101FF000D32002F0DFFE002002F0DCFEDC2002F045
:10200000D9FE002002F0D6FEF32002F0D3FE00201D
:1020100002F0D0FEE62002F0D3FE112002F0CAFE4C
:10202000002002F0C7FE342002F0C4FE002002F0BF
:10203000C1FE562002F0BEFE002002F0BBFE76205C
:1020400002F0B8FE002002F0B5FE772002F0B2FEEA
:10205000002002F0AFFE662002F0ACFE002002F08D
:10206000A9FE882002F0A6FE002002F0A3FE99201F
:1020700002F0A0FE002002F09DFEBB2002F09AFEBE
:10208000002002F097FE992002F094FE002002F05A
:1020900091FE662002F08EFE002002F08BFE55209D
:1020A00002F088FE002002F085FE552002F082FE3C
:1020B000002002F07FFE452002F07CFE002002F0AE
:1020C00079FE432002F076FE002002F073FE4420E9
:1020D00002F070FE002002F06DFEE72002F070FEBC
:1020E000322002F067FE002002F064FE552002F06C
:1020F00061FE002002F05EFE762002F05BFE002012
:1021000002F058FE662002F055FE002002F052FE5A
:10211000672002F04FFE002002F04CFE672002F024
:1021200049FE002002F046FE872002F043FE002018
:1021300002F040FE992002F03DFE002002F03AFE3F
:10214000BB2002F037FE002002F034FE992002F09E
:1021500031FE002002F02EFE772002F02BFE002040
:1021600002F028FE442002F025FE002002F022FEAC
:10217000562002F01FFE002002F01CFE232002F079
:1021800019FE002002F016FE332002F013FE00209C
:1021900002F010FE452002F00DFE002002F00AFEC3
:1021A000E82002F00DFE002002F004FE002002F004
:1021B00001FE992002F0FEFD002002F0FBFD8720C9
:1021C00002F0F8FD002002F0F5FD882002F0F2FD9B
:1021D000002002F0EFFD772002F0ECFD002002F07D
:1021E000E9FD662002F0E6FD002002F0E3FD882014
:1021F00002F0E0FD002002F0DDFDAA2002F0DAFD91
:10220000002002F0D7FDBB2002F0D4FD002002F038
:10221000D1FD992002F0CEFD002002F0CBFD66201A
:1022200002F0C8FD002002F0C5FD552002F0C2FDFD
:10223000002002F0BFFD552002F0BCFD002002F09E
:10224000B9FD442002F0B6FD002002F0B3FD4420A9
:1022500002F0B0FD002002F0ADFD552002F0AAFD15
:10226000002002F0A7FDE92002F0AAFDAA2002F05A
:10227000A1FD002002F09EFD002002F09BFD002049
:1022800002F098FD002002F09BFDAA2002F092FDD2
:10229000CF2002F095FD002002F08CFD002002F01E
:1022A00089FD002002F086FD002002F083FD002061
:1022B00002F080FD002002F07DFD002002F07AFD9A
:1022C000002002F077FD002002F074FD002002F0F3
:1022D00071FD002002F06EFD002002F06BFD002079
:1022E00002F068FD002002F065FD002002F062FDB2
:1022F000002002F05FFD002002F05CFDF02002F003
:102300005FFD002002F056FD502002F053FD00203A
:1023100002F050FD002002F04DFD002002F04AFDC9
:10232000F32002F04DFD002002F044FDF92002F000
:1023300047FD062002F03EFD102002F03BFD292063
:1023400002F038FD002002F035FD3A2002F038FDA1
:10235000552002F02FFD112002F032FD642003F021
:1023600017FB292002F02CFD352002F029FD00206A
:1023700002F020FD512002F023FDFF2002F01AFDA3
:10238000532002F01DFD2C2002F014FD552002F018
:1023900017FD822002F00EFD2C2002F011FD02F04C
:1023A000E5B8FE488088A0F5AA4110397ED15521B4
:1023B0004FF4704002F014FDAA214FF2010002F028
:1023C0000FFD52214FF2020002F00AFD08214FF2E8
:1023D000030002F005FD01214FF2040002F000FDB0
:1023E0000D214FF4304002F0FBFC0D214BF20100B7
:1023F00002F0F6FC0D214BF2020002F0F1FC342158
:102400004FF4364002F0ECFC34214BF2016002F054
:10241000E7FC34214BF2026002F0E2FC0D214FF4A4
:10242000314002F0DDFC0D214BF2011002F0D8FC2E
:102430000D214BF2021002F0D3FC34214FF437404F
:1024400002F0CEFC34214BF2017002F0C9FC3421C1
:102450004BF2027002F0C4FC00214FF4324002F053
:10246000BFFC00214BF2012002F0BAFC00214BF22C
:10247000022002F0B5FC24214FF4384002F0B0FCF9
:1024800024214BF6010002F0ABFC24214BF60200A4
:1024900002F0A6FC01214FF43F4002F0A1FC0F2105
:1024A0004FF4334002F09CFC0F2100E0FEE34BF2BE
:1024B000013002F095FC0F214BF2023002F090FC4B
:1024C00034214FF4394002F08BFC34214BF60110DB
:1024D00002F086FC34214BF6021002F081FC082148
:1024E0004FF4354002F07CFC08214BF2015002F021
:1024F00077FC08214BF2025002F072FC03214FF4EA
:10250000424002F06DFC24214FF43A4002F068FC96
:1025100024214BF6012002F063FC24214BF602201B
:1025200002F05EFC00214FF43C4002F059FC78219F
:102530004BF6014002F054FC00214BF6024002F041
:102540004FFC00214FF43D4002F04AFC78214BF64D
:10255000015002F045FC00214BF6025002F040FC15
:1025600000214FF43E4002F03BFC64214BF6016039
:1025700002F036FC00214FF4514002F031FC3321CF
:102580004DF2011002F02CFC00214DF2021002F07D
:1025900027FC34214DF2031002F022FC00214DF201
:1025A000041002F01DFC3A214DF2051002F018FC57
:1025B00000214DF2061002F013FC4A214DF20710E3
:1025C00002F00EFC00214DF2081002F009FC5C2123
:1025D0004DF2091002F004FC00214DF20A1002F045
:1025E000FFFB81214DF20B1002F0FAFB00214DF2AE
:1025F0000C1002F0F5FBA6214DF20D1002F0F0FBDD
:1026000000214DF20E1002F0EBFBE5214DF20F1010
:1026100002F0E6FB01214DF2101002F0E1FB132164
:102620004DF2111002F0DCFB01214DF2121002F00C
:10263000D7FB54214DF2131002F0D2FB01214DF2D1
:10264000141002F0CDFB82214DF2151002F0C8FBF0
:1026500001214DF2161002F0C3FBCA214DF21710F2
:1026600002F0BEFB02214DF2181002F0B9FB00216E
:102670004DF2191002F0B4FB02214DF21A1002F0D3
:10268000AFFB01214DF21B1002F0AAFB02214DF21B
:102690001C1002F0A5FB34214DF21D1002F0A0FB2E
:1026A00002214DF21E1002F09BFB67214DF21F101C
:1026B00002F096FB02214DF2201002F091FB8421E2
:1026C0004DF2211002F08CFB02214DF2221002F09B
:1026D00087FBA4214DF2231002F082FB02214DF270
:1026E000241002F07DFBB7214DF2251002F078FB9B
:1026F00002214DF2261002F073FBCF214DF227107C
:1027000002F06EFB02214DF2281002F069FBDE217F
:102710004DF2291002F064FB02214DF22A1002F062
:102720005FFBF2214DF22B1002F05AFB02214DF219
:102730002C1002F055FBFE214DF22D1002F050FB43
:1027400003214DF22E1002F04BFB10214DF22F1001
:1027500002F046FB03214DF2301002F041FB332121
:102760004DF2311002F03CFB03214DF2321002F029
:1027700037FB6D214DF2331002F032FB00214FF494
:10278000524002F02DFB33214DF2012002F028FBD4
:1027900000214DF2022002F023FB01E0A600002000
:1027A00034214DF2032002F01BFB00214DF20420E6
:1027B00002F016FB3A214DF2052002F011FB002138
:1027C0004DF2062002F00CFB4A214DF2072002F0E8
:1027D00007FB00214DF2082002F002FB5C214DF2C4
:1027E000092002F0FDFA00214DF20A2002F0F8FA69
:1027F00081214DF20B2002F0F3FA00214DF20C2062
:1028000002F0EEFAA6214DF20D2002F0E9FA0021C5
:102810004DF20E2002F0E4FAE5214DF20F2002F015
:10282000DFFA01214DF2102002F0DAFA13214DF205
:10283000112002F0D5FA01214DF2122002F0D0FA57
:1028400054214DF2132002F0CBFA01214DF2142055
:1028500002F0C6FA82214DF2152002F0C1FA0121E0
:102860004DF2162002F0BCFACA214DF2172002F0F8
:10287000B7FA02214DF2182002F0B2FA00214DF20F
:10288000192002F0ADFA02214DF21A2002F0A8FA46
:1028900001214DF21B2002F0A3FA02214DF21C206F
:1028A00002F09EFA34214DF21D2002F099FA022125
:1028B0004DF21E2002F094FA67214DF21F2002F023
:1028C0008FFA02214DF2202002F08AFA84214DF283
:1028D000212002F085FA02214DF2222002F080FA36
:1028E000A4214DF2232002F07BFA02214DF2242094
:1028F00002F076FAB7214DF2252002F071FA02219A
:102900004DF2262002F06CFACF214DF2272002F082
:1029100067FA02214DF2282002F062FADE214DF220
:10292000292002F05DFA02214DF22A2002F058FA25
:10293000F2214DF22B2002F053FA02214DF22C200D
:1029400002F04EFAFE214DF22D2002F049FA032149
:102950004DF22E2002F044FA10214DF22F2002F009
:102960003FFA03214DF2302002F03AFA33214DF2C2
:10297000312002F035FA03214DF2322002F030FA14
:102980006D214DF2332002F02BFA00214FF4534019
:1029900002F026FA33214DF2013002F021FA002133
:1029A0004DF2023002F01CFA34214DF2033002F0F5
:1029B00017FA00214DF2043002F012FA3A214DF2DA
:1029C000053002F00DFA00214DF2063002F008FA4F
:1029D0004A214DF2073002F003FA00214DF208308F
:1029E00002F0FEF95C214DF2093002F0F9F9002104
:1029F0004DF20A3002F0F4F981214DF20B3002F071
:102A0000EFF900214DF20C3002F0EAF9A6214DF267
:102A10000D3002F0E5F900214DF20E3002F0E0F940
:102A2000E5214DF20F3002F0DBF901214DF21030BB
:102A300002F0D6F913214DF2113002F0D1F9012143
:102A40004DF2123002F0CCF954214DF2133002F065
:102A5000C7F901214DF2143002F0C2F982214DF282
:102A6000153002F0BDF901214DF2163002F0B8F92F
:102A7000CA214DF2173002F0B3F902214DF218309D
:102A800002F0AEF900214DF2193002F0A9F902214D
:102A90004DF21A3002F0A4F901214DF21B3002F080
:102AA0009FF902214DF21C3002F09AF934214DF2C7
:102AB0001D3002F095F902214DF21E3002F090F91E
:102AC00067214DF21F3002F08BF902214DF22030C8
:102AD00002F086F984214DF2213002F081F90221C1
:102AE0004DF2223002F07CF9A4214DF2233002F0A5
:102AF00077F902214DF2243002F072F9B7214DF23C
:102B0000253002F06DF902214DF2263002F068F90D
:102B1000CF214DF2273002F063F902214DF2283027
:102B200002F05EF9DE214DF2293002F059F902215E
:102B30004DF22A3002F054F9F2214DF22B3002F01E
:102B40004FF902214DF22C3002F04AF9FE214DF2EC
:102B50002D3002F045F903214DF22E3002F040F9FC
:102B600010214DF22F3002F03BF903214DF23030AD
:102B700002F036F933214DF2313002F031F9032100
:102B80004DF2323002F02CF96D214DF2333002F06B
:102B900027F900214FF4544002F022F933214DF27D
:102BA000014002F01DF900214DF2024002F018F937
:102BB00034214DF2034002F013F900214DF204409C
:102BC00002F00EF93A214DF2054002F009F9002118
:102BD0004DF2064002F004F94A214DF2074002F09E
:102BE000FFF800214DF2084002F0FAF85C214DF2A6
:102BF000094002F0F5F800214DF20A4002F0F0F829
:102C000081214DF20B4002F0EBF800214DF20C4017
:102C100002F0E6F8A6214DF20D4002F0E1F80021A5
:102C20004DF20E4002F0DCF8E5214DF20F4002F0CB
:102C3000D7F801214DF2104002F0D2F813214DF2E5
:102C4000114002F0CDF801214DF2124002F0C8F817
:102C500054214DF2134002F0C3F801214DF214400B
:102C600002F0BEF882214DF2154002F0B9F80121C0
:102C70004DF2164002F0B4F8CA214DF2174002F0AE
:102C8000AFF802214DF2184002F0AAF800214DF2EF
:102C9000194002F0A5F802214DF21A4002F0A0F806
:102CA00001214DF21B4002F09BF800E004E30221F9
:102CB0004DF21C4002F094F834214DF21D4002F018
:102CC0008FF802214DF21E4002F08AF867214DF282
:102CD0001F4002F085F802214DF2204002F080F8FA
:102CE00084214DF2214002F07BF802214DF2224076
:102CF00002F076F8A4214DF2234002F071F802218F
:102D00004DF2244002F06CF8B7214DF2254002F05C
:102D100067F802214DF2264002F062F8CF214DF211
:102D2000274002F05DF802214DF2284002F058F8E9
:102D3000DE214DF2294002F053F802214DF22A40E3
:102D400002F04EF8F2214DF22B4002F049F8022138
:102D50004DF22C4002F044F8FE214DF22D4002F0DD
:102D60003FF803214DF22E4002F03AF810214DF2C7
:102D70002F4002F035F803214DF2304002F030F8D8
:102D800033214DF2314002F02BF803214DF2324055
:102D900002F026F86D214DF2334002F021F80021B7
:102DA0004FF4554002F01CF833214DF2015002F06F
:102DB00017F800214DF2025002F012F834214DF2C2
:102DC000035002F00DF800214DF2045002F008F813
:102DD0003A214DF2055002F003F800214DF2065061
:102DE00001F0FEFF4A214DF2075001F0F9FF0021EA
:102DF0004DF2085001F0F4FF5C214DF2095001F052
:102E0000EFFF00214DF20A5001F0EAFF81214DF25F
:102E10000B5001F0E5FF00214DF20C5001F0E0FFF6
:102E2000A6214DF20D5001F0DBFF00214DF20E50B6
:102E300001F0D6FFE5214DF20F5001F0D1FF012145
:102E40004DF2105001F0CCFF13214DF2115001F062
:102E5000C7FF01214DF2125001F0C2FF54214DF283
:102E6000135001F0BDFF01214DF2145001F0B8FFE5
:102E700082214DF2155001F0B3FF01214DF21650A1
:102E800001F0AEFFCA214DF2175001F0A9FF022157
:102E90004DF2185001F0A4FF00214DF2195001F03D
:102EA0009FFF02214DF21A5001F09AFF01214DF2CD
:102EB0001B5001F095FF02214DF21C5001F090FFD4
:102EC00034214DF21D5001F08BFF02214DF21E50B6
:102ED00001F086FF67214DF21F5001F081FF0221B2
:102EE0004DF2205001F07CFF84214DF2215001F081
:102EF00077FF02214DF2225001F072FFA4214DF222
:102F0000235001F06DFF02214DF2245001F068FFC3
:102F1000B7214DF2255001F063FF02214DF22650FA
:102F200001F05EFFCF214DF2275001F059FF022141
:102F30004DF2285001F054FFDE214DF2295001F0EE
:102F40004FFF02214DF22A5001F04AFFF2214DF2CB
:102F50002B5001F045FF02214DF22C5001F040FFB3
:102F6000FE214DF22D5001F03BFF03214DF22E507A
:102F700001F036FF10214DF22F5001F031FF0321F7
:102F80004DF2305001F02CFF33214DF2315001F061
:102F900027FF03214DF2325001F022FF6D214DF247
:102FA000335001F01DFF00214FF4564001F018FF8F
:102FB00033214DF2016001F013FF00214DF2026058
:102FC00001F00EFF34214DF2036001F009FF0021F2
:102FD0004DF2046001F004FF3A214DF2056001F06A
:102FE000FFFE00214DF2066001F0FAFE4A214DF28B
:102FF000076001F0F5FE00214DF2086001F0F0FEDF
:103000005C214DF2096001F0EBFE00214DF20A60F7
:1030100001F0E6FE81214DF20B6001F0E1FE00219E
:103020004DF20C6001F0DCFEA6214DF20D6001F0C6
:10303000D7FE00214DF20E6001F0D2FEE5214DF2E7
:103040000F6001F0CDFE01214DF2106001F0C8FECD
:1030500013214DF2116001F0C3FE01214DF2126007
:1030600001F0BEFE54214DF2136001F0B9FE0121C2
:103070004DF2146001F0B4FE82214DF2156001F0B2
:10308000AFFE01214DF2166001F0AAFECA214DF2F9
:10309000176001F0A5FE02214DF2186001F0A0FEBC
:1030A00000214DF2196001F09BFE02214DF21A60E1
:1030B00001F096FE01214DF21B6001F091FE02210C
:1030C0004DF21C6001F08CFE34214DF21D6001F0C8
:1030D00087FE02214DF21E6001F082FE67214DF253
:1030E0001F6001F07DFE02214DF2206001F078FEAC
:1030F00084214DF2216001F073FE02214DF2226025
:1031000001F06EFEA4214DF2236001F069FE022160
:103110004DF2246001F064FEB7214DF2256001F00C
:103120005FFE02214DF2266001F05AFECF214DF2E2
:10313000276001F055FE02214DF2286001F050FE9B
:10314000DE214DF2296001F04BFE02214DF22A6092
:1031500001F046FEF2214DF22B6001F041FE02210A
:103160004DF22C6001F03CFEFE214DF22D6001F08D
:1031700037FE03214DF22E6001F032FE10214DF298
:103180002F6001F02DFE03214DF2306001F028FE8A
:1031900033214DF2316001F023FE03214DF2326004
:1031A00001F01EFE6D214DF2336001F019FE552134
:1031B0004FF4704001F014FEAA214FF2010001F01B
:1031C0000FFE52214FF2020001F00AFE08214FF2D9
:1031D000030001F005FE00214FF2040001F000FEA3
:1031E000CC214FF4314001F0FBFD00214BF20110E6
:1031F00001F0F6FD05214FF4364001F0F1FD70219C
:103200004FF4374001F0ECFD70214BF2017001F0FA
:10321000E7FD01214FF4384001F0E2FD03214BF6B8
:10322000010001F0DDFD03214BF6020001F0D8FDA5
:1032300003214BF6030001F0D3FD02214FF43C4083
:1032400001F0CEFD00214BF6014001F0C9FD002147
:103250004BF6024001F0C4FDD0214FF4494001F08B
:10326000BFFD02214CF6011001F0BAFD50214CF6D1
:10327000021001F0B5FD50214CF6031001F0B0FD35
:1032800050214CF6041001F0ABFD00214FF45450D6
:1032900001F0A6FD55214FF4685001F0A1FD4FF457
:1032A000885001F08DFD782002F08DFB4FF4245002
:1032B00001F086FD01F05AB9FE488088A0F513415F
:1032C00025397DD147F6F001E52001F089FD4FF465
:1032D0008071012001F084FD4FF4E061022001F0D3
:1032E0007FFD41F23001032001F07AFD002104202E
:1032F00001F076FD40F20221082001F071FD00216D
:10330000092001F06DFD00210A2001F069FD002176
:103310000C2001F065FD00210D2001F061FD002170
:103320000F2001F05DFD0021102001F059FD072163
:10333000112001F055FD0021122001F051FD002166
:10334000132001F04DFD0021072001F049FD41F25D
:103350009061102001F044FD40F22721112001F07E
:103360003FFD9D21122001F03BFD4FF4C851132079
:1033700001F036FD2521292001F032FD0D212B2001
:1033800001F02EFD0721302001F02AFD40F203312B
:10339000312001F025FD0321322001F021FD40F212
:1033A0000621352001F01CFD0821362001F018FD12
:1033B00040F20641372001F013FD4FF4417100E067
:1033C00058E0382001F00CFD0721392001F008FDFC
:1033D00040F202613C2001F003FD08213D2001F094
:1033E000FFFC0021502001F0FBFCEF21512001F0F7
:1033F000F7FC0021522001F0F3FC40F23F11532072
:1034000001F0EEFC4FF42741602001F0E9FC0121BE
:10341000612001F0E5FC00216A2001F0E1FC0021BF
:10342000802001F0DDFC0021812001F0D9FC002189
:10343000822001F0D5FC0021832001F0D1FC002185
:10344000842001F0CDFC0021852001F0C9FC102171
:10345000902001F0C5FC4FF4C061922001F0C0FC47
:1034600040F23311072001F0BBFC2221002001F0C3
:10347000B7FC1FE78F488088A0F5134128397DD11C
:1034800041F28F01EC2001F0ABFC41F23421EF203E
:1034900001F0A6FC4FF48071012001F0A1FC4FF473
:1034A000E061022001F09CFC41F23001032001F0B8
:1034B00097FC0021042001F093FC40F20221082037
:1034C00001F08EFC0021092001F08AFC00210A2075
:1034D00001F086FC01210C2001F082FC00210D206E
:1034E00001F07EFC00210F2001F07AFC0021102069
:1034F00001F076FC0721112001F072FC002112205E
:1035000001F06EFC0021132001F06AFC012107206C
:1035100001F066FC322002F03BFA41F290411020AB
:1035200001F05EFC40F22721112001F059FC32200D
:1035300002F02EFA8A21122001F052FC322002F011
:1035400027FA4FF4D051132001F04AFC062129201C
:1035500001F046FC0D212B2001F042FC322002F04C
:1035600017FA0021202001F03BFC0021212001F06E
:1035700037FC322002F00CFA002100E075E0302028
:1035800001F02EFC40F20461312001F029FC40F2F0
:103590000531322001F024FC0021352001F020FC0F
:1035A00040F60941362001F01BFC4FF40171372031
:1035B00001F016FC40F20131382001F011FC40F21C
:1035C0000771392001F00CFC00213C2001F008FCBF
:1035D00040F60A213D2001F003FC322002F0D8F928
:1035E0000021502001F0FCFBEF21512001F0F8FBFD
:1035F0000021522001F0F4FB40F23F11532001F072
:10360000EFFB4FF42741602001F0EAFB012161202C
:1036100001F0E6FB00216A2001F0E2FB002180209E
:1036200001F0DEFB0021812001F0DAFB0021822085
:1036300001F0D6FB0021832001F0D2FB0021842081
:1036400001F0CEFB0021852001F0CAFB1021902063
:1036500001F0C6FB4FF4C061922001F0C1FB40F2C3
:103660003311072001F0BCFB24E612488088A0F546
:10367000134120397ED1084601F0B2FB4FF480712E
:10368000012001F0ADFB4FF4E061022001F0A8FB46
:1036900041F23001032001F0A3FB0021042001F0DE
:1036A0009FFB40F20221082001F09AFB0021092033
:1036B00002E00000A600002001F092FB00210A2099
:1036C00001F08EFB01210C2001F08AFB00210D206E
:1036D00001F086FB00210F2001F082FB322002F076
:1036E00057F940F20111072001F07AFB322002F075
:1036F0004FF94FF48651102001F072FB0721112081
:1037000001F06EFB4FF48871122001F069FB4FF459
:103710003061132001F064FB0021292001F060FBDF
:1037200044F210012B2001F05BFB0021502001F03E
:1037300057FBEF21512001F053FB0021522001F0F3
:103740004FFB40F23F11532001F04AFB4FF41C5154
:10375000602001F045FB0121612001F041FB0021C7
:103760006A2001F03DFB0021802001F039FB00219F
:10377000812000E030E001F033FB0021822001F0E5
:103780002FFB0021832001F02BFB0021842001F07E
:1037900027FB0021852001F023FB1021902001F060
:1037A0001FFB0021922001F01BFB0121932001F05F
:1037B00017FB4FF48871952001F012FB0021972030
:1037C00001F00EFB0021982001F00AFB40F273117A
:1037D000072001F005FB6DE5FE488088A0F5134148
:1037E00031397DD141F21401E72001F0F9FA4FF4AB
:1037F0008071012001F0F4FA4FF40071022001F011
:10380000EFFA41F23801032001F0EAFA40F2022116
:10381000082001F0E5FA0021092001F0E1FA002179
:103820000A2001F0DDFA00210C2001F0D9FA002174
:103830000D2001F0D5FA00210F2001F0D1FA00216E
:10384000102001F0CDFA0721112001F0C9FA002162
:10385000122001F0C5FA0021132001F0C1FAC8209E
:1038600002F096F841F29061102001F0B9FA40F2AE
:103870002721112001F0B4FA322002F089F80C213E
:10388000122001F0ADFA322002F082F84FF400610C
:10389000132001F0A5FA1121292001F0A1FA0B2132
:1038A0002B2001F09DFA322002F072F80021202036
:1038B00001F096FA40F23F11212001F091FA002127
:1038C000302001F08DFA4FF48371312001F088FA35
:1038D0000021322001F084FA4FF40171352000E01C
:1038E00064E001F07DFA41F20A61362001F078FAD5
:1038F00040F20771372001F073FA4FF483713820DA
:1039000001F06EFA40F20771392001F069FA40F2D5
:1039100002413C2001F064FA40F60F413D2001F0E5
:103920005FFA0021502001F05BFAEF21512001F0F5
:1039300057FA0021522001F053FA40F23F11532070
:1039400001F04EFA4FF41C51602001F049FA0121B8
:10395000612001F045FA00216A2001F041FA0021BE
:10396000802001F03DFA0021812001F039FA002188
:10397000822001F035FA0021832001F031FA002184
:10398000842001F02DFA0021852001F029FA102170
:10399000902001F025FA4FF4C061922001F020FA46
:1039A00040F23311072001F01BFA83E48948808834
:1039B000A0F5A84108397DD14FF48071012001F0B4
:1039C0000FFA4FF4E061022001F00AFA41F23001EF
:1039D000032001F005FA0021042001F001FA40F271
:1039E0000721082001F0FCF90021092001F0F8F975
:1039F00000210A2001F0F4F900210C2001F0F0F977
:103A000000210D2001F0ECF900210F2001F0E8F970
:103A1000142001F0BDFF41F2B061102001F0E0F987
:103A20000121112001F0DCF90121172001F0D8F962
:103A30004FF49C71122001F0D3F94FF40061132070
:103A400001F0CEF90921292001F0CAF909212A2023
:103A500001F0C6F90021A42001F0C2F90021502094
:103A600001F0BEF9EF21512001F0BAF900215220F6
:103A700001F0B6F940F23F11532001F0B1F94FF4D3
:103A80001C51602001F0ACF90121612001F0A8F97E
:103A900000216A2001F0A4F90021802001F0A0F9A2
:103AA0000021812001F09CF90021822001F098F989
:103AB000002100E024E0832001F092F9002184201D
:103AC00001F08EF90021852001F08AF91321902060
:103AD00001F086F90021922001F082F90321932060
:103AE00001F07EF94FF48871952001F079F940F2E8
:103AF0007311072001F074F9322001F049FFB8E496
:103B000034488088A0F5A851053965D1072001F017
:103B100067F9322001F03CFF4FF48E71122001F062
:103B20005FF90121A42001F05BF90F21082001F0C9
:103B300057F908210A2001F053F908210D2001F05E
:103B40004FF940F20771302001F04AF90721312086
:103B500001F046F940F20361322001F041F94FF4DF
:103B6000E061332001F03CF940F20221342001F001
:103B700037F90221352001F033F941F60F71362073
:103B800001F02EF940F20771372001F029F90021E8
:103B9000382001F025F90021392001F021F940F207
:103BA00007713A2001F01CF900213B2001F018F9BF
:103BB00007213C2001F014F900213D2001F010F90B
:103BC000322001F0E5FE0121072001F009F9012171
:103BD000172002E0A6000020AEE001F001F932203B
:103BE00001F0D6FE4FF4BD51102001F0F9F840F27B
:103BF0001721112001F0F4F84FF48F71122001F019
:103C0000EFF84FF47061132001F0EAF800212A2048
:103C100001F0E6F80A21292001F0E2F84FF49F7143
:103C2000122001F0DDF80021502001F0D9F8EF2139
:103C3000512001F0D5F80021522001F0D1F840F2D6
:103C40003F11532001F0CCF84FF41C51602001F0DB
:103C5000C7F80121612001F0C3F800216A2001F0BA
:103C6000BFF80021802001F0BBF80021812001F085
:103C7000B7F80021822001F0B3F80021832001F081
:103C8000AFF80021842001F0ABF80021852001F07D
:103C9000A7F81321902001F0A3F84FF4407192206F
:103CA00001F09EF80521932001F09AF8002195205B
:103CB00001F096F80021972001F092F80021982059
:103CC00001F08EF84FF48071012001F089F84FF473
:103CD000E061022001F084F841F23801032001F094
:103CE0007FF80021042001F07BF800210C2001F076
:103CF00077F800210F2001F073F80021202001F057
:103D00006FF80021212001F06BF82121072001F03C
:103D100067F8142001F03CFE6121072001F060F8F3
:103D2000142001F035FE40F27311072001F058F81D
:103D3000142001F02DFE97E4FE488088A0F535415F
:103D400005397DD1084601F04BF80021084601F005
:103D500047F80021084601F043F80021084601F029
:103D60003FF80121A42001F03BF8142001F010FEDF
:103D70004FF41C51602001F033F840F2022108207A
:103D800001F02EF84FF40571302001F029F843F2CC
:103D90001571312001F024F840F20461322001F065
:103DA0001FF840F61661332001F01AF842F2112193
:103DB000342001F015F84FF4A851352001F010F827
:103DC00048F20751362001F00BF841F20741372045
:103DD00001F006F841F20341382001F001F82021FA
:103DE000392000F0FDFF1A21902000F0F9FF00219A
:103DF000102000F0F5FF0721112000F0F1FF002155
:103E0000122000F0EDFF0021132000F0E9FF142044
:103E100001F0BEFD4FF4E661102000F0E1FF40F23A
:103E20003711112000F0DCFF142001F0B1FD4FF438
:103E3000DC71122000F0D4FF142001F0A9FD00E095
:103E400083E04FF47061132000F0CAFF80212A2024
:103E500000F0C6FF4821292000F0C2FF142001F025
:103E600097FD4FF48071012000F0BAFF4FF4E0613C
:103E7000022000F0B5FF41F23801032000F0B0FF4E
:103E800040F20221082000F0ABFF00210A2000F0E0
:103E9000A7FF00210C2000F0A3FF00210D2000F05F
:103EA0009FFF30210E2000F09BFF0021502000F0EA
:103EB00097FFEF21512000F093FF0021522000F0E6
:103EC0008FFF40F23F11532000F08AFF4FF41C5146
:103ED000602000F085FF0121612000F081FF0021BA
:103EE0006A2000F07DFF1121902000F079FF4FF44F
:103EF000C061922000F074FF40F20241932000F074
:103F00006FFF0221942000F06BFF142001F040FDB0
:103F10000121072000F064FF142001F039FD612128
:103F2000072000F05DFF40F27311072000F058FFFA
:103F30000021202000F054FF0021212000F050FF3C
:103F40002221002000F04CFF10E37A488088A0F581
:103F5000454105397DD1084600F042FF0021084661
:103F600000F03EFF142001F013FD0021084600F090
:103F700037FF0021084600F033FF0021084600F01B
:103F80002FFF0021084600F02BFF0121A42000F0A4
:103F900027FF142001F0FCFC4FF41C51602000F0BE
:103FA0001FFF40F60601082000F01AFF40F20371DF
:103FB000302000F015FF0121312000F011FF042115
:103FC000322000F00DFF4FF48171332000F008FF24
:103FD0004FF44071342000F003FF40F2031135200C
:103FE00000F0FEFE1F21362000F0FAFE40F20371C1
:103FF000372000F0F5FE0121382000F0F1FE042109
:10400000392000F0EDFE1521902000F0E9FE4FF47C
:104010008261102000F0E4FE40F24721112000F000
:10402000DFFE4FF4DE71122000F0DAFE4FF4606123
:10403000132000F0D5FE782001F0AAFC4FF4807127
:10404000012000F0CDFE4FF40071022000F0C8FE08
:1040500000E050E041F23001032000F0C1FE0821F1
:104060000A2000F0BDFE00210C2000F0B9FE202146
:104070000E2000F0B5FE00210F2000F0B1FE00215F
:10408000202000F0ADFE0021212000F0A9FE3D21FE
:104090002A2000F0A5FE142001F07AFC2D21292011
:1040A00000F09EFE0021502000F09AFE4DF2EF013C
:1040B000512000F095FE0021522000F091FE40F2C8
:1040C0003F11532000F08CFE0021612000F088FE9B
:1040D00000216A2000F084FE4FF44071922000F02D
:1040E0007FFE0521932000F07BFE4FF480710720B6
:1040F00000F076FE3AE20F488088A0F58A41313917
:104100007ED10121002000F06BFE0A2001F040FC6E
:1041100041F22861102000F063FE0E21122000F011
:104120005FFE40F63921132000F05AFE0A2001F00C
:104130002FFC01E0A60000204021112000F050FEDD
:104140005021152000F04CFE0A2001F021FC1E2118
:10415000122000F045FE0A2001F01AFC4FF4B15184
:10416000102000F03DFE42F63921132000F038FE09
:104170000A2001F00DFC4FF48071012000F030FEA8
:104180004FF44071022000F02BFE41F23801032071
:1041900000F026FE40F20221082000F021FE082156
:1041A0000A2000F01DFE0021302000F019FE40F230
:1041B0000241312000F014FE4FF48371322000F0F0
:1041C0000FFE40F20351332000F00AFE4FF48271DB
:1041D000342000F005FE40F20131352000F000FEF1
:1041E00040F20771362000F0FBFD40F20531372028
:1041F00000F0F6FD4FF40271382000F0F1FD00E010
:104200003EE040F60B71392000F0EAFD022141202A
:1042100000F0E6FD4FF41C51602000F0E1FD0121AB
:10422000612000F0DDFD4FF40471902000F0D8FD16
:104230004FF48571922000F0D3FD0421932000F00B
:10424000CFFD4FF48071A02000F0CAFD01210720AE
:1042500000F0C6FD2121072000F0C2FD2321072028
:1042600000F0BEFD3321072000F0BAFD40F233110B
:10427000072000F0B5FD0021A02000F0B1FD75E1A0
:10428000C0488088A0F58A4135397CD1302115207D
:1042900000F0A6FD10219A2000F0A2FD202111209F
:1042A00000F09EFD43F22841102000F099FD02210C
:1042B000122000F095FD41F23801132000F090FD2E
:1042C000282001F065FB1221084600F089FD282016
:1042D00001F05EFB43F22041102000F081FD43F22B
:1042E0003801132000F07CFD462001F051FB002135
:1042F000302000F075FD40F20241312000F070FDE9
:1043000040F20731322000F06BFD4FF44171332051
:1043100000F066FD0421342000F062FD40F201410E
:10432000352000F05DFD40F20771362000F058FDA9
:1043300040F20531372000F053FD4FF4C2613820C0
:1043400000F04EFD4FF4C261392000F049FD4FF4FA
:104350008071012000F044FD4FF44071022000F014
:104360003FFD41F23001032000F03AFD40F6080124
:10437000082000F035FD08210A2000F031FD4FF43F
:104380001C51602000E033E000F02AFD0121612093
:1043900000F026FD4FF49F71902000F021FD4FF4B6
:1043A0008071922000F01CFD4FF48071932000F08A
:1043B00017FD4FF44051A02000F012FD1021A32062
:1043C00000F00EFD0121072000F00AFD2121072049
:1043D00000F006FD2321072000F002FD3321072015
:1043E00000F0FEFC40F23311072000F0F9FCBDE0C4
:1043F00064488088A0F5C8516339F8D1E22000F004
:10440000DFFC1D2000F0D6FC022000F0D3FC0420CD
:1044100000F0D0FC642001F0D6FAE02000F0D0FCDF
:10442000012000F0C7FC0A2001F0B2FAE02000F001
:10443000C7FC032000F0BEFC0C2001F0A9FA01200B
:1044400000F0BEFC0A2001F0A3FAE62000F0B8FC60
:104450002F2000F0AFFCFF2000F0ACFCFF2000F0AC
:10446000A9FCB02000F0ACFC202000F0A3FC002050
:1044700000F0A0FC032000F09DFC40F21F3000F093
:1044800099FC012000F096FC40F2DF1000F092FC55
:10449000002000F08FFCB42000F092FC042000F01B
:1044A00089FC40F21F4000F085FC002000F082FCF7
:1044B0002E2000F07FFC002000F07CFC002000F0AB
:1044C00079FC002000F076FC002000F073FCB620A0
:1044D00000F076FC022000F06DFC4FF4037000F059
:1044E00069FC002000F066FC172000F063FC15203A
:1044F00000F060FC002000F05DFC002000F05AFCA1
:10450000F02000F05DFC032000F054FC292000F0B6
:1045100057FCD02000F054FC002000F04BFCBE20E3
:1045200000F04EFC052000F045FCFE2000F042FCAF
:10453000012000F03FFC002000F03CFC002000F0D7
:1045400039FC002000F036FCB82000F039FC0320D4
:1045500000F030FC012000F02DFCBA2000F030FC0F
:10456000012000F027FC642000F032F80020FCF766
:10457000FBF90120044908604FF6FF70FCF7BEF913
:104580001FB000BDA60000208081214210B5024668
:10459000012000E050430B00A1F10104E1B2F9D188
:1045A00010BD000008B5034800880090BDF8000069
:1045B00008BD00000008006C10B50446204600F05D
:1045C000FFFB052001F0FFF9FFF7ECFF10BD000035
:1045D0002DE9F0470446BE2000F0F2FB052000F074
:1045E000E9FB2046FBF744FE07464FF066320C4BD2
:1045F000FBF7CCFD0546FBF748FE1FFA80F948465D
:1046000000F0D8FB012000F0D5FBFF2000F0D2FB2A
:10461000002000F0CFFB002000F0CCFBBDE8F087CD
:1046200066660440F0B5054600240027B748807947
:1046300001280BD1B5488088A0F5D041043905D0B8
:10464000B2488088A0F5C851633908D1AF48807955
:10465000F0B9AE488088A0F5C851633918D1082D4B
:1046600015D2DFE805F00406080A0C0E1012062524
:104670000DE007250BE0042509E0052507E00125ED
:1046800005E0002503E0032501E0022500BF00BF8F
:104690009E488088A0F51341413917D09B488088F7
:1046A000A0F5D041043911D098488088A0F5A641E2
:1046B00010390BD095488088A0F5AA41103905D053
:1046C00092488088A0F5C85163397DD1082D1CD24D
:1046D000DFE805F00406090C0F12151800BF14E0FE
:1046E00044F0800411E044F040040EE044F0C004C3
:1046F0000BE044F0200408E044F0600405E044F0DE
:10470000A00402E044F0E00400BF00BF7F488088BE
:10471000A0F5AA41103902D14FF4585700E03627CE
:104720007A488088A0F5A64110390DD07748808856
:10473000A0F5AA41103907D074488088A0F5C85167
:10474000633901D044F0080470488088A0F5D04156
:10475000043901D144F002042146384600F040FB00
:104760006A488088A0F5C85163391DD014F0200F25
:104770000DD06648008865494988884214DA634844
:104780000688408861490880084646800CE05F48FA
:1047900000885E494988884206DD5C480688408872
:1047A0005A4908800846468058488088A0F5AA41A2
:1047B000103954D15549488900F002FB002000F01F
:1047C000F9FA5249498900E078E0491C88B200F0C2
:1047D000F7FA002000F0EEFA4C494989891C88B2AA
:1047E00000F0EEFA49490988491EC1F30F2000F094
:1047F000E1FA46494989C91C88B200F0E1FA434907
:104800000978491EC8B200F0D5FA4049888900F0FD
:10481000D7FA002000F0CEFA3C498989491C88B2B9
:1048200000F0CEFA002000F0C5FA38498989891CC9
:1048300088B200F0C5FA35494988491EC1F30F20F6
:1048400000F0B8FA31498989C91C88B200F0B8FA79
:104850002E498978491EC8B200F0ACFA55E02B49C0
:10486000488900F0ADFA002000F0A4FA002000F022
:10487000A1FA26490988491EC1F30F2000F09AFACF
:1048800022490978491EC8B200F094FA1F49888964
:1048900000F096FA002000F08DFA002000F08AFA6D
:1048A0001A494988491EC1F30F2000F083FA1749BD
:1048B0008978491EC8B200F07DFA26E0082D1CD286
:1048C000DFE805F004070A0D0F12151844F0300454
:1048D00013E044F0100410E044F020040DE000BFA9
:1048E0000BE044F0380408E044F0280405E044F00C
:1048F000180402E044F0080400BF00BF032744F49A
:1049000080542146384600F06BFAF0BDA600002026
:1049100010B503460C4667488088A0F5134141391D
:1049200005D064488088A0F5A641103914D16149AA
:10493000488900F045FA181200F03CFAD8B200F0AD
:1049400039FA5C49888900F03BFA201200F032FA0B
:10495000E0B200F02FFAABE056488088A0F5D041D5
:1049600004391DD153488079012804D15148008869
:10497000401EC01A83B24F49488900F021FA18122C
:1049800000F018FAD8B200F015FA4A49888900F008
:1049900017FA201200F00EFAE0B200F00BFA87E0EE
:1049A00044488088A0F5C851633947D1414880798F
:1049B000A8B940480088401EC01A83B23D494889C2
:1049C00000F0FEF9002000F0F5F9002000F0F2F907
:1049D000181200F0EFF9D8B200F0ECF916E0354902
:1049E000488900F0EDF9181200F0E4F9D8B200F0AF
:1049F000E1F930490988491EC1F30F2000F0DAF9C6
:104A00002C490978491EC8B200F0D4F9294988898F
:104A100000F0D6F9201200F0CDF9E0B200F0CAF9AA
:104A200024494988491EC1F30F2000F0C3F92149E8
:104A30008978491EC8B200F0BDF939E01D48808868
:104A4000A0F5AA41103920D11A49488900F0B8F9D7
:104A5000181200F0AFF917494989491C88B200F0D3
:104A6000AFF9D8B200F0A6F91249888900F0A8F988
:104A7000201200F09FF90F498989491C88B200F083
:104A80009FF9E0B200F096F912E00A488079012817
:104A900004D108480088401EC01A83B205494889DD
:104AA000194600F09DF903498889214600F098F9DC
:104AB00010BD0000A60000202DE9FF4F9B46009B83
:104AC000029CDDF80490DA4627488088A0F513415F
:104AD000413922D12A2000F073F9181200F06AF946
:104AE000D8B200F067F9201200F064F9E0B200F0EB
:104AF00061F92B2000F064F94FEA292000F05AF9FF
:104B000009F0FF0000F056F94FEA2A2000F052F9B0
:104B10000AF0FF0000F04EF924E013488088A0F569
:104B20000941893909D14425442643EA042083B246
:104B30001C4645274FF0460804E0502551265227D1
:104B40004FF053081946284600F04AF921463046EE
:104B500000F046F94946384600F042F951464046D1
:104B600000F03EF9BDE8FF8FA60000202DE9F84FC8
:104B700080460E4617461C46B3462046E31704EB14
:104B80005373DB1021464FEAE47C04EB5C7C4FEA74
:104B9000EC0CB4EBCC0C02D04FF0010C01E04FF068
:104BA000000C6344224604EBD27C4FEA6C0C03FBFE
:104BB0000CF3DBB20093A7F12000C7B2002556E04A
:104BC0000C2C07D107EB47002B4901EB800010F8B4
:104BD000059013E0102C05D1284800EB071010F8C1
:104BE00005900BE0182C07D107EBC700244901EB17
:104BF000800010F8059001E0BDE8F88F4FF0000A42
:104C00002FE019F0800F06D01E480288314640463A
:104C1000FBF7F4FF07E00A9828B91B4802883146E1
:104C20004046FBF7EBFF4FEA49604FEA1069701C02
:104C300086B216484088B04200DCDDE7A6EB0B00E8
:104C4000A0420AD15E4608F101001FFA80F80F4821
:104C50000088404500DCCFE706E00AF1010000F0E3
:104C6000FF0ABAF1080FCCDB00BF681CC5B2009880
:104C70008542A5DB00BFBFE7C86A00083C6F00089B
:104C80002C750008180000201A000020A600002043
:104C90002DE9F84704460D4690469946DDE9096737
:104CA00004F0FF0A08EB04001FFA80F809EB050086
:104CB0001FFA80F916E0444502DB5446A81985B274
:104CC0004D4500DB14E0002000903A783346294639
:104CD0002046FFF74BFF304606EBD07104EB610135
:104CE0008CB27F1C38787E2802DC38782028E2DA03
:104CF00000BFBDE8F8872DE9FF4F82B00646924617
:104D00001F46DDE90F480020019000254DE0781B8B
:104D1000401EC1B20A20FFF739FCBAFBF0F00A21AD
:104D2000B0FBF1F201FB1209019850BB781EA842BA
:104D300027DDB9F1000F22D118F0800F0FD008F055
:104D40000100A34604EBDB71491001FB05610090F3
:104D500088B2234630220399FFF708FF0EE008F0DF
:104D60000100A34604EBDB71491001FB05610090D3
:104D700088B2234620220399FFF7F8FE13E00120B2
:104D8000019008F00100A34604EBDB71491001FB20
:104D90000561009088B209F13001CAB22346039937
:104DA000FFF7E4FE00BF681CC5B2BD42AFDB06B032
:104DB000BDE8F08F01490880704700000008006CD2
:104DC0000149088070470000FE07006C0248008916
:104DD0000249088070470000A6000020FE07006C12
:104DE000024A1080921C118070470000FE07006C80
:104DF00008B50121402000F083F86020ADF80000E4
:104E000010208DF8030003208DF802006946064843
:104E1000FBF769FC20210448FBF7F0FC4021024825
:104E2000FBF7ECFC08BD00000018014000BFFEE7E6
:104E30007047000070B5002100230F22C4780CB326
:104E4000164C246804F4E064C4F5E064210AC1F15E
:104E50000403CA40447804FA03F1847814402143DF
:104E600009010F4C0678A155047804F01F050124B0
:104E7000AC4005786D114FF0E02606EB8505C5F8CE
:104E8000004109E0047804F01F050124AC40054D01
:104E90000678761145F8264070BD00000CED00E064
:104EA00000E400E080E100E002490143024A1160B1
:104EB000704700000000FA050CED00E070470000AC
:104EC00029B1064A52690243044B5A6104E0034A7D
:104ED00052698243014B5A61704700000010024042
:104EE00029B1064AD2690243044BDA6104E0034A5D
:104EF000D2698243014BDA61704700000010024022
:104F000029B1064A92690243044B9A6104E0034ABC
:104F100092698243014B9A61704700000010024081
:104F200030B500210022002400232D4D6D6805F0CE
:104F30000C0121B1042905D0082923D105E0294D10
:104F4000056022E0274D05601FE0254D6D6805F4E2
:104F50007012234D6D6805F48034022505EB9242F2
:104F60001CB9214D554305600BE01D4D6D6815F4CE
:104F7000003F03D01C4D5543056002E0194D5543D9
:104F8000056002E0174D056000BF00BF144D6D685D
:104F900005F0F0010909154D6B5C0568DD404560C1
:104FA0000F4D6D6805F4E061090A104D6B5C4568B2
:104FB000DD4085600A4D6D6805F46051C90A0B4DEE
:104FC0006B5C4568DD40C560054D6D6805F440418A
:104FD000890B074D6B5CC568B5FBF3F5056130BD0A
:104FE0000010024000127A0000093D002500002058
:104FF00035000020704710B500F002F810BD000029
:105000000CB50020019000903248006840F48030D8
:105010003049086000BF2F48006800F4003000905D
:105020000198401C0190009818B90198B0F5A06F44
:10503000F1D12848006810F4003F02D00120009010
:1050400001E0002000900098012842D12248006829
:1050500040F01000204908600846006820F0030076
:1050600008600846006840F002000860194840687F
:10507000184948600846406848600846406840F45F
:10508000806048600846406820F47C10486008460C
:10509000406840F4E81048600846006840F08070BE
:1050A000086000BF0B48006810F0007FFAD0094884
:1050B000406820F00300074948600846406840F017
:1050C0000200486000BF0348406800F00C00082858
:1050D000F9D10CBD001002400020024070470000D2
:1050E00010B51348006840F00100114908600846F7
:1050F0004068104908400E494860084600680E495B
:1051000008400B4908600846006820F480200860C9
:105110000846406820F4FE0048604FF41F00886095
:10512000FFF769FF4FF000600449086010BD000000
:10513000001002400000FFF8FFFFF6FE08ED00E05F
:105140001CB50121684800F0EEF801287ED100214D
:10515000664800F0ECF90021654800F0E8F901200C
:105160006449087064480078401C634908706348CB
:105170000078401C61490870084600783C2806D138
:10518000002008705E480078401C5D4908705C484B
:1051900000783C2807D15B480078401C59490870CA
:1051A00000205749087057480078182802D100207D
:1051B000544908705148007809281BDC052000F08C
:1051C000E7FB0020102101230246CDE900100A214F
:1051D000A220FFF790FD052000F0DAFB002010214F
:1051E0000123CDE90010454802780A21AA20FFF7E3
:1051F00082FD0DE0052000F0CBFB002010210223F2
:10520000CDE900103D4802780A21A220FFF773FD86
:105210003B48007809281DDC052000F0B9FB002080
:10522000102101230246CDE900100A218A20FFF750
:1052300062FD052000F0ACFB002010210123CDE928
:1052400000102F4802780A21922000E04AE0FFF780
:1052500052FD0DE0052000F09BFB002010210223F1
:10526000CDE90010264802780A218A20FFF743FD85
:105270002448007809281BDC052000F089FB002069
:10528000102101230246CDE900100A217220FFF708
:1052900032FD052000F07CFB002010210123CDE928
:1052A0000010184802780A217A20FFF724FD0DE04B
:1052B000052000F06DFB002010210223CDE9001035
:1052C000104802780A217220FFF715FD01210648D7
:1052D00000F01AF80121054800F029F901210448DD
:1052E00000F025F91CBD000000040040003801401A
:1052F0000044004020000020210000202400002065
:105300002300002022000020CA430282704721B1FE
:10531000028842F00102028004E002884FF6FE7328
:105320001A400280704730B5024600200023002456
:10533000158A05EA0103958905EA010413B10CB148
:10534000012000E0002030BD1AB183890B43838126
:1053500002E083898B43838170470000002202882A
:105360001D4B98420ED01D4B98420BD0B0F1804F90
:1053700008D01B4B984205D01A4B984202D01A4BCA
:10538000984204D14FF68F731A404B881A43174B3B
:10539000984207D0164B984204D04FF6FF431A406C
:1053A000CB881A4302808B8883850B8803850A4B40
:1053B00098420BD0094B984208D00E4B984205D02A
:1053C0000D4B984202D00D4B984201D10B7A0386C7
:1053D0000123838270470000002C0140003401400B
:1053E0000004004000080040000C00400010004095
:1053F00000140040004001400044014000480140CA
:1054000010B540F22551124800F0AAF801281ED12B
:105410000F4800F061F9C4B2BB2C03D00D480078EE
:10542000002814DD0B4801780078401C094A1070F0
:105430000948445410460078062808D10648807868
:10544000012804D10549088000201146087010BDCC
:105450000038014006000020100000200800002055
:1054600010B540F22551114800F07AF801281BD1FF
:105470000E4800F031F9C4B2FF2C03D00C4800787C
:10548000002811DD0A4801780078401C084A107095
:105490000848445410460078092805D101200649DF
:1054A000088000201146087010BD00000044004034
:1054B00000000020500000200200002010B5002451
:1054C00040F22551114800F04BF801281DD10F483A
:1054D00000F002F9C4B27B2C03D00D4800780028FC
:1054E00013DD0B4801780078401C094A1070094808
:1054F00044547D2C03D0104600784B2805D1012060
:105500000549088000200249087010BD004800408D
:10551000010000205A0000200400002001F4007265
:10552000B2F5007F00D100BFCA430280704721B1AD
:10553000828942F40052828104E082894DF6FF7331
:105540001A408281704702460020B1F5007F00D1E9
:1055500000BF13880B4201D0012000E000207047FB
:1055600070B502460024002300250020A1F5106636
:105570006A3E00D100BFC1F3421501F01F030126AE
:1055800006FA03F3012D02D19689334006E0022D7D
:1055900002D1168A334001E0968A33400C1201266C
:1055A00006FA04F41688344013B10CB1012000E06F
:1055B000002070BDF0B50346002400260025002021
:1055C000A1F510676A3F00D100BF1846C1F342142D
:1055D00001F01F06012707FA06F5012C01D10C3056
:1055E00004E0022C01D1103000E014301AB1076839
:1055F0002F43076002E00768AF430760F0BD00007B
:105600002DE9F04786B005460E460024A24600BFAD
:10561000A1460027B08900B100BF2F462C8A4CF666
:10562000FF700440F08804432C82AC894EF6F310DE
:105630000440B08831890843718908430443AC8130
:10564000AC8A4FF6FF400440B0890443AC8201A805
:10565000FFF766FC1F48874202D1DDF810A001E089
:10566000DDF80CA0A88910F4004F08D00AEBCA009E
:1056700000EB0A1031684900B0FBF1F807E00AEBD3
:10568000CA0000EB0A1031688900B0FBF1F8642011
:10569000B8FBF0F004012009642101FB1089A889FE
:1056A00010F4004F08D0322000EBC900B0FBF1F03D
:1056B00000F00700044308E0322000EB09106421E9
:1056C000B0FBF1F000F00F0004432C8106B0BDE800
:1056D000F08700000038014001468888C0F30800C8
:1056E000704730B504460D46C5F30800A08000BFE2
:1056F00080212046FFF727FF0028F9D030BD30B5C4
:1057000005460C4604E021782846FFF7EAFF641CB2
:1057100020780028F7D130BD00BFFEE702E008C8BE
:10572000121F08C1002AFAD170477047002001E01B
:1057300001C1121F002AFBD1704700007CB500BFD9
:1057400032480579C67846EA05244FF47A7094FB0E
:10575000F0F0642148434FF47A7194FBF1F201FBBD
:105760001241642291FBF2F101EB810100EB410057
:10577000114694FBF1F201FB12410A2291FBF2F176
:105780000844234908700A2094FBF0F100FB114003
:10579000204908704FF47A7094FBF0F030301E49C5
:1057A00008704FF47A7094FBF0F100FB1140642113
:1057B00090FBF1F0303018494870642094FBF0F110
:1057C00000FB11400A2190FBF1F030301249887043
:1057D0002E20C8700A2094FBF0F100FB11403030FD
:1057E0000D49087100204871032000F0D1F80A48E3
:1057F00010210B462822CDE9001092219720FFF7B7
:1058000047FA032000F0C4F87CBD0000100000201F
:105810004A0000204B0000203F0000207CB500BF64
:1058200000BF00BF2348C578067905EB85008000DE
:105830006421484306EB860100EB81041E48057095
:105840001E4806704FF47A70B4FBF0F030301C49FB
:1058500008704FF47A70B4FBF0F100FB1140642142
:10586000B0FBF1F03030164948702E20887064206B
:10587000B4FBF0F100FB11400A21B0FBF1F0303035
:105880000F49C8700A20B4FBF0F100FB1140303022
:105890000B49087100204871052000F079F808488C
:1058A00010210B462822CDE900107E219720FFF71A
:1058B000EFF97CBD50000020480000204900002086
:1058C0003900002000B587B0002201212D48FFF7E4
:1058D0003BFD05A906A8FAF724FE01221146294836
:1058E000FFF732FD9DF818000A2190FBF1F03030EF
:1058F000C0B28DF810009DF8180090FBF1F201FB8A
:1059000012003030C0B28DF8110000208DF8120066
:10591000052000F03DF804A810210B460A46CDE909
:1059200000107E213320FFF7B3F99DF814000A21FF
:1059300090FBF1F03030C0B28DF80C009DF81400EF
:1059400090FBF1F201FB12003030C0B28DF80D0077
:1059500000208DF80E00052000F01AF803A8102191
:105960000B460A46CDE9001092213320FFF790F94B
:105970009DF81800044908709DF814000349087048
:1059800007B000BD00040040460000204700002092
:10599000014642F228324A434FF0E0235A61012285
:1059A0001A6100229A6100BF4FF0E022106910F0E6
:1059B000010F02D010F4803FF6D000224FF0E02318
:1059C0001A619A617047014601EBC1024FF0E02372
:1059D0005A6101221A6100229A6100BF4FF0E02251
:1059E000106910F0010F02D010F4803FF6D00022B1
:1059F0004FF0E0231A619A617047000010B5002152
:105A00000348FFF794FD00210248FFF790FD10BD09
:105A1000003801400044004010B501210348FFF761
:105A200086FD01210248FFF782FD10BD00380140CC
:105A3000004400402DE9FC4106460F4614464FF055
:105A40000808254604EB08002978CDE90010A8884D
:105A50003844401E83B268883044401E82B23946C2
:105A6000304600F011F8BDE8FC8110B502462AB1BD
:105A700011F8014B20020B78184304E011F8010BD8
:105A80000B7840EA032010BD2DE9F84F8046894687
:105A900015461E46DDE90A4A4FF0000B14F0030FCD
:105AA00041D1A01106D0012812D002281ED003280F
:105AB00038D129E00020FEF7B5FD33462A46494695
:105AC0004046FEF7F9FF49464046FEF721FF29E030
:105AD0000120FEF7A7FD33462A4649464046FEF719
:105AE000EBFF31464046FEF713FF1BE00220FEF7B6
:105AF00099FD33462A4649464046FEF7DDFF4946B2
:105B00002846FEF705FF0DE00320FEF78BFD334628
:105B10002A4649464046FEF7CFFF31462846FEF763
:105B2000F7FE00BF41E0A01106D0012812D00228E4
:105B30001ED0032838D129E00420FEF773FD334638
:105B40002A4649464046FEF7B7FF49464046FEF71B
:105B5000DFFE29E00620FEF765FD33462A4649466A
:105B60004046FEF7A9FF31464046FEF7D1FE1BE056
:105B70000520FEF757FD33462A4649464046FEF7C4
:105B80009BFF49462846FEF7C3FE0DE00720FEF7BF
:105B900049FD33462A4649464046FEF78DFF3146C9
:105BA0002846FEF7B5FE00BF00BFFFF70FF9A5EBD3
:105BB0000800401CA6EB0901491C00FB01FB002763
:105BC0000AE004F010005146FFF74FFF0090FFF786
:105BD000F1F80AF1020A7F1C5F45F2D340F23F134D
:105BE000EF2200210846FEF767FFBDE8F88F0000AE
:105BF0001CB54FF6FF70FAF781FE01201021042337
:105C000040F2E272CDE900100A210846FFF773F86E
:105C10004FF6FF7000210223B7A2CDE900100A2140
:105C20002A20FAF7EDFD0120102103460622CDE9D6
:105C300000100A213A20FFF75EF84FF6FF700021AE
:105C40000223AEA2CDE900100A214220FAF7D8FDC6
:105C50000120102102230722CDE900100A21522041
:105C6000FFF749F84FF6FF7000210223A4A2CDE907
:105C700000100A216220FAF7C3FD0120102102233F
:105C80000D22CDE900100A217220FFF734F89DA003
:105C900010210B460822CDE9001009218220FEF7D1
:105CA000F7FF0120102102232F22CDE900100A2145
:105CB0008A20FFF720F893A010210B460822CDE997
:105CC000001009219A20FEF7E3FF01201021022392
:105CD0003222CDE900100A21A220FFF70CF84FF67E
:105CE000FF700021062388A2CDE900100A21B5200B
:105CF000FAF786FD4FF6FF7000210A2385A2CDE951
:105D000000101E211846FAF77BFD86A010210B46D5
:105D10002022CDE900101E215A20FEF7B9FF3223C0
:105D2000EF2219460020FAF7FFFE4A23EF22194618
:105D30000020FAF7F9FE6223EF2219460020FAF755
:105D4000F3FE7A23EF2219460020FAF7EDFE7A23BC
:105D5000392232211046FAF7E7FE7A2372223221E5
:105D60001046FAF7E1FE7A23B82232211046FAF7FC
:105D7000DBFE4FF6FF70002104236CA2CDE900107A
:105D800036210C20FAF73CFD4FF6FF70002104236A
:105D900068A2CDE9001036214620FAF731FD4FF612
:105DA000FF700021042365A2CDE900103621852073
:105DB000FAF726FD4FF6FF700021042361A2CDE91A
:105DC00000103621C420FAF71BFD60A010210B46FD
:105DD0000A46CDE900104E210C20FEF759FF4FF680
:105DE000FF70002102235AA2CDE900104E211C2091
:105DF000FAF706FD4FF6FF700021022355A2CDE908
:105E000000104E215D20FAF7FBFC4FF6FF700021D9
:105E1000022351A2CDE900104E217520FAF7F0FCC3
:105E20004FF6FF70002104234CA2CDE900104E2153
:105E30009520FAF7E5FC4FF6FF700021062349A2F2
:105E4000CDE900104E21BC20FAF7DAFC4FF6FF70C6
:105E50000021062346A2CDE900107E210320FAF797
:105E6000CFFC4FF6FF700021022343A2CDE90010C2
:105E70007E214320FAF7C4FC4FF6FF70002108236F
:105E80003EA2CDE900107E215720FAF7B9FC3EA0D2
:105E900010210B462822CDE900107E21C720FEF7F5
:105EA000F7FE4FF6FF700021062339A2CDE900105E
:105EB00092210320FAF7A4FC37A010210B461822E8
:105EC000CDE9001092214320FEF7E2FE4FF6FF706D
:105ED0000021062331A2CDE9001092216720FAF7B4
:105EE0008FFC30A010210B460A46CDE9001092210C
:105EF000BF20FEF7CDFE1CBDE5B9B400E69C8800CE
:105F0000E697A5003A000000E6989FE69C9FE59B77
:105F10009B000000E7B3BBE7BB9FE78AB6E6808142
:105F2000000000004F46462100000000E7BABFE82D
:105F3000B7AF0000E8B79DE7A6BB0000E697B6E95B
:105F400097B40000E78AB6E6808100005858000048
:105F5000E8B7AF00E7B1B300E7BAA600E58886E985
:105F6000929F0000E5BE85E58F91E8BDA600000088
:105F7000E6B094E6B8A90000E5BAA600E9A297E762
:105F8000B292E789A900000075672F6D3300000009
:105F9000E6B9BFE5BAA6000025726800E599AAE94E
:105FA0009FB300006442000092B0002011900026D0
:105FB0008246242108A8FAF7DEF84FF4A060FEF725
:105FC00073FFFAF737FFFEF713FF40F2DC50FFF7DD
:105FD000DFFCFFF70DFE4FF4E13000F073FC4FF4EF
:105FE000165000F0C3FC4FF4E13000F015FD4FF403
:105FF0007A70FFF7CDFC0120FE490870FAF73CFAF1
:1060000018B10120FB4908700CE0FBA018210B46D9
:106010005022CDE900100A216420FEF739FE00204D
:10602000F449087048F69F414FF4FA6000F012FC02
:106030004FF4FA70FFF7ACFCFFF7E0FCD7E30AF18E
:10604000010000F0FF0A4021ED48FAF7D5FB2021BE
:10605000EB48FAF7D1FBBAF1030F03D14FF0000A76
:10606000FFF730FCFFF7D8FC9620FFF791FC2021CA
:10607000E348FAF7C3FB9620FFF78AFCFFF7BEFC64
:10608000E048008820B10020DE490880FFF756FB79
:10609000DD4800780F287DD10020DB490870DB48FF
:1060A0000078C043D94908700520FFF771FC4FF60E
:1060B000FF70EF2340F23F12A72100900020FAF773
:1060C0005BFED248007868B10121D148FFF72BF977
:1060D000012807D00520FFF75BFCCE4AA7212D2021
:1060E000FFF7A8FCC948007868B90121C848FFF744
:1060F0001AF9012807D00520FFF74AFCC64AA72154
:106100002D20FFF797FC3220FFF742FCB9480078BA
:1061100001287DD161208DF820003D208DF82100DF
:10612000FF208DF8220026208DF8230062208DF8B4
:1061300024003D208DF8250031208DF826002620F2
:106140008DF8270063208DF828003D208DF8290068
:10615000B24800783030C0B28DF82A0026208DF881
:106160002B0064208DF82C003D208DF82D00AC48CC
:1061700000783030C0B28DF82E0026208DF82F0028
:1061800065208DF830003D208DF83100A54800785D
:10619000303000E057E0C0B28DF8320026208DF894
:1061A000330066208DF834003D208DF835009E4880
:1061B00000783030C0B28DF8360026208DF83700D8
:1061C00067208DF838003D208DF839009748007819
:1061D0003030C0B28DF83A0026208DF83B006820A0
:1061E0008DF83C003D208DF83D009148007830301E
:1061F000C0B28DF83E0026208DF83F0069208DF852
:1062000040003D208DF8410030208DF8420000E034
:1062100007E000208DF8430008A98648FFF76FFAD1
:106220000FE061208DF820003D208DF82100FE2038
:106230008DF8220000208DF8430008A97D48FFF763
:106240005EFAFFF7E9FB7C48008870B100207A49CC
:10625000088009217948FAF733FA11907748017AD2
:106260001198814201D1FFF7D9FA754800880028BA
:106270007ED000244FF0300B302007900020069095
:106280000590049000250390002780468146402118
:106290005B48FAF7B3FA00206949088000BF99E229
:1062A0006848005D61281ED16649E01C11F800B005
:1062B000ABF1300001280BD14FF6FF70002106230F
:1062C00061A2CDE900104E21BC20FAF799FA0AE04C
:1062D0004FF6FF70002106235EA2CDE900104E218B
:1062E000BC20FAF78DFA5748005D622825D1554940
:1062F000E01C085C079007983038012813D14FF64E
:10630000FF702E237A221E2100907220FAF734FDAE
:1063100053A010210B461822CDE900101E215A204F
:10632000FEF7B6FC09E04FA010210B462022CDE974
:1063300000101E215A20FEF7ABFC4248005D632886
:1063400037D14049201D085C2C281AD1E01C085C7C
:106350003038C0B206904FF6FF705E238D224E217A
:1063600000908520FAF708FD00201021012300E0AD
:106370003DE2CDE900104E218D20069AFEF7BBFCD0
:1063800017E03049201D095C2E4AE01C105C3038B3
:1063900000EB800001EB40003038C0B206900020D6
:1063A00010210223CDE900104E218520069AFEF728
:1063B000A2FC2448005D642873D12249201D085C9A
:1063C0002C2856D1E01C085C3038C0B205904FF63E
:1063D000FF705E2345224E2100903D20FAF7CCFC51
:1063E000002010210123CDE900104E214520059AFF
:1063F0003CE00000450000204572726F7200000012
:106400000018014008000020210000204C0000205E
:106410000004004088820008062901084600002088
:106420004700002048000020490000204A000020CA
:106430004B000020004800400200002050000020D7
:10644000040000205A000020E8BF90E8A18CE4B8C6
:10645000AD000000E5BE85E58F91E8BDA600000017
:106460004F4B21004F46462100000000FEF743FC41
:1064700017E0DF49201D095CDD4AE01C105C303864
:1064800000EB800001EB40003038C0B205900020E6
:1064900010210223CDE900104E213D20059AFEF780
:1064A0002AFCD348005D652835D1D149201D085C00
:1064B0002C2818D1E01C085C3038C0B204904FF68C
:1064C000FF705E235D224E2100905520FAF754FCA8
:1064D000002010210123CDE900104E214D20049A07
:1064E000FEF709FC17E0C249201D095CC04AE01C08
:1064F000105C303800EB800001EB40003038C0B257
:106500000490002010210223CDE900104E214D20DF
:10651000049AFEF7F0FBB648005D66285FD1B449E7
:10652000E01C085C3038C5B2012D0AD14FF6FF706F
:1065300000210623AFA2CDE900100A21B520FAF709
:106540005FF9022D0AD14FF6FF7000210623ACA29D
:10655000CDE900100A21B520FAF752F9032D0AD12E
:106560004FF6FF7000210623A8A2CDE900100A21F2
:10657000B520FAF745F9042D0AD14FF6FF70002136
:106580000623A5A2CDE900100A21B520FAF738F9B3
:10659000052D0AD14FF6FF7000210623A1A2CDE9F7
:1065A00000100A21B520FAF72BF9062D0AD14FF673
:1065B000FF70002106239EA2CDE900100A21B5201C
:1065C000FAF71EF9072D0AD14FF6FF7000210623B6
:1065D0009AA2CDE900100A21B520FAF711F98448F2
:1065E000005D672835D18249201D085C2C2818D110
:1065F000E01C085C3038C0B203904FF6FF701A23DD
:106600005A220A2100905220FAF7B6FB00201021EE
:106610000123CDE900100A215A20039AFEF76BFBF3
:1066200017E07349201D095C714AE01C105C30388A
:1066300000EB800001EB40003038C0B20390002036
:1066400010210223CDE900100A215220039AFEF7FF
:1066500052FB6748005D682838D16549201D085CF9
:106660002C281AD1E01C085C3038C7B27648077075
:106670000020102101230246CDE900100A217220DA
:10668000FEF739FB0020102101233A46CDE9001026
:106690000A217A20FEF72FFB18E05549201D095CDE
:1066A000534AE01C105C303800EB800001EB4000E6
:1066B0003038C7B2644807700020102102233A46E0
:1066C000CDE900100A217220FEF715FB4848005D55
:1066D00069283CD14649201D085C2C281CD1E01CAF
:1066E000085C303800F0FF08584880F8008000202F
:1066F000102101230246CDE900100A218A20FEF76D
:10670000FAFA0020102101234246CDE900100A21A7
:106710009220FEF7F0FA1AE03549201D095C344A50
:10672000E01C105C303800EB800001EB400030389A
:1067300000F0FF08454880F8008000201021022367
:106740004246CDE900100A218A20FEF7D4FA2848F3
:10675000005D6A283CD12649201D085C7D281CD19B
:10676000E01C085C303800F0FF09394880F80090E0
:106770000020102101230246CDE900100A21A220A9
:10678000FEF7B9FA0020102101234A46CDE9001096
:106790000A21AA20FEF7AFFA1AE01549201D095C6C
:1067A000134AE01C105C303800EB800001EB400025
:1067B000303800F0FF09264880F8009000201021B2
:1067C00002234A46CDE900100A21A220FEF793FADF
:1067D000601CC4B24B2CFFF663AD002604E0002021
:1067E00003498855701CC6B24B2EF8DD00BF26E465
:1067F0005A000020E6989FE69C9FE4B880000000C5
:10680000E6989FE69C9FE4BA8C000000E6989FE61D
:106810009C9FE4B889000000E6989FE69C9FE59B5A
:106820009B000000E6989FE69C9FE4BA940000005D
:10683000E6989FE69C9FE585AD000000E6989FE600
:106840009C9FE697A5000000220000202300002066
:10685000240000207FB505460C4601210220FEF7EA
:106860003FFB01211648FEF74FFDA8B2ADF8080026
:10687000A0B2ADF804000020ADF80A00ADF80600A3
:1068800001A90F48FEF76AFD01210D48FEF73FFD03
:10689000012211460A48FEF757FD4FF4C060FEF78B
:1068A00003FB1D208DF8000000208DF80100012061
:1068B0008DF802008DF803006846FEF7BBFA7FBD35
:1068C0000004004010B586B00446012144F20500E2
:1068D000FEF716FB4FF40070ADF8140003208DF89E
:1068E000160018208DF8170005A91E48F9F7FBFEC1
:1068F0004FF48060ADF8140004208DF8170005A94E
:106900001848F9F7F0FE25208DF8000003208DF8D7
:10691000010001208DF802008DF803006846FEF7A3
:1069200089FA01940020ADF80800ADF80A00ADF82E
:106930000C00ADF810000C20ADF80E0001A90A48BB
:10694000FEF75EFE40210848FEF7E8FD012240F216
:1069500025510548FEF72EFE01210348FEF7E7FD0D
:1069600006B010BD000801400038014010B586B0E7
:10697000044601210420FEF7C3FA01214804FEF772
:10698000AFFA0420ADF8140003208DF8160018208B
:106990008DF8170005A91E48F9F7A5FE0820ADF8E7
:1069A000140004208DF8170005A91948F9F79BFE7B
:1069B00026208DF8000002208DF8010003208DF8BC
:1069C000020001208DF803006846FEF733FA0194B7
:1069D0000020ADF80800ADF80A00ADF80C00ADF8E5
:1069E00010000C20ADF80E0001A90A48FEF708FEC1
:1069F00040210848FEF792FD012240F2255105484A
:106A0000FEF7D8FD01210348FEF791FD06B010BD49
:106A1000000801400044004010B586B00446012142
:106A20000820FEF76DFA01218804FEF759FA4FF4A9
:106A30008060ADF8140003208DF8160018208DF842
:106A4000170005A91E48F9F74EFE4FF40060ADF897
:106A5000140004208DF8170005A91948F9F743FE22
:106A600027208DF8000001208DF8010002208DF80C
:106A7000020001208DF803006846FEF7DBF901945F
:106A80000020ADF80800ADF80A00ADF80C00ADF834
:106A900010000C20ADF80E0001A90A48FEF7B0FD69
:106AA00040210848FEF73AFD012240F225510548F1
:106AB000FEF780FD01210348FEF739FD06B010BD49
:106AC000000C0140004800400000000000000000F1
:106AD00000000000000000003F4000000000000037
:106AE00000003000400030004000000009000BC0F2
:106AF0003D000BC03D00090018C024407FE022404B
:106B000031800000180024C01B000D80324001803D
:106B100003801C4027401C8007400040100060009C
:106B200000000000000000000000000000001F80C6
:106B3000204040200000402020401F800000000036
:106B4000090006001F800600090000000400040080
:106B50003F800400040000000010006000000000FE
:106B60000000000004000400040004000400000011
:106B7000000000400000000000000000002001C0F4
:106B800006003800400000001F80204020402040C8
:106B90001F800000000010403FC0004000000000C7
:106BA00018C021402240244018400000108020409E
:106BB000244024401B80000002000D0011003FC053
:106BC000014000003C8024402440244023800000F9
:106BD0001F80244024403440038000003000200007
:106BE00027C03800200000001B802440244024409F
:106BF0001B8000001C0022C0224022401F80000099
:106C0000000000000840000000000000000000003C
:106C10000460000000000000000004000A001100F1
:106C20002080404009000900090009000900000017
:106C300000004040208011000A00040018002000DD
:106C400023402400180000001F80204027402940D6
:106C50001F400000004007C039000F0001C0004085
:106C600020403FC0244024401B8000001F80204063
:106C7000204020403080000020403FC02040204085
:106C80001F80000020403FC024402E4030C0000044
:106C900020403FC024402E00300000000F00108034
:106CA000204022403380020020403FC00400040006
:106CB0003FC02040204020403FC0204020400000F6
:106CC0000060202020203FC02000200020403FC046
:106CD00024400B0030C0204020403FC020400040F6
:106CE000004000C03FC03C0003C03C003FC000006B
:106CF00020403FC00C4023003FC020001F802040A8
:106D0000204020401F80000020403FC0244024003D
:106D1000180000001F802140214020E01FA000003B
:106D200020403FC02440260019C0004018C0244025
:106D30002440224031800000300020403FC02040ED
:106D40003000000020003F80004000403F802000D5
:106D500020003E0001C0070038002000380007C0B6
:106D60003C0007C038000000204039C0060039C090
:106D7000204000002000384007C0384020000000BC
:106D8000304021C02640384020C0000000000000F4
:106D90007FE0402040200000000070000C000380D5
:106DA000004000000000402040207FE00000000084
:106DB0000000200040002000000000000010001033
:106DC0000010001000100010000000004000000043
:106DD00000000000000002800540054003C00040A4
:106DE00020003FC0044004400380000000000380F6
:106DF000044004400640000000000380044024409A
:106E00003FC00040000003800540054003400000F3
:106E1000000004401FC0244024402000000002E085
:106E2000055005500650042020403FC00440040097
:106E300003C000400000044027C0004000000000E4
:106E400000100010041027E00000000020403FC0A8
:106E50000140070004C00440204020403FC00040E3
:106E60000040000007C0040007C0040003C0000089
:106E7000044007C00440040003C000400000038039
:106E80000440044003800000041007F00450044054
:106E900003800000000003800440045007F000104D
:106EA000044007C002400400040000000000064047
:106EB0000540054004C00000000004001F8004409D
:106EC00000400000040007800040044007C000406C
:106ED0000400070004C0018006000400060001C091
:106EE000070001C006000000044006C0010006C003
:106EF000044000000410071004E0018006000400B4
:106F00000000044005C006400440000000000000EE
:106F100004007BE040200000000000000000FFF0C3
:106F200000000000000040207BE0040000000000A2
:106F300040008000400020002000400000000000D1
:106F40000000000000000000000000000000000041
:106F500000001FCC000C0000000000000000080032
:106F6000300060000800300060000000022003FCD8
:106F70001E20022003FC1E200220000000000E182C
:106F800011043FFF10840C78000000000F001084F3
:106F90000F3800C0077818840078000000780F844C
:106FA00010C411240E9800E4008400080800680052
:106FB0007000000000000000000000000000000061
:106FC000000007E018182004400200000000400202
:106FD0002004181807E000000000000002400240F2
:106FE00001800FF00180024002400000008000801C
:106FF00000800FF800800080008000000001000D7C
:10700000000E0000000000000000000000000080F2
:107010000080008000800080008000800000000C64
:10702000000C00000000000000000000000000064E
:10703000001800600180060018002000000007F022
:10704000080810041004080807F0000000000804F5
:1070500008041FFC000400040000000000000E0CE7
:1070600010141024104411840E0C000000000C18A1
:1070700010041104110412880C700000000000E0DC
:107080000320042408241FFC0024000000001F9893
:10709000108411041104108810700000000007F023
:1070A00008881104110418880070000000001C00FA
:1070B000100010FC13001C001000000000000E382F
:1070C00011441084108411440E38000000000700A1
:1070D000088C10441044088807F0000000000000ED
:1070E0000000030C030C0000000000000000000082
:1070F0000001010600000000000000000000008008
:1071000001400220041008081004000002200220A0
:1071100002200220022002200220000000001004B1
:1071200008080410022001400080000000000E004A
:107130001200100C106C10800F00000003E00C18FF
:1071400013E4142417C4082807D000000004003CEE
:1071500003C41C40074000E4001C000410041FFC92
:107160001104110411040E880070000003E00C18D3
:1071700010041004100410081C10000010041FFC60
:10718000100410041004080807F0000010041FFC8D
:107190001104110417C410040818000010041FFC87
:1071A0001104110017C010000800000003E00C18C3
:1071B0001004100410441C780040000010041FFC50
:1071C00010840080008010841FFC10040000100454
:1071D00010041FFC10041004000000000003000154
:1071E000100110011FFE10001000000010041FFC11
:1071F000110403801464181C1004000010041FFC08
:107200001004000400040004000C000010041FFC23
:107210001F0000FC1F001FFC1004000010041FFCD6
:107220000C04030000E010181FFC100007F0080811
:10723000100410041004080807F0000010041FFCDC
:1072400010841080108010800F00000007F00818D4
:1072500010241024101C080A07F2000010041FFC60
:107260001104110011C011300E0C000400000E1C9E
:1072700011041084108410441C3800001800100001
:1072800010041FFC100410001800000010001FF86C
:1072900010040004000410041FF8100010001E0069
:1072A00011E0001C007013801C0010001FC0103C77
:1072B00000E01F0000E0103C1FC000001004180C8C
:1072C000163401C001C01634180C100410001C0044
:1072D000130400FC13041C00100000000804101C20
:1072E0001064108413041C04101800000000000037
:1072F00000007FFE4002400240020000000030001B
:107300000C0003800060001C00030000000040022D
:10731000400240027FFE000000000000000000006C
:10732000200040004000400020000000000100015B
:107330000001000100010001000100010000400007
:107340004000200000000000000000000000009845
:10735000012401440144014400FC000410001FFC0E
:107360000088010401040088007000000000007023
:10737000008801040104010400880000000000707E
:1073800000880104010411081FFC0004000000F83B
:10739000014401440144014400C80000000001040C
:1073A00001040FFC1104110411001800000000D6A4
:1073B00001290129012901C90106000010041FFC4F
:1073C000008401000100010400FC0004000001042D
:1073D000190419FC00040004000000000000000370
:1073E00000010101190119FE0000000010041FFC3A
:1073F0000024004001B4010C01040000000010044E
:1074000010041FFC0004000400000000010401FC43
:107410000104010001FC0104010000FC010401FC65
:10742000008401000100010400FC0004000000F8D9
:10743000010401040104010400F80000010101FF3E
:107440000085010401040088007000000000007045
:10745000008801040104010501FF00010104010489
:1074600001FC00840104010001800000000000CC48
:1074700001240124012401240198000000000100DE
:10748000010007F80104010400000000010001F8F8
:10749000000400040004010801FC00040100018054
:1074A0000170000C001001600180010001F0010C6E
:1074B000003001C00030010C01F0010000000104A7
:1074C000018C00740170018C010400000101018134
:1074D0000171000E001801600180010000000184AC
:1074E000010C013401440184010C00000000000083
:1074F0000000000001003EFC4002400200000000CD
:1075000000000000FFFF000000000000000040023B
:1075100040023EFC0100000000000000000060008E
:10752000800080004000400020002000000000009B
:10753000000000000000000000000000000000004B
:10754000000000000000000000000000000000003B
:107550000000000000000000000000000000000F1C
:1075600080380FFE380F8038000000000000000057
:107570000000000000000000000001000006000004
:107580000C00003800003100000600000C0000383C
:107590000000300000000000000000006180006773
:1075A000F807F980006180006180006180006180DF
:1075B0000067F807F980006180000000000000000B
:1075C000000001C0E003E0F00630080418081FFFC7
:1075D000FE040E080787F00381E0000000000000B1
:1075E00001F000060C00040408060C7001F9C0004C
:1075F0000E00003BE000EC18070808040C1800031C
:10760000E00000000001E00007F003F818041C0887
:1076100004170807E1D003C0E00023B0003C0800D5
:1076200020080000100000000000000100003100F0
:10763000003200001C0000000000000000000000FC
:10764000000000000000000000000000000000003A
:107650000000000000000000000000007F0001FFAB
:10766000C00780F00C001810000420000200000089
:107670000000002000021000040C00180780F00138
:10768000FFC0007F000000000000000000000000BC
:1076900000000000000000004200006600006600DC
:1076A000003C0000180003FFC0001800003C000070
:1076B00066000066000042000000000008000008AC
:1076C0000000080000080000080001FFC0000800DA
:1076D000000800000800000800000800000000008A
:1076E000000100003100003200001C00000000001A
:1076F000000000000000000000000000000000008A
:107700000000000008000008000008000008000059
:107710000800000800000800000800000800000839
:1077200000000000000000000000000038000038E9
:107730000000380000000000000000000000000011
:107740000000000000000000000000000006000033
:107750001C000070000180000E0000380000C00016
:107760000700001C000030000000000000000000C6
:107770007F8001FFE0038070060018040008040009
:107780000806001803807001FFE0007F8000000001
:1077900000000000000001000801000801000803CB
:1077A000FFF807FFF80000080000080000080000CC
:1077B0000000000000000001C03802C0580400981A
:1077C000040118040218040418061C1803F8180110
:1077D000E0F800000000000000000001C0E003C06D
:1077E000F004000804080804080806180803F41840
:1077F00001E7F00001E000000000000000000000D0
:107800000300000D00001100006100008108030169
:107810000807FFF80FFFF80001080001080000004A
:107820000000000000E007FCD0060808061008066B
:107830001008061008061838060FF00607C00000EA
:1078400000000000000000003F8001FFE0038430E2
:107850000208180410080410080410080718100380
:107860000FF00007C000000000000000000003C08F
:10787000000700000600000600F80607F8061800DA
:1078800006E0000700000600000000000000000104
:10789000E1E003F7F0063410041808041808040C9B
:1078A00008040C0806161803F3F001C1E0000000FC
:1078B00000000000F80003FC30030638040208044E
:1078C00002080402080404100308F001FFC0007F4E
:1078D00000000000000000000000000000000000A8
:1078E00000000000703800703800703800000000A0
:1078F0000000000000000000000000000000000088
:107900000000000000000000301A00301C000000E1
:107910000000000000000000000000000000000067
:107920000000000800001400002200004100008058
:107930008001004002002004001008000800000040
:1079400000000000210000210000210000210000B3
:107950002100002100002100002100002100002161
:1079600000000000000000000000080008040010F3
:107970000200200100400080800041000022000041
:10798000140000080000000000000003C00004C054
:1079900000040000080038080F38080838081000F4
:1079A0000C300007E00003C00000000000000000F1
:1079B0003F8000FFE0038070020F1006708804C053
:1079C00088048308047F8802C09003012000FE40E1
:1079D0000000080000180001F8003E0801C200077E
:1079E000020007E20000FE00001FC80001F80000CE
:1079F0003800000804000807FFF807FFF80408082B
:107A000004080804080804080806180803F4180104
:107A1000E7F00001E0000000000000003F8001FFEF
:107A2000E003807002001804000804000804000845
:107A30000400100600200780C000000004000807B2
:107A4000FFF807FFF8040008040008040008040019
:107A50001802001003807001FFE0007F800000002A
:107A600004000807FFF807FFF804080804080804E2
:107A70000808040808043E0804000806001801006D
:107A80006000000004000807FFF807FFF80408087A
:107A9000040800040800040800043E000600000674
:107AA0000000018000000000000000003F8001FF96
:107AB000E0038070060018040008040208040208AD
:107AC0000203F00783F00002000002000400080730
:107AD000FFF807FFF8040808000800000800000885
:107AE0000000080004080807FFF807FFF804000872
:107AF000000000000000040008040008040008075B
:107B0000FFF807FFF804000804000804000800005C
:107B10000000000000000000000600000700000157
:107B200004000104000104000307FFFE07FFFC043A
:107B3000000004000004000004000807FFF807FF2D
:107B4000F8040C08001800003E0004C7800503C8B4
:107B50000600F804003804001800000804000807B4
:107B6000FFF807FFF8040008000008000008000004
:107B70000800000800000800001800006000000075
:107B800004000807FFF807800807FC00007FC0001A
:107B900003F80007C000780007800807FFF807FF18
:107BA000F804000804000807FFF807000803C000F5
:107BB00000E000003800001E000007000001C004C3
:107BC00000F007FFF8040000000000007F8001FFC4
:107BD000E00380700600180400080400080600187E
:107BE00003003001FFE0007F800000000400080770
:107BF000FFF807FFF8040408040400040400040468
:107C000000040400060C0003F80001F0000000006E
:107C1000000000007F8001FFE00380700600880400
:107C200000880400C806003C03003E01FFE6007F18
:107C30008400000004000807FFF807FFF8040808A4
:107C4000040800040C00040F00040BC00610F0032D
:107C5000F03801E00800000800000001E0F803F03F
:107C600030063010041808041808040C08040C0826
:107C70000206180207F00781E000000001800006FC
:107C8000000004000004000004000807FFF807FFDC
:107C9000F804000804000004000006000001800051
:107CA00004000007FFE007FFF004001800000800D0
:107CB000000800000800000800000804001007FF8A
:107CC000E004000004000006000007E00007FE00DA
:107CD000041FE00001F80000380001E0043E000746
:107CE000C00006000004000004000007E00007FFD9
:107CF000C0041FF80007C007F80007FF80043FF822
:107D00000007C004F80007000004000000000004A1
:107D1000000806001807C07805F1C8003E00001FE3
:107D2000800463E80780F8060018040008000000DB
:107D300004000006000007800007E008047C08003B
:107D40001FF80007F800180804E008070000060004
:107D5000000400000000000100080600380400F8DC
:107D60000403E8040F08047C0805F00807C00807AE
:107D70000018040060000000000000000000000087
:107D8000000000000000003FFFFE20000220000273
:107D9000200002200002200002000000000000007D
:107DA000000008000007000000C0000038000006C6
:107DB000000001C000003000000E000001000000C3
:107DC000000000000000200002200002200002202D
:107DD00000022000023FFFFE000000000000000043
:107DE000000000000000000000000000000800008B
:107DF00010000030000020000030000010000008DB
:107E00000000000000000000000001000001000070
:107E1000010000010000010000010000010000015C
:107E2000000001000001000001000001000000004E
:107E300000000000002000002000001000001000E2
:107E40000000000000000000000000000000000032
:107E50000000000000F00019F8001B1800220800C4
:107E60002608002408002410003FF8001FF8000036
:107E70000800001800000004000007FFF80FFFF0E2
:107E80000018180010080020080020080030180012
:107E90001FF0000FC00000000000000007C0001F1E
:107EA000F0001830002008002008002008003C08DE
:107EB000001C100000600000000000000000000036
:107EC00007C0001FF000381800200800200800201C
:107ED0000804101007FFF80FFFF00000100000006A
:107EE0000000000000000007C0001FF0001230007A
:107EF0002218002208002208003208001E10000E7E
:107F000020000000000000002000002008002008E1
:107F100001FFF803FFF806200804200804200807E2
:107F2000200003000000000000000000000E000E12
:107F30006E001FF30031B10020B10020B10031917B
:107F4000001F13002E1E00200E0030000000000451
:107F5000000807FFF80FFFF80010080020000020BD
:107F600000002008003FF8001FF800000800000093
:107F70000000000000000020080020080020080683
:107F80003FF8063FF8000008000008000008000065
:107F900000000000000000000000000003000003DB
:107FA000002001002001002003063FFE063FFC00E8
:107FB000000000000000000000000004000807FFAF
:107FC000F80FFFF8000188000300002FC00038F808
:107FD0000020380020080000080000000000000019
:107FE000000004000804000804000807FFF80FFF61
:107FF000F800000800000800000800000000000071
:10800000002008003FF8003FF800100800200000A2
:108010003FF8003FF8001008002000003FF8003F44
:10802000F8000008000000002008003FF8003FF8BA
:10803000001008001000002000002008003FF80099
:108040001FF80000080000000000000007C0000F3B
:10805000F000183000300800200800200800300828
:10806000001830000FF00007C00000000000000002
:108070002001003FFF003FFF0010110020090020F9
:1080800008002008003038001FF0000FC00000007A
:108090000000000007C0001FF00038180020080092
:1080A0002008002009001011001FFF003FFF000002
:1080B00001000000002008002008002008003FF810
:1080C000003FF80008080010080020080020000009
:1080D0003000003000000000000000000000000C34
:1080E00078001E18003308002308002108002188AA
:1080F0000021980030F0003860000000000000000F
:10810000200000200000200000FFF003FFF8002006
:1081100008002008002008000030000000000000D7
:10812000000000002000003FF0007FF80000180071
:108130000008000008002010003FF8007FF0000059
:1081400010000000000000002000003000003C0093
:10815000003F800023F000007800007000238000C2
:108160003C00003000002000002000003C00003FE8
:10817000E00023F80000E0002700003E00003FE0A0
:108180000021F80001E0003E000020000000000097
:108190002008002008003838003E680027800003CF
:1081A000C8002CF800383800201800200800000013
:1081B000000000002000003003003C01003F83006D
:1081C00023EC000070002380003C00002000002011
:1081D0000000000000000000000000380800203807
:1081E0000020F80023E8002F88003E08003808002F
:1081F00020180000700000000000000000000000D7
:10820000000000000000000008000014001FF7FC40
:108210003000062000020000000000000000000006
:108220000000000000000000000000000000FFFF50
:10823000FF0000000000000000000000000000003F
:108240000000000000002000023000061FF7FC00C4
:108250001400000800000000000000000000000002
:108260000000000000000018000060000040000056
:10827000400000200000100000080000040000047E
:1082800000000C0000100000001095008F00011B82
:10829000FFFFFFFFFFFFFFFFFFFFFFFFFFFFFFFFEE
:1082A000FFFFFFFFFFFFFFFFFFFFFFFFFFFFFFFFDE
:1082B000FFFFFFFFFFFFFFFFFFFFFFFFFFFFFFFFCE
:1082C000FFFFFFFFFFFFFFFFFFFFFFFFFFFFFFFFBE
:1082D000FFFFFFFFFFFFFFFFFFFFFFFFFFFFFFFFAE
:1082E000FFFFFFFFFFFFFFFFFFFFFFFFFFFFFFFF9E
:1082F000FFFFFFFFFFFFFFFFFFFFFFFFFFFFFFFF8E
:10830000FFFFFFFFFFFFFFFFFFFFFFFFFFFFFFFF7D
:10831000FFFFFFFFFFFFFFFFFFFFFFFFFFFFFFFF6D
:10832000FFFFFFFFFFFFFFFFFFFFFFFFFFFFFFFF5D
:10833000FFFFFFFFFFFFFFFFFFFFFFFFFFFFFFFF4D
:10834000FFFFFFFFFFFFFFFFFFFFFFFFFFFFFFFF3D
:10835000FFFFFFFFFFFFFFFFFFFFFFFFFFFFFFFF2D
:10836000FFFFFFFFFFFFFFFFFFFFFFFFFFFFFFFF1D
:10837000FFFFFFFFFFFFFFFFFFFFFFFFFFFFFFFF0D
:10838000FFFFFFFFFFFFFFFFFFFFFFFFFFFFFFFFFD
:10839000FFFFFFFFFFFFFFFFFFFFFFFFFFFFFFFFED
:1083A000FFFFFFFFFFFFFFFFFFFFFFFFFFFFFFFFDD
:1083B000FFFFFFFFFFFFFFFFFFFFFFFFFFFFFFFFCD
:1083C000FFFFFFFFFFFFFFFFFFFFFFFFFFFFFFFFBD
:1083D000FFFFFFFFFFFFFFFFFFFFFFFFFFFFFFFFAD
:1083E000FFFFFFFFFFFFFFFFFFFFFFFFFFFFFFFF9D
:1083F000FFFFFFFFFFFFFFFFFFFFFFFFFFFFFFFF8D
:10840000FFFFFFFFFFFFFFFFFFFFFFFFFFFFFFFF7C
:10841000FFFFFFFFFFFFFFFFFFFFFFFFFFFFFFFF6C
:10842000FFFFFFFFFFFFFFFFFFFFFFFFFFFFFFFF5C
:10843000FFFFFFFFFFFFFFFFDFFF7EE71EC79DAED1
:108440003C8EBB755A5D1A4DF93CB934B934B93418
:10845000B934D93CFA443A557B65DB7D5C96BDB6B0
:108460003ED7BFEFFFFFFFFFFFFFFFFFFFFFFFFF55
:10847000FFFFFFFFFFFFFFFFFFFFFFFFFFFFFFFF0C
:10848000FFFFFFFFFFFFFFFFFFFFFFFFFFFFFFFFFC
:10849000FFFFFFFFFFFFFFFFFFFFFFFFFFFFFFFFEC
:1084A000FFFFFFFFFFFFFFFFFFFFFFFFFFFFFFFFDC
:1084B000FFFFFFFFFFFFFFFFFFFFFFFFFFFFFFFFCC
:1084C000FFFFFFFFFFFFFFFFFFFFFFFFFFFFFFFFBC
:1084D000FFFFFFFFFFFFFFFFFFFFFFFFFFFFFFFFAC
:1084E000FFFFFFFFFFFFFFFFFFFFFFFFFFFFFFFF9C
:1084F000FFFFFFFFFFFFFFFFFFFFFFFFFFFFFFFF8C
:10850000FFFFFFFFFFFFFFFFFFFFFFFFFFFFFFFF7B
:10851000FFFFFFFFFFFFFFFFFFFFFFFFFFFFFFFF6B
:10852000FFFFFFFFFFFFFFFFFFFFFFFFFFFFFFFF5B
:10853000FFFFFFFFFFFFFFFFFFFFFFFFFFFFFFFF4B
:10854000FFFFFFFFFFFFFFFFFFFFFFFFFFFFFFFF3B
:10855000FFFFFFFFFFFFFFFFDFF73ECF5C9E7B6566
:10856000B934180CB70377039703B703D803180C73
:10857000591C992CB934B934D93CB934B92C792463
:10858000581C180CD703970377039703D703381C9D
:10859000FA44DB75BDAE7EDFFFFFFFFFFFFFFFFF8D
:1085A000FFFFFFFFFFFFFFFFFFFFFFFFFFFFFFFFDB
:1085B000FFFFFFFFFFFFFFFFFFFFFFFFFFFFFFFFCB
:1085C000FFFFFFFFFFFFFFFFFFFFFFFFFFFFFFFFBB
:1085D000FFFFFFFFFFFFFFFFFFFFFFFFFFFFFFFFAB
:1085E000FFFFFFFFFFFFFFFFFFFFFFFFFFFFFFFF9B
:1085F000FFFFFFFFFFFFFFFFFFFFFFFFFFFFFFFF8B
:10860000FFFFFFFFFFFFFFFFFFFFFFFFFFFFFFFF7A
:10861000FFFFFFFFFFFFFFFFFFFFFFFFFFFFFFFF6A
:10862000FFFFFFFFFFFFFFFFFFFFFFFFFFFFFFFF5A
:10863000FFFFFFFFFFFFFFFFFFFFFFFFFFFFFFFF4A
:10864000FFFFFFFFFFFFFFFFFFFFFFFFFFFFFFFF3A
:10865000FFFFFFFFFFFFFFFFFFFFFFFFFFFFFFFF2A
:10866000FFFFFFFFFFFFFFFFFFFFFFFFFFFFFFFF1A
:10867000FFFFFFFFFFFFFFFFFFFFFFFF3ECF1C8E4F
:10868000FA44F80B77039703F80399345A5D1C8E6C
:10869000BDAE1ECF7EE7BFF7FFFFFFFFFFFFFFFF6F
:1086A000FFFFFFFFFFFFFFFFFFFFFFFFDFF7BFEF52
:1086B0005EDFFDC67CA6DB7D1A4D7924D7037703E8
:1086C0009703381C5A5D7CA67EE7FFFFFFFFFFFF84
:1086D000FFFFFFFFFFFFFFFFFFFFFFFFFFFFFFFFAA
:1086E000FFFFFFFFFFFFFFFFFFFFFFFFFFFFFFFF9A
:1086F000FFFFFFFFFFFFFFFFFFFFFFFFFFFFFFFF8A
:10870000FFFFFFFFFFFFFFFFFFFFFFFFFFFFFFFF79
:10871000FFFFFFFFFFFFFFFFFFFFFFFFFFFFFFFF69
:10872000FFFFFFFFFFFFFFFFFFFFFFFFFFFFFFFF59
:10873000FFFFFFFFFFFFFFFFFFFFFFFFFFFFFFFF49
:10874000FFFFFFFFFFFFFFFFFFFFFFFFFFFFFFFF39
:10875000FFFFFFFFFFFFFFFFFFFFFFFFFFFFFFFF29
:10876000FFFFFFFFFFFFFFFFFFFFFFFFFFFFFFFF19
:10877000FFFFFFFFFFFFFFFFFFFFFFFFFFFFFFFF09
:10878000FFFFFFFFFFFFFFFFFFFFFFFFFFFFFFFFF9
:10879000FFFFFFFFFFFFFFFFFFFFFFFFFFFFDFFF09
:1087A000DDBE7B6538147703970358247A657CA671
:1087B0003ED7DFF7FFFFFFFFFFFFFFFFFFFFFFFFDA
:1087C000FFFFFFFFFFFFFFFFFFFFFFFFFFFFFFFFB9
:1087D000FFFFFFFFFFFFFFFFFFFFFFFFFFFFFFFFA9
:1087E000FFFFFFFFFFFFBFEFFDC61C8E1A4D180CE9
:1087F000770397039934FB853ED7FFFFFFFFFFFF09
:10880000FFFFFFFFFFFFFFFFFFFFFFFFFFFFFFFF78
:10881000FFFFFFFFFFFFFFFFFFFFFFFFFFFFFFFF68
:10882000FFFFFFFFFFFFFFFFFFFFFFFFFFFFFFFF58
:10883000FFFFFFFFFFFFFFFFFFFFFFFFFFFFFFFF48
:10884000FFFFFFFFFFFFFFFFFFFFFFFFFFFFFFFF38
:10885000FFFFFFFFFFFFFFFFFFFFFFFFFFFFFFFF28
:10886000FFFFFFFFFFFFFFFFFFFFFFFFFFFFFFFF18
:10887000FFFFFFFFFFFFFFFFFFFFFFFFFFFFFFFF08
:10888000FFFFFFFFFFFFFFFFFFFFFFFFFFFFFFFFF8
:10889000FFFFFFFFFFFFFFFFFFFFFFFFFFFFFFFFE8
:1088A000FFFFFFFFFFFFFFFFFFFFFFFFFFFFFFFFD8
:1088B000FFFFFFFFFFFFFFFFFFFFFFFFFFFFFFFFC8
:1088C000FFFFFFFF1ECF9B6D18145703D8031A4DEF
:1088D0005C9E5EDFFFFFFFFFFFFFFFFFFFFFFFFF6D
:1088E000FFFFFFFFFFFFFFFFFFFFFFFFFFFFFFFF98
:1088F000FFFFFFFFFFFFFFFFFFFFFFFFFFFFFFFF88
:10890000FFFFFFFFFFFFFFFFFFFFFFFFFFFFFFFF77
:10891000FFFFFFFFFFFFFFFFDFF71DC7FB85992C60
:1089200097037703992C1C8E9EE7FFFFFFFFFFFF45
:10893000FFFFFFFFFFFFFFFFFFFFFFFFFFFFFFFF47
:10894000FFFFFFFFFFFFFFFFFFFFFFFFFFFFFFFF37
:10895000FFFFFFFFFFFFFFFFFFFFFFFFFFFFFFFF27
:10896000FFFFFFFFFFFFFFFFFFFFFFFFFFFFFFFF17
:10897000FFFFFFFFFFFFFFFFFFFFFFFFFFFFFFFF07
:10898000FFFFFFFFFFFFFFFFFFFFFFFFFFFFFFFFF7
:10899000FFFFFFFFFFFFFFFFFFFFFFFFFFFFFFFFE7
:1089A000FFFFFFFFFFFFFFFFFFFFFFFFFFFFFFFFD7
:1089B000FFFFFFFFFFFFFFFFFFFFFFFFFFFFFFFFC7
:1089C000FFFFFFFFFFFFFFFFFFFFFFFFFFFFFFFFB7
:1089D000FFFFFFFFFFFFFFFFFFFFFFFFFFFFFFFFA7
:1089E000FFFFFFFFFFFFFFFFDFF75C9E992C770380
:1089F000B7031A4D9DAEBFEFFFFFFFFFFFFFFFFF65
:108A0000FFFFFFFFFFFFFFFFFFFFFFFFFFFFFFFF76
:108A1000FFFFFFFFFFFFFFFFFFFFFFFFFFFFFFFF66
:108A2000FFFFFFFFFFFFFFFFFFFFFFFFFFFFFFFF56
:108A3000FFFFFFFFFFFFFFFFFFFFFFFFFFFFFFFF46
:108A4000FFFFFFFFFFFFFFFFFFFF5EDF1C8E992C84
:108A50007703B7033A55FDBEFFFFFFFFFFFFFFFFA0
:108A6000FFFFFFFFFFFFFFFFFFFFFFFFFFFFFFFF16
:108A7000FFFFFFFFFFFFFFFFFFFFFFFFFFFFFFFF06
:108A8000FFFFFFFFFFFFFFFFFFFFFFFFFFFFFFFFF6
:108A9000FFFFFFFFFFFFFFFFFFFFFFFFFFFFFFFFE6
:108AA000FFFFFFFFFFFFFFFFFFFFFFFFFFFFFFFFD6
:108AB000FFFFFFFFFFFFFFFFFFFFFFFFFFFFFFFFC6
:108AC000FFFFFFFFFFFFFFFFFFFFFFFFFFFFFFFFB6
:108AD000FFFFFFFFFFFFFFFFFFFFFFFFFFFFFFFFA6
:108AE000FFFFFFFFFFFFFFFFFFFFFFFFFFFFFFFF96
:108AF000FFFFFFFFFFFFFFFFFFFFFFFFFFFFFFFF86
:108B0000FFFFFFFFFFFFFFFFFFFFFFFFFFFF9EE7EE
:108B1000DB7DF80B5703792C3C969EE7FFFFFFFFA8
:108B2000FFFFFFFFFFFFFFFFFFFFFFFFFFFFFFFF55
:108B30007DEFBAD6FFFFFFFFFFFFFFFFFFFFFFFF45
:108B4000FFFFFFFFFFFFFFFFFFFFFFFFFFFFFFFF35
:108B5000FFFFFFFFFFFFFFFFFFFFFFFFFFFFFFFF25
:108B6000FFFFFFFFFFFFFFFFFFFFFFFFFFFFFFFF15
:108B7000FFFFFFFFFFFFFFFFFFFF3ECF9B6DF80BE7
:108B80005703792C7CA6FFFFFFFFFFFFFFFFFFFFCE
:108B9000FFFFFFFFFFFFFFFFFFFFFFFFFFFFFFFFE5
:108BA000FFFFFFFFFFFFFFFFFFFFFFFFFFFFFFFFD5
:108BB000FFFFFFFFFFFFFFFFFFFFFFFFFFFFFFFFC5
:108BC000FFFFFFFFFFFFFFFFFFFFFFFFFFFFFFFFB5
:108BD000FFFFFFFFFFFFFFFFFFFFFFFFFFFFFFFFA5
:108BE000FFFFFFFFFFFFFFFFFFFFFFFFFFFFFFFF95
:108BF000FFFFFFFFFFFFFFFFFFFFFFFFFFFFFFFF85
:108C0000FFFFFFFFFFFFFFFFFFFFFFFFFFFFFFFF74
:108C1000FFFFFFFFFFFFFFFFFFFFFFFFFFFFFFFF64
:108C2000FFFFFFFFFFFFFFFFFFFFFFFFFFFFFFFF54
:108C3000FFFFFFFF9EE79B6DB70377031A4DFDBE55
:108C4000FFFFFFFFFFFFFFFFFFFFFFFFFFFFFFFF34
:108C5000FFFFFFFFFFFFFFFF96B5A6392008518CED
:108C6000FFFFFFFFFFFFFFFFFFFFFFFFFFFFFFFF14
:108C7000FFFFFFFFFFFFFFFFFFFFFFFFFFFFFFFF04
:108C8000FFFFFFFFFFFFFFFFFFFFFFFFB6BD694ACA
:108C90001BE7FFFFFFFFFFFFFFFFFFFFFFFFFFFFE0
:108CA000FFFFFFFFFFFFFFFFBFF75C9E5824570346
:108CB000381C5C9EFFFFFFFFFFFFFFFFFFFFFFFF72
:108CC000FFFFFFFFFFFFFFFFFFFFFFFFFFFFFFFFB4
:108CD000FFFFFFFFFFFFFFFFFFFFFFFFFFFFFFFFA4
:108CE000FFFFFFFFFFFFFFFFFFFFFFFFFFFFFFFF94
:108CF000FFFFFFFFFFFFFFFFFFFFFFFFFFFFFFFF84
:108D0000FFFFFFFFFFFFFFFFFFFFFFFFFFFFFFFF73
:108D1000FFFFFFFFFFFFFFFFFFFFFFFFFFFFFFFF63
:108D2000FFFFFFFFFFFFFFFFFFFFFFFFFFFFFFFF53
:108D3000FFFFFFFFFFFFFFFFFFFFFFFFFFFFFFFF43
:108D4000FFFFFFFFFFFFFFFFFFFFFFFFFFFFFFFF33
:108D5000FFFFFFFFFFFFFFFFFFFFBFEFBB7DB7037D
:108D600097035A5D3ED7FFFFFFFFFFFFFFFFFFFFA7
:108D7000FFFFFFFFFFFFFFFFFFFFFFFFFFFFD39C92
:108D8000484A4008200800007194FFFFFFFFFFFFE2
:108D9000FFFFFFFFFFFFFFFFFFFFFFFFFFFFFFFFE3
:108DA000FFFFFFFFFFFFFFFFFFFFFFFFFFFFFFFFD3
:108DB000FFFFFFFFFFFFAA5A0000B29CFFFFFFFF6B
:108DC000FFFFFFFF9EF7FFFFFFFFFFFFFFFFFFFF1C
:108DD000FFFFFFFFFFFFFFFFBDAE9934570358248D
:108DE0009DA6FFFFFFFFFFFFFFFFFFFFFFFFFFFF4E
:108DF000FFFFFFFFFFFFFFFFFFFFFFFFFFFFFFFF83
:108E0000FFFFFFFFFFFFFFFFFFFFFFFFFFFFFFFF72
:108E1000FFFFFFFFFFFFFFFFFFFFFFFFFFFFFFFF62
:108E2000FFFFFFFFFFFFFFFFFFFFFFFFFFFFFFFF52
:108E3000FFFFFFFFFFFFFFFFFFFFFFFFFFFFFFFF42
:108E4000FFFFFFFFFFFFFFFFFFFFFFFFFFFFFFFF32
:108E5000FFFFFFFFFFFFFFFFFFFFFFFFFFFFFFFF22
:108E6000FFFFFFFFFFFFFFFFFFFFFFFFFFFFFFFF12
:108E7000FFFFFFFFFFFFFFFFFFFFFFFFFFFFFFFF02
:108E8000FFFF3C96F80B77033A5D5ED7FFFFFFFFCD
:108E9000FFFFFFFFFFFFFFFFFFFFFFFFFFFFFFFFE2
:108EA000FFFFFFFFFFFF34AD000041108110A63926
:108EB000D39CFFFFFFFFFFFFFFFFFFFFFFFFFFFF51
:108EC000FFFFFFFFFFFFFFFFFFFFFFFFFFFFFFFFB2
:108ED000FFFFFFFFFFFFFFFFFFFFFFFFFFFFFFFFA2
:108EE0007194000014A5FFFFFFFFFFFFDBDEE3200E
:108EF0000F84DEFFFFFFFFFFFFFFFFFFFFFFFFFF0E
:108F0000FFFFFFFFFFFFBDAE792C57039934FDC66D
:108F1000FFFFFFFFFFFFFFFFFFFFFFFFFFFFFFFF61
:108F2000FFFFFFFFFFFFFFFFFFFFFFFFFFFFFFFF51
:108F3000FFFFFFFFFFFFFFFFFFFFFFFFFFFFFFFF41
:108F4000FFFFFFFFFFFFFFFFFFFFFFFFFFFFFFFF31
:108F5000FFFFFFFFFFFFFFFFFFFFFFFFFFFFFFFF21
:108F6000FFFFFFFFFFFFFFFFFFFFFFFFFFFFFFFF11
:108F7000FFFFFFFFFFFFFFFFFFFFFFFFFFFFFFFF01
:108F8000FFFFFFFFFFFFFFFFFFFFFFFFFFFFFFFFF1
:108F9000FFFFFFFFFFFFFFFFFFFFFFFFFFFFFFFFE1
:108FA000FFFFFFFFFFFFFFFF1DC7792C3603D944EA
:108FB0001ECFFFFFFFFFFFFFFFFFFFFFFFFFFFFFD2
:108FC000FFFFFFFFFFFFFFFFFFFFFFFFFFFFFFFFB1
:108FD00075B581100008508CFFFFFFFFFFFFFFFFFA
:108FE000FFFFFFFFFFFFFFFFFFFFFFFFFFFFFFFF91
:108FF000FFFFFFFFFFFFFFFFFFFFFFFFFFFFFFFF81
:10900000FFFFFFFFFFFFFFFFFFFFB6BD0000F7C53B
:10901000FFFFFFFFFFFF7DEFC3200000BADEFFFF71
:10902000FFFFFFFFFFFFFFFFFFFFFFFFFFFFFFFF50
:10903000FFFFFFFF7C9E181457035A65BFEFFFFF29
:10904000FFFFFFFFFFFFFFFFFFFFFFFFFFFFFFFF30
:10905000FFFFFFFFFFFFFFFFFFFFFFFFFFFFFFFF20
:10906000FFFFFFFFFFFFFFFFFFFFFFFFFFFFFFFF10
:10907000FFFFFFFFFFFFFFFFFFFFFFFFFFFFFFFF00
:10908000FFFFFFFFFFFFFFFFFFFFFFFFFFFFFFFFF0
:10909000FFFFFFFFFFFFFFFFFFFFFFFFFFFFFFFFE0
:1090A000FFFFFFFFFFFFFFFFFFFFFFFFFFFFFFFFD0
:1090B000FFFFFFFFFFFFFFFFFFFFFFFFFFFFFFFFC0
:1090C000FFFFFFFFFFFFFFFFFFFFFFFFFFFFDFF7D8
:1090D0009B6D570318149DA6FFFFFFFFFFFFFFFFC7
:1090E000FFFFFFFFFFFFFFFFFFFFFFFFFFFFFFFF90
:1090F000FFFFFFFFFFFFFFFFFFFF1CE740108E7326
:10910000FFFFFFFFDFFF18C675B5DFFFFFFFFFFFA3
:10911000FFFFFFFFFFFFFFFFFFFFFFFFFFFFFFFF5F
:10912000FFFFFFFFFFFFFFFFFFFFFFFFFFFF79CE06
:10913000694AB6B53CE796B5FFFFFFFFFFFFFFFFAB
:1091400095B520002C6BFFFFFFFFFFFFFFFFFFFF28
:10915000FFFFFFFFFFFFFFFFFFFFFFFFFFFFFFFF1F
:10916000DFF7BB757703F80B9CA6FFFFFFFFFFFF40
:10917000FFFFFFFFFFFFFFFFFFFFFFFFFFFFFFFFFF
:10918000FFFFFFFFFFFFFFFFFFFFFFFFFFFFFFFFEF
:10919000FFFFFFFFFFFFFFFFFFFFFFFFFFFFFFFFDF
:1091A000FFFFFFFFFFFFFFFFFFFFFFFFFFFFFFFFCF
:1091B000FFFFFFFFFFFFFFFFFFFFFFFFFFFFFFFFBF
:1091C000FFFFFFFFFFFFFFFFFFFFFFFFFFFFFFFFAF
:1091D000FFFFFFFFFFFFFFFFFFFFFFFFFFFFFFFF9F
:1091E000FFFFFFFFFFFFFFFFFFFFFFFFFFFFFFFF8F
:1091F000FFFFFFFFFFFFFDBE382457039B6DDFF726
:10920000FFFFFFFFFFFFFFFFFFFFFFFFFFFFFFFF6E
:10921000FFFFFFFFFFFFFFFFFFFFFFFFFFFFFFFF5E
:10922000FFFFFFFFD29C8218DFFFFFFFFBDEC63986
:1092300040084008DADEFFFFFFFFFFFFFFFFFFFFF0
:10924000FFFFFFFFFFFFFFFFFFFFFFFFFFFFFFFF2E
:10925000FFFFFFFFFFFFFFFFEF830000A639FFFFC7
:10926000FFFFBEFFB2949EF7FFFF8631410879D61B
:10927000FFFFFFFFFFFFFFFFFFFFFFFFFFFFFFFFFE
:10928000FFFFFFFFFFFFFFFFFFFFFFFFFFFF3ECFDF
:10929000B93436031A55BFEFFFFFFFFFFFFFFFFF93
:1092A000FFFFFFFFFFFFFFFFFFFFFFFFFFFFFFFFCE
:1092B000FFFFFFFFFFFFFFFFFFFFFFFFFFFFFFFFBE
:1092C000FFFFFFFFFFFFFFFFFFFFFFFFFFFFFFFFAE
:1092D000FFFFFFFFFFFFFFFFFFFFFFFFFFFFFFFF9E
:1092E000FFFFFFFFFFFFFFFFFFFFFFFFFFFFFFFF8E
:1092F000FFFFFFFFFFFFFFFFFFFFFFFFFFFFFFFF7E
:10930000FFFFFFFFFFFFFFFFFFFFFFFFFFFFFFFF6D
:10931000FFFFFFFFFFFFFFFFFFFFFFFFFFFFDB7D03
:109320005703381CFDBEFFFFFFFFFFFFFFFFFFFFDE
:10933000FFFFFFFFFFFFFFFFFFFFFFFFFFFFFFFF3D
:10934000FFFFFFFFFFFFFFFFFFFFFFFFFFFFAA5A27
:10935000D29CFBDE484A65314110A218C218FBDEE0
:10936000FFFFFFFFFFFFFFFFFFFFFFFFFFFFFFFF0D
:10937000FFFFFFFFFFFFFFFFFFFFFFFFFFFFFFFFFD
:10938000FFFF58CE6110AE7BDFFFBEF738C600008E
:10939000C639EB620000484A9294E74179CEFFFF5C
:1093A000FFFFFFFFFFFFFFFFFFFFFFFFFFFFFFFFCD
:1093B000FFFFFFFFFFFFFFFFFFFFFFFF1B8E770396
:1093C000F813DDB6FFFFFFFFFFFFFFFFFFFFFFFF0B
:1093D000FFFFFFFFFFFFFFFFFFFFFFFFFFFFFFFF9D
:1093E000FFFFFFFFFFFFFFFFFFFFFFFFFFFFFFFF8D
:1093F000FFFFFFFFFFFFFFFFFFFFFFFFFFFFFFFF7D
:10940000FFFFFFFFFFFFFFFFFFFFFFFFFFFFFFFF6C
:10941000FFFFFFFFFFFFFFFFFFFFFFFFFFFFFFFF5C
:10942000FFFFFFFFFFFFFFFFFFFFFFFFFFFFFFFF4C
:10943000FFFFFFFFFFFFFFFFFFFFFFFFFFFFFFFF3C
:10944000FFFFFFFF9EE7D94436035A65DFF7FFFFB2
:10945000FFFFFFFFFFFFFFFFFFFFFFFFFFFFFFFF1C
:10946000FFFFFFFFFFFFFFFFFFFFFFFFFFFFFFFF0C
:10947000FFFFFFFFFFFF7DEFE741B29CAA5A00000C
:109480002008E320A21803213CEFFFFFFFFFFFFFAE
:10949000FFFFFFFFFFFFFFFFFFFFFFFFFFFFFFFFDC
:1094A000FFFFFFFFFFFFFFFFFFFFFFFFFFFF79CE83
:1094B000D39C95B5BEF7B2940000C2186110CB5A88
:1094C000AA5A411000002C6BFFFFFFFFFFFFFFFFB8
:1094D000FFFFFFFFFFFFFFFFFFFFFFFFFFFFFFFF9C
:1094E000FFFFFFFFFFFFFFFF3ECF592C5703DB7D40
:1094F000FFFFFFFFFFFFFFFFFFFFFFFFFFFFFFFF7C
:10950000FFFFFFFFFFFFFFFFFFFFFFFFFFFFFFFF6B
:10951000FFFFFFFFFFFFFFFFFFFFFFFFFFFFFFFF5B
:10952000FFFFFFFFFFFFFFFFFFFFFFFFFFFFFFFF4B
:10953000FFFFFFFFFFFFFFFFFFFFFFFFFFFFFFFF3B
:10954000FFFFFFFFFFFFFFFFFFFFFFFFFFFFFFFF2B
:10955000FFFFFFFFFFFFFFFFFFFFFFFFFFFFFFFF1B
:10956000FFFFFFFFFFFFFFFFFFFFFFFFFDBEF81341
:1095700097037CA6FFFFFFFFFFFFFFFFFFFFFFFF3B
:10958000FFFFFFFFFFFFFFFFFFFFFFFFFFFFFFFFEB
:10959000FFFFFFFFFFFFFFFFFFFFFFFFFFFFFFFFDB
:1095A00075AD8531A218B29413A56D6BA218400851
:1095B000CF7BFFFFFFFFFFFFFFFFFFFFFFFFFFFF6F
:1095C000FFFFFFFFFFFFFFFFFFFFFFFFFFFFFFFFAB
:1095D000FFFFFFFFFBDEAE73494A14A538CE695288
:1095E000EF838952CA5A8631FFFFFFFF074200000E
:1095F000C739FFFFFFFFFFFFFFFFFFFFFFFFFFFF79
:10960000FFFFFFFFFFFFFFFFFFFFFFFFFFFFFFFF6A
:10961000FFFFFFFFDFF77A653603F94CBFEFFFFF6F
:10962000FFFFFFFFFFFFFFFFFFFFFFFFFFFFFFFF4A
:10963000FFFFFFFFFFFFFFFFFFFFFFFFFFFFFFFF3A
:10964000FFFFFFFFFFFFFFFFFFFFFFFFFFFFFFFF2A
:10965000FFFFFFFFFFFFFFFFFFFFFFFFFFFFFFFF1A
:10966000FFFFFFFFFFFFFFFFFFFFFFFFFFFFFFFF0A
:10967000FFFFFFFFFFFFFFFFFFFFFFFFFFFFFFFFFA
:10968000FFFFFFFFFFFFFFFFFFFFFFFFFFFFFFFFEA
:10969000FFFFFFFF5C9E770338245ED7FFFFFFFFCD
:1096A000FFFFFFFFFFFFFFFFFFFFFFFFFFFFFFFFCA
:1096B000FFFFFFFFFFFFFFFFFFFFFFFFFFFFFFFFBA
:1096C000FFFFFFFFFFFFFFFFFFFFAA5ACF7B863997
:1096D0001BE7FFFF1CE7C218811086319AD6FFFFF7
:1096E000FFFFFFFFFFFFFFFFFFFFFFFFFFFFFFFF8A
:1096F000FFFFFFFFFFFFFFFFFFFFB6BD65318110DA
:10970000284ABAD6FFFF4C6B0000284A4529C320DF
:10971000A218BADE79CE61108110D7BDFFFFFFFF1E
:10972000FFFFFFFFFFFFFFFFFFFFFFFFFFFFFFFF49
:10973000FFFFFFFFFFFFFFFFFFFFFFFFFFFFFFFF39
:10974000FFFF5C9E770338245ED7FFFFFFFFFFFF1C
:10975000FFFFFFFFFFFFFFFFFFFFFFFFFFFFFFFF19
:10976000FFFFFFFFFFFFFFFFFFFFFFFFFFFFFFFF09
:10977000FFFFFFFFFFFFFFFFFFFFFFFFFFFFFFFFF9
:10978000FFFFFFFFFFFFFFFFFFFFFFFFFFFFFFFFE9
:10979000FFFFFFFFFFFFFFFFFFFFFFFFFFFFFFFFD9
:1097A000FFFFFFFFFFFFFFFFFFFFFFFFFFFFFFFFC9
:1097B000FFFFFFFFFFFFFFFFFFFFFFFFDB7D360324
:1097C000F94CDFF7FFFFFFFFFFFFFFFFFFFFFFFF8A
:1097D000FFFFFFFFFFFFFFFFFFFFFFFFFFFFFFFF99
:1097E000FFFFFFFFFFFFFFFFFFFFFFFFFFFFFFFF89
:1097F000FFFF1BE745291BE7653154ADD6BDCB5AAA
:1098000081100000A218DBDEFFFFFFFFFFFFFFFF5C
:10981000FFFFFFFFFFFFFFFFFFFFFFFFFFFFFFFF58
:10982000FFFF1CE7442900004D6BFFFFFFFFFFFF18
:10983000284AE320B29CE3208110AA5A95B5442916
:109840004108D7BDFFFFFFFFFFFFFFFFFFFFFFFF47
:10985000FFFFFFFFFFFFFFFFFFFFFFFFFFFFFFFF18
:10986000FFFFFFFFFFFFFFFFFFFFFFFFFFFF1DC722
:10987000F80BB703FDBEFFFFFFFFFFFFFFFFFFFF7A
:10988000FFFFFFFFFFFFFFFFFFFFFFFFFFFFFFFFE8
:10989000FFFFFFFFFFFFFFFFFFFFFFFFFFFFFFFFD8
:1098A000FFFFFFFFFFFFFFFFFFFFFFFFFFFFFFFFC8
:1098B000FFFFFFFFFFFFFFFFFFFFFFFFFFFFFFFFB8
:1098C000FFFFFFFFFFFFFFFFFFFFFFFFFFFFFFFFA8
:1098D000FFFFFFFFFFFFFFFFFFFFFFFFFFFFFFFF98
:1098E000FFFFFFFF5A6536039A6DFFFFFFFFFFFF83
:1098F000FFFFFFFFFFFFFFFFFFFFDFFFBEF7FFFFE1
:10990000FFFFFFFFFFFFFFFFFFFFFFFFFFFFFFFF67
:10991000FFFFFFFFFFFFFFFFFFFFFFFFEF83695226
:10992000FFFFEF830000E320E320CA5AAE7B9AD604
:10993000FFFFFFFFFFFFFFFFFFFFFFFFFFFFFFFF37
:10994000FFFFFFFFFFFFFFFFFFFFFFFF75AD000001
:1099500061101CE7FFFFFFFF3CE78218C21881106F
:109960006110C2180C6324290000B29CFFFFFFFFA6
:10997000FFFFFFFFFFFFFFFFFFFFFFFFFFFFFFFFF7
:10998000FFFFFFFFFFFFFFFFFFFFFFFFFFFFFFFFE7
:10999000FFFFFFFFFFFFFFFFFFFF7EDF582C770376
:1099A0009DA6FFFFFFFFFFFFFFFFFFFFFFFFFFFF82
:1099B000FFFFFFFFFFFFFFFFFFFFFFFFFFFFFFFFB7
:1099C000FFFFFFFFFFFFFFFFFFFFFFFFFFFFFFFFA7
:1099D000FFFFFFFFFFFFFFFFFFFFFFFFFFFFFFFF97
:1099E000FFFFFFFFFFFFFFFFFFFFFFFFFFFFFFFF87
:1099F000FFFFFFFFFFFFFFFFFFFFFFFFFFFFFFFF77
:109A0000FFFFFFFFFFFFFFFFFFFFFFFF1A553603BA
:109A1000FB85FFFFFFFFFFFFFFFFFFFFFFFFFFFFD4
:109A2000FFFFFFFFEB6207429EF7FFFFFFFFFFFF15
:109A3000FFFFFFFFFFFFFFFFFFFFFFFFFFFFFFFF36
:109A4000FFFFFFFFFFFF8A5234ADFFFFBEF7C739AC
:109A500065317DEFFFFFFFFFFFFFFFFFFFFFFFFF10
:109A6000FFFFFFFFFFFFFFFFFFFFFFFFFFFFFFFF06
:109A7000FFFFFFFFFFFF3CE72C6B14A5FFFFFFFF7D
:109A8000FFFF9EF7AA5A75AD2C6B653140080000A8
:109A900004299294FFFFFFFFFFFFFFFFFFFFFFFF7F
:109AA000FFFFFFFFFFFFFFFFFFFFFFFFFFFFFFFFC6
:109AB000FFFFFFFFFFFFFFFFFFFFFFFFFFFFFFFFB6
:109AC000FFFFFFFFFFFFDFF7B93C57035C9EFFFF7F
:109AD000FFFFFFFFFFFFFFFFFFFFFFFFFFFFFFFF96
:109AE000FFFFFFFFFFFFFFFFFFFFFFFFFFFFFFFF86
:109AF000FFFFFFFFFFFFFFFFFFFFFFFFFFFFFFFF76
:109B0000FFFFFFFFFFFFFFFFFFFFFFFFFFFFFFFF65
:109B1000FFFFFFFFFFFFFFFFFFFFFFFFFFFFFFFF55
:109B2000FFFFFFFFFFFFFFFFFFFFFFFFFFFFFFFF45
:109B3000FFFFFFFFFA4C36035C96FFFFFFFFFFFFBE
:109B40000F84EB62FFFFBEFFDEFFFFFF5DEFE7412B
:109B5000A21844295DEFFFFFFFFFFFFFFFFFFFFF9C
:109B6000FFFFFFFFFFFFFFFFFFFFFFFFFFFF7DEF97
:109B7000484A9EF7FFFFFFFFDFFFD7BDDFFFFFFF74
:109B8000FFFFFFFFFFFFFFFFFFFFFFFFFFFFFFFFE5
:109B9000FFFFFFFFFFFFFFFFFFFFFFFFFFFFFFFFD5
:109BA000FFFFFFFFFFFFFFFFFFFFFFFFFFFFFFFFC5
:109BB000FFFFFFFF9EF71084B6BDBEF7FFFFFFFF5C
:109BC000FFFFFFFFFFFFFFFFFFFFFFFFFFFFFFFFA5
:109BD000FFFFFFFFFFFFFFFFFFFFFFFFFFFFFFFF95
:109BE000FFFFFFFFFFFFFFFFFFFFFFFFFFFFFFFF85
:109BF000FFFFFFFFFA4C36035C96FFFFFFFFFFFFFE
:109C0000FFFFFFFFFFFFFFFFFFFFFFFFFFFFFFFF64
:109C1000FFFFFFFFFFFFFFFFFFFFFFFFFFFFFFFF54
:109C2000FFFFFFFFFFFFFFFFFFFFFFFFFFFFFFFF44
:109C3000FFFFFFFFFFFFFFFFFFFFFFFFFFFFFFFF34
:109C4000FFFFFFFFFFFFFFFFFFFFFFFFFFFFFFFF24
:109C5000FFFFFFFFFFFFFFFFFFFFFFFFFA4C570370
:109C60005C9EFFFFFFFFFFFFFFFF074240081CE76E
:109C70008639D39CDFFF284AB6B53CE70842242941
:109C8000BADEFFFFFFFFFFFFFFFFFFFFFFFFFFFF4A
:109C9000FFFFFFFFFFFFDFFFAE7B308CFFFFFFFF0B
:109CA000FFFFFFFFFFFFFFFFFFFFFFFFFFFFFFFFC4
:109CB000FFFFFFFFFFFFFFFFFFFFFFFFFFFFFFFFB4
:109CC000FFFFFFFFFFFFFFFFFFFFFFFFFFFFFFFFA4
:109CD000FFFFFFFFFFFFFFFFFFFFFFFFFFFFFFFF94
:109CE000FFFFFFFFFFFFFFFFFFFFFFFFFFFFFFFF84
:109CF000FFFFFFFFFFFFFFFFFFFFFFFFFFFFFFFF74
:109D0000FFFFFFFFFFFFFFFFFFFFFFFFFFFFFFFF63
:109D1000FFFFFFFFFFFFFFFFDBDEDFFFFFFFFFFFB8
:109D20001A5536035C9EFFFFFFFFFFFFFFFFFFFF9B
:109D3000FFFFFFFFFFFFFFFFFFFFFFFFFFFFFFFF33
:109D4000FFFFFFFFFFFFFFFFFFFFFFFFFFFFFFFF23
:109D5000FFFFFFFFFFFFFFFFFFFFFFFFFFFFFFFF13
:109D6000FFFFFFFFFFFFFFFFFFFFFFFFFFFFFFFF03
:109D7000FFFFFFFFFFFFFFFFFFFFFFFFFFFFFFFFF3
:109D8000FFFFFFFF3A5536037C9EFFFFFFFFFFFFFB
:109D9000FFFFFFFFBAD6A63969524429DADE6D6BA0
:109DA0001084FFFFFFFFFFFFB29424291CE7FFFF91
:109DB000FFFFFFFFFFFFFFFFFFFFFFFFFFFFFFFFB3
:109DC0005DEFE741BEF7FFFFFFFFFFFFFFFFFFFF74
:109DD000FFFFFFFFFFFFFFFFFFFFFFFFFFFFFFFF93
:109DE000FFFFFFFFFFFFFFFFFFFFFFFFFFFFFFFF83
:109DF000FFFFFFFFFFFFFFFFFFFFFFFFFFFFFFFF73
:109E0000FFFFFFFFFFFFFFFFFFFFFFFFFFFFFFFF62
:109E1000FFFFFFFFFFFFFFFFFFFFFFFFFFFFFFFF52
:109E2000FFFFFFFFFFFFFFFFFFFFFFFFFFFFFFFF42
:109E3000FFFF3CE7CB5A7194FFFFFFFFFFFFFFFFDF
:109E400055AD2000508CFFFFFFFFFFFF1A4D570359
:109E50009CA6FFFFFFFFFFFFFFFFFFFFFFFFFFFFCE
:109E6000FFFFFFFFFFFFFFFFFFFFFFFFFFFFFFFF02
:109E7000FFFFFFFFFFFFFFFFFFFFFFFFFFFFFFFFF2
:109E8000FFFFFFFFFFFFFFFFFFFFFFFFFFFFFFFFE2
:109E9000FFFFFFFFFFFFFFFFFFFFFFFFFFFFFFFFD2
:109EA000FFFFFFFFFFFFFFFFFFFFFFFF9B6D36037D
:109EB0003C96FFFFFFFFFFFFFFFFFFFFFFFFFFFFDE
:109EC000FFFFC318284ADBDE00009294FFFFFFFF6C
:109ED000FFFFFFFFEB624C6BFFFFFFFFFFFFFFFF8A
:109EE000FFFFFFFFFFFFFFFFFFFFFFFF79CEFFFF39
:109EF000FFFFFFFFFFFFFFFFFFFFFFFFFFFFFFFF72
:109F0000FFFFFFFFFFFFFFFFDFEF9FDF5EC73EB7F3
:109F1000FEAEFEA6DDA6FDAE1EB73EC75ED79FE72E
:109F2000DFFFFFFFFFFFFFFFFFFFFFFFFFFFFFFF61
:109F3000FFFFFFFFFFFFFFFFFFFFFFFFFFFFFFFF31
:109F4000FFFFFFFFFFFFFFFFFFFFFFFFFFFFFFFF21
:109F5000FFFFFFFFFFFFFFFFFFFFFFFF6D7300002D
:109F60000000F3A4DFFF9AD6EB62200840080B63E1
:109F7000FFFFFFFFFFFFFFFFD9445703DDB6FFFFE1
:109F8000FFFFFFFFFFFFFFFFFFFFFFFFFFFFFFFFE1
:109F9000FFFFFFFFFFFFFFFFFFFFFFFFFFFFFFFFD1
:109FA000FFFFFFFFFFFFFFFFFFFFFFFFFFFFFFFFC1
:109FB000FFFFFFFFFFFFFFFFFFFFFFFFFFFFFFFFB1
:109FC000FFFFFFFFFFFFFFFFFFFFFFFFFFFFFFFFA1
:109FD000FFFFFFFFFB853603DB7DFFFFFFFFFFFF7A
:109FE000FFFFFFFFFFFFFFFFFFFFF39C2C6BAA5A51
:109FF000A218E320F7BDFFFFFFFFFFFFFFFF75ADD6
:10A00000E741FFFFFFFFFFFFFFFFFFFFFFFFFFFF36
:10A01000FFFFFFFFFFFFFFFFFFFFFFFFFFFFFFFF50
:10A02000FFFFFFFFFFFFFFFF9FE71EBF9D8E3D6607
:10A03000DC357C155C051B051B05FB04DB04BA0441
:10A04000BA04BA04BA04BA04DA0C1A255B3DDC651A
:10A050009D963ECFDFF7FFFFFFFFFFFFFFFFFFFFF4
:10A06000FFFFFFFFFFFFFFFFFFFFFFFFFFFFFFFF00
:10A07000FFFFFFFFFFFFFFFFFFFFFFFFFFFFFFFFF0
:10A08000FFFFFFFFFFFF75B5E741E3208218C739E7
:10A09000C3204008CE7BFBDE7DEFFFFFFFFFFFFF0D
:10A0A000FFFFDFF7793497033ECFFFFFFFFFFFFF8E
:10A0B000FFFFFFFFFFFFFFFFFFFFFFFFFFFFFFFFB0
:10A0C000FFFFFFFFFFFFFFFFFFFFFFFFFFFFFFFFA0
:10A0D000FFFFFFFFFFFFFFFFFFFFFFFFFFFFFFFF90
:10A0E000FFFFFFFFFFFFFFFFFFFFFFFFFFFFFFFF80
:10A0F000FFFFFFFFFFFFFFFFFFFFFFFF9DA63603F0
:10A100007A65FFFFFFFFFFFFFFFFFFFFFFFFFFFF7E
:10A11000FFFFB6BD2008BEF78D7324292C6B853157
:10A1200038C6FFFFFFFFFFFF13A5494AFFFFFFFFF0
:10A13000FFFFFFFFFFFFFFFFFFFFFFFFFFFFFFFF2F
:10A14000FFFFFFFFFFFFFFFFFFFFDFF75ECF9D96E3
:10A150001D669C457C2D5C255C1D5C0D5C055C05CD
:10A160003C053B051B051B05FB04FB04DB04DA0473
:10A17000BA04BA049A047904590439045904B91C7C
:10A180007B557C9E7EDFFFFFFFFFFFFFFFFFFFFF92
:10A19000FFFFFFFFFFFFFFFFFFFFFFFFFFFFFFFFCF
:10A1A000FFFFFFFF38C65DEF9EF75DEFFBE617C6CA
:10A1B00034ADCB5A41102008200861100F843CE7D1
:10A1C000FFFFFFFFFFFFFFFFFFFFFFFFFFFFBFEFEF
:10A1D000181C18149FEFFFFFFFFFFFFFFFFFFFFF9B
:10A1E000FFFFFFFFFFFFFFFFFFFFFFFFFFFFFFFF7F
:10A1F000FFFFFFFFFFFFFFFFFFFFFFFFFFFFFFFF6F
:10A20000FFFFFFFFFFFFFFFFFFFFFFFFFFFFFFFF5E
:10A21000FFFFFFFFFFFFFFFFFFFFFFFFFFFFFFFF4E
:10A22000FFFFFFFF3ECF9703B93CFFFFFFFFFFFF9C
:10A23000FFFFFFFFFFFFFFFFFFFFFFFF3CE7BAD677
:10A24000B6B5AE7B3084653161108E7379D65DEF23
:10A250009EF74D6BCF7BFFFFFFFFFFFFFFFFFFFF71
:10A26000FFFFFFFFFFFFFFFFFFFFFFFFFFFFFFFFFE
:10A270007FD7BE9EFD6DBC4D9C459C459C459C3D3D
:10A280009C357C2D7C1D5C0D5C053C053C053B052F
:10A290001B05FB04FB04FB04DA04DA04BA04BA0469
:10A2A0009A049A047904790459041804F8035904A7
:10A2B0001A457C9EBFEFFFFFFFFFFFFFFFFFFFFF81
:10A2C000FFFFFFFFFFFFFFFFFFFFFFFFFFFF0B632E
:10A2D0000842E7416531E3206110A2188531AE7371
:10A2E00075AD0B6320080000308CFFFFFFFFFFFF00
:10A2F000FFFFFFFFFFFFFFFFFFFF5ED79703B93CA4
:10A30000FFFFFFFFFFFFFFFFFFFFFFFFFFFFFFFF5D
:10A31000FFFFFFFFFFFFFFFFFFFFFFFFFFFFFFFF4D
:10A32000FFFFFFFFFFFFFFFFFFFFFFFFFFFFFFFF3D
:10A33000FFFFFFFFFFFFFFFFFFFFFFFFFFFFFFFF2D
:10A34000FFFFFFFFFFFFFFFFFFFFFFFFBFF7381C0F
:10A350001814BFEFFFFFFFFFFFFFFFFFFFFFFFFF2F
:10A36000FFFFFFFFFFFFFFFFFFFF2429C218C639D1
:10A370004010C3204429C218A2184531A21838CE73
:10A38000FFFFFFFFFFFFFFFFFFFFFFFFFFFFFFFFDD
:10A39000FFFFFFFFDFF73EC75D8EFD65DD5DDD5D25
:10A3A000DD5DBD55BC4DBC459C3D9C357C2D7C2563
:10A3B0007C0D5C055C053C053B051B051B05FB0492
:10A3C000FB04DA04DA04BA04BA049A049A0499047D
:10A3D00079047904590459043904F803D803591449
:10A3E000BB6D5ED7FFFFFFFFFFFFFFFFFFFFFFFF1C
:10A3F000FFFFFFFFFFFFFFFFFFFF9DF73CE71CE7AD
:10A40000BAD6DBDE7DEFFFFFFFFFFFFFFFFFF39C10
:10A4100069523CE7FFFFFFFFFFFFFFFFFFFFFFFF6A
:10A42000FFFFFFFFFFFFBDAE36039B6DFFFFFFFF8A
:10A43000FFFFFFFFFFFFFFFFFFFFFFFFFFFFFFFF2C
:10A44000FFFFFFFFFFFFFFFFFFFFFFFFFFFFFFFF1C
:10A45000FFFFFFFFFFFFFFFFFFFFFFFFFFFFFFFF0C
:10A46000FFFFFFFFFFFFFFFFFFFFFFFFFFFFFFFFFC
:10A47000FFFFFFFFFFFF1A4D77031EC7FFFFFFFF20
:10A48000FFFFFFFFFFFFFFFFFFFFFFFFFFFFFFFFDC
:10A49000FFFFFFFF1CE70F844008E320C639A21826
:10A4A000AA5AEF832008C3209EF7FFFFFFFFFFFF9C
:10A4B000FFFFFFFFFFFFFFFFFFFFDFF71EC75D8E00
:10A4C000FD6DFD6D1D6EFD6DFD65DD5DDD55BC4DEC
:10A4D000BC459C3D9C357C2D7C257C0D5C055C053C
:10A4E0003C053B051B051B05FB04FB04DA04DA04F1
:10A4F000BA04BA049A049A049904790479045904B0
:10A500005904390439041804F803B703F8035A5DF1
:10A510003ED7FFFFFFFFFFFFFFFFFFFFFFFFFFFF34
:10A52000FFFFFFFFFFFFFFFFFFFFFFFFFFFFFFFF3B
:10A53000FFFF4D6B75ADFFFFFFFFFFFFFFFFFFFF4D
:10A54000FFFFFFFFFFFFFFFFFFFFFFFFFFFFFFFF1B
:10A55000FFFFDB7536039CA6FFFFFFFFFFFFFFFF3A
:10A56000FFFFFFFFFFFFFFFFFFFFFFFFFFFFFFFFFB
:10A57000FFFFFFFFFFFFFFFFFFFFFFFFFFFFFFFFEB
:10A58000FFFFFFFFFFFFFFFFFFFFFFFFFFFFFFFFDB
:10A59000FFFFFFFFFFFFFFFFFFFFFFFFFFFF5C96D7
:10A5A00036033C8EFFFFFFFFFFFFFFFFFFFFFFFFB4
:10A5B000FFFFFFFFFFFFFFFFFFFFFFFFFFFF55ADA7
:10A5C000494AD29CF7C5284AC320E3205DEF55AD28
:10A5D000AE7BFFFFFFFFFFFFFFFFFFFFFFFFFFFF60
:10A5E000FFFF5ED79E963D7E3D7E3D7E1D761D6EB5
:10A5F000FD6DFD65DD5DDD55BC4DBC4D9C3D9C3D5F
:10A600009C2D7C257C155C055C053C053B051B05EC
:10A610001B05FB04FB04DB04DA04BA04BA04BA0425
:10A620009A049904790479045904590439043904C1
:10A63000180418041804F803B703F7037A659EE7B3
:10A64000FFFFFFFFFFFFFFFFFFFFFFFFFFFFFFFF1A
:10A65000FFFFFFFFFFFFFFFFFFFFF7C500000F84B5
:10A66000FFFFFFFFFFFFFFFFFFFFFFFFFFFFFFFFFA
:10A67000FFFFFFFFFFFFFFFFFFFFFFFFFFFFB93CF3
:10A68000B7037EDFFFFFFFFFFFFFFFFFFFFFFFFFBF
:10A69000FFFFFFFFFFFFFFFFFFFFFFFFFFFFFFFFCA
:10A6A000FFFFFFFFFFFFFFFFFFFFFFFFFFFFFFFFBA
:10A6B000FFFFFFFFFFFFFFFFFFFFFFFFFFFFFFFFAA
:10A6C000FFFFFFFFFFFF5ED797031A4DFFFFFFFF5E
:10A6D000FFFFFFFFFFFFFFFFFFFFFFFFFFFFFFFF8A
:10A6E000FFFFFFFFFFFFFFFF9AD6C218DBDEFFFF71
:10A6F00008424C6BB29C0742FFFFFFFFFFFFFFFFCA
:10A70000FFFFFFFFFFFFFFFF9FE7DEAE5D8E5D8E69
:10A710005D8E5D863D7E1D761D76FD6DFD65DD5D84
:10A72000DD55BD4DBC4D9C459C3D9C357C257C1527
:10A730005C055C053C053B051B051B05FB04FB0498
:10A74000DB04DA04BA04BA04BA049A04990479045A
:10A7500079045904590439043904180418041804F4
:10A76000F803F803F803970318143B96FFFFFFFF65
:10A77000FFFFFFFFFFFFFFFFFFFFFFFFFFFFFFFFE9
:10A78000FFFFFFFF0F840000518CFFFFFFFFFFFF63
:10A79000FFFFFFFFFFFFFFFFFFFFFFFFFFFFFFFFC9
:10A7A000FFFFFFFFFFFFFFFF9EE7B703B93CFFFF7F
:10A7B000FFFFFFFFFFFFFFFFFFFFFFFFFFFFFFFFA9
:10A7C000FFFFFFFFFFFFFFFFFFFFFFFFFFFFFFFF99
:10A7D000FFFFFFFFFFFFFFFFFFFFFFFFFFFFFFFF89
:10A7E000FFFFFFFFFFFFFFFFFFFFFFFFFFFFFFFF79
:10A7F0009934D80BBFEFFFFFFFFFFFFFFFFFFFFF05
:10A80000FFFFFFFFFFFFFFFFFFFFFFFFFFFFFFFF58
:10A81000FFFFFFFF14A58531DFFFBEF7DFFFFFFF5E
:10A8200085312C63FFFFFFFFFFFFFFFFFFFFFFFFEF
:10A830003ECF9E9E7E967E967E965D8E5D863D7E0A
:10A840001D761D76FD6DFD65DD5DDD55BC4DBC4D98
:10A850009C459C3D9C357C257C155C055C053C0538
:10A860003B051B051B05FB04FB04DB04DA04BA04EF
:10A87000BA04BA049A04990479047904590459046D
:10A8800039043904180418041804F803F803F80309
:10A89000F803D7039603B83C3ED7FFFFFFFFFFFF47
:10A8A000FFFFFFFFFFFFFFFFFFFFFFFFFFFF07426D
:10A8B000000055ADFFFFFFFFFFFFFFFFFFFFFFFFA2
:10A8C000FFFFFFFFFFFFFFFFFFFFFFFFFFFFFFFF98
:10A8D000FFFFFFFF9CA636031C8EFFFFFFFFFFFF5D
:10A8E000FFFFFFFFFFFFFFFFFFFFFFFFFFFFFFFF78
:10A8F000FFFFFFFFFFFFFFFFFFFFFFFFFFFFFFFF68
:10A90000FFFFFFFFFFFFFFFFFFFFFFFFFFFFFFFF57
:10A91000FFFFFFFFFFFFFFFF3C8E36039DAEFFFFF3
:10A92000FFFFFFFFFFFFFFFFFFFFFFFFFFFFFFFF37
:10A93000FFFFFFFFFFFFFFFFFFFFFFFFFFFFFFFF27
:10A94000C639EB5ADFFFFFFFFFFF79CE494ABEF75A
:10A95000FFFFFFFFFFFFDFEF1EBFBEA69EA69E9E6E
:10A960007E967E965D8E5D863D7E1D761D76FD6DA6
:10A97000FD65DD5DDD55BC4DBC4DBC459C3D9C354C
:10A980007C257C155C055C053C053B051B051B0512
:10A99000FB04FB04DB04DA04BA04BA04BA049A0424
:10A9A0007904590459045904590439043904380400
:10A9B0001804F803D803F803F803F803F703F703C0
:10A9C0009603D70B3B96FFFFFFFFFFFFFFFFFFFF45
:10A9D000FFFFFFFFFFFFF7BD2008EF83FFFFFFFF33
:10A9E000FFFFFFFFFFFFFFFFFFFFFFFFFFFFFFFF77
:10A9F000FFFFFFFFFFFFFFFFFFFFFFFFFFFFFFFF67
:10AA00001A4D97037EDFFFFFFFFFFFFFFFFFFFFFF2
:10AA1000FFFFFFFFFFFFFFFFFFFFFFFFFFFFFFFF46
:10AA2000FFFFFFFFFFFFFFFFFFFFFFFFFFFFFFFF36
:10AA3000FFFFFFFFFFFFFFFFFFFFFFFFFFFFFFFF26
:10AA40007EE797031A4DFFFFFFFFFFFFFFFFFFFFAA
:10AA5000FFFFFFFFFFFFFFFFFFFFFFFFFFFFFFFF06
:10AA6000FFFFFFFFFFFFFFFFFFFFBAD60000B29C12
:10AA7000FFFFFFFFFFFFFFFFFFFFFFFFFFFF9FE75E
:10AA8000FEB6DEAEDEAEBEA69E9E7E967E965D8E47
:10AA90005D863D7E1D761D76FD6DFD65DD5DDD55BA
:10AAA000BC4DBC4D9C459C3D9C357C257C155C0576
:10AAB0005C053C053B051B051B05FB04FB04DB0497
:10AAC000DA04BA049A047904BA04FA24FA2CD91CD8
:10AAD000990C59041904F80318045914B92CD934E1
:10AAE0009924F803D703D703D703F703D7037603D3
:10AAF000395DDFF7FFFFFFFFFFFFFFFFFFFFFFFFF6
:10AB00001CE79AD6FFFFFFFFFFFFFFFFFFFFFFFFDE
:10AB1000FFFFFFFFFFFFFFFFFFFFFFFFFFFFFFFF45
:10AB2000FFFFFFFFFFFFFFFFFFFF9FEFB703D93CD2
:10AB3000FFFFFFFFFFFFFFFFFFFFFFFFFFFFFFFF25
:10AB4000FFFFFFFFFFFFFFFFFFFFFFFFFFFFFFFF15
:10AB5000FFFFFFFFFFFFFFFFFFFFFFFFFFFFFFFF05
:10AB6000FFFFFFFFFFFFFFFFFFFF1A4DB7039EE749
:10AB7000FFFFFFFFFFFFFFFFFFFFFFFFFFFFFFFFE5
:10AB8000FFFFFFFFFFFFFFFFFFFFFFFFFFFFFFFFD5
:10AB9000FFFFFFFFFFFFF7BD9AD6FFFFFFFFFFFF9D
:10ABA000FFFFFFFFFFFF7FDFFEBEFEB6DEAEBEAEE5
:10ABB000BEA69E9E7E967E8E5D8E5D863D7E1D76B9
:10ABC0001D76FD6DFD65DD5DDD55BC4DBC4D9C45C7
:10ABD0009C3D9C357C257C155C055C053C053B0556
:10ABE0001B051B05FB04DB04BA049A04FB14BB4DD4
:10ABF000FC6DFC6DDB6D9B5D5A4D1A3DFA341A45B8
:10AC00009B65BB6D5A5DD934581C3814581C782488
:10AC100078243814F703F703D703760378347EDFFC
:10AC2000FFFFFFFFFFFFFFFFFFFFFFFFFFFFFFFF34
:10AC3000FFFFFFFFFFFFFFFFFFFFFFFFFFFFFFFF24
:10AC4000FFFFFFFFFFFFFFFFFFFFFFFFFFFFFFFF14
:10AC5000FFFFFFFFFFFF5C9636039DAEFFFFFFFF88
:10AC6000FFFFFFFFFFFFFFFFFFFFFFFFFFFFFFFFF4
:10AC7000FFFFFFFFFFFFFFFFFFFFFFFFFFFFFFFFE4
:10AC8000FFFFFFFFFFFFFFFFFFFFFFFFFFFFFFFFD4
:10AC9000FFFFFDBE57031C8EFFFFFFFFFFFFFFFFFF
:10ACA000FFFFFFFFFFFFFFFFFFFFFFFFFFFFFFFFB4
:10ACB000FFFFFFFFFFFFFFFFFFFFFFFFFFFFFFFFA4
:10ACC000FFFFFFFFFFFFFFFFFFFFFFFFFFFF7FD73C
:10ACD0001EBFFEBEFEB6DEAEBEAE9EA69E9E7E969B
:10ACE0007E8E5D863D863D7E1D761D76FD6DFD6505
:10ACF000DD5DDD55BC4DBC4D9C459C3D9C2D7C25B2
:10AD00007C155C055C053C053B051B05DB04BA04B2
:10AD10001B0DDC559D8E9D967D8E3C7EFB6DDB650F
:10AD2000DB751C7E1C86FC7DDB757B5D1A451A4538
:10AD30003A4D7A5D5A5D1A4DD93C78243814F703A0
:10AD4000F703D703D7037603171C1DCFFFFFFFFFC1
:10AD5000FFFFFFFFFFFFFFFFFFFFFFFFFFFFFFFF03
:10AD6000FFFFFFFFFFFFFFFFFFFFFFFFFFFFFFFFF3
:10AD7000FFFFFFFFFFFFFFFFFFFFFFFFFFFFFFFFE3
:10AD8000FFFF992C1814DFF7FFFFFFFFFFFFFFFF06
:10AD9000FFFFFFFFFFFFFFFFFFFFFFFFFFFFFFFFC3
:10ADA000FFFFFFFFFFFFFFFFFFFFFFFFFFFFFFFFB3
:10ADB000FFFFFFFFFFFFFFFFFFFFFFFF7924381CAE
:10ADC000FFFFFFFFFFFFFFFFFFFFFFFFFFFFFFFF93
:10ADD000FFFFFFFFFFFFFFFFFFFFFFFFFFFFFFFF83
:10ADE000FFFFFFFFFFFFFFFFFFFFFFFFFFFFFFFF73
:10ADF000FFFFFFFFFFFF5FD71EC71EBFFEBEFEB6F1
:10AE0000DEAEBEA69E9E9E9E7E967D8E5D863D8615
:10AE10003D7E1D761D6EFD6DFD65DD5DDD55BC4D18
:10AE2000BC4D9C3D9C357C2D7C257C155C055C05D2
:10AE30003C05FB04FB049C3D9D8EFDAEBD9E7D8EBE
:10AE40005C865C865C867C8E7C969D9E9D9E5C8EE0
:10AE5000FB75DB75FB7DDB7D9B65F9443814F803DE
:10AE6000F803D703B703D703D703B703B603960393
:10AE700096035503B603DDBEFFFFFFFFFFFFFFFF95
:10AE8000FFFFFFFFFFFFFFFFFFFFFFFFFFFFFFFFD2
:10AE9000FFFFFFFFFFFFFFFFFFFFFFFFFFFFFFFFC2
:10AEA000FFFFFFFFFFFFFFFFFFFFFFFF1DC7570370
:10AEB000FB85FFFFFFFFFFFFFFFFFFFFFFFFFFFF20
:10AEC000FFFFFFFFFFFFFFFFFFFFFFFFFFFFFFFF92
:10AED000FFFFFFFFFFFFFFFFFFFFFFFFFFFFFFFF82
:10AEE000FFFFFFFF7CA63603BDAEFFFFFFFFFFFFA6
:10AEF000FFFFFFFFFFFFFFFFFFFFFFFFFFFFFFFF62
:10AF0000FFFFFFFFFFFFFFFFFFFFFFFFFFFFFFFF51
:10AF1000FFFFFFFFFFFFFFFFFFFFFFFFFFFF5FD709
:10AF20001EC71EC7FEBEFEB6DEAEBEAEBEA69E9E4F
:10AF30007E967E965D8E5D863D7E3D7E1D761D6E87
:10AF4000FD65DD65DD5DBD55BC4DBC459C3D9C355D
:10AF50007C2D7C257C0D5C051B053B051C5EFEAE37
:10AF60003EBFDDA6BD9E3EC77ED71DBF3EC79EE746
:10AF70009EE71DBF7C963C861C863C8E1C86DB753E
:10AF8000BB75BB757A5DF944992C3814F803180C1D
:10AF9000581C78249834B834B83CB83498343724E2
:10AFA00017241DCFFFFFFFFFFFFFFFFFFFFFFFFF86
:10AFB000FFFFFFFFFFFFFFFFFFFFFFFFFFFFFFFFA1
:10AFC000FFFFFFFFFFFFFFFFFFFFFFFFFFFFFFFF91
:10AFD000FFFFFFFFFFFFFFFF1A4DB703BFEFFFFFAC
:10AFE000FFFFFFFFFFFFFFFFFFFFFFFFFFFFFFFF71
:10AFF000FFFFFFFFFFFFFFFFFFFFFFFFFFFFFFFF61
:10B00000FFFFFFFFFFFFFFFFFFFFFFFFFFFF381CFA
:10B01000992CFFFFFFFFFFFFFFFFFFFFFFFFFFFF79
:10B02000FFFFFFFFFFFFFFFFFFFFFFFFFFFFFFFF30
:10B03000FFFFFFFFFFFFFFFFFFFFFFFFFFFFFFFF20
:10B04000FFFFFFFFFFFF5FD71EC71EC71EBFFEBE6D
:10B05000FEB6DEAEBEA69E9E9E9E7E967D8E5D8ECA
:10B060003D863D7E1D7E1D761D6EFD65DD5DDD5DD3
:10B07000BD55BC4DBC459C3D9C357C2D5C1D3C05A7
:10B080005C0D5D6E5ECF7ED71EBF3EC7DFEFFFFF5C
:10B09000FFFFDFF7FFFFFFFF1EBF7C965C8E7C9EED
:10B0A000FDBE9FE79EE71DC7BDAE5C96FB85DB7DC1
:10B0B000DB7DFB7D1B8E3B8E3B8E1B8EFB85BA752D
:10B0C0009A6D7A65395DF94CD844772C17241DCFD9
:10B0D000FFFFFFFFFFFFFFFFFFFFFFFFFFFFFFFF80
:10B0E000FFFFFFFFFFFFFFFFFFFFFFFFFFFFFFFF70
:10B0F000FFFFFFFFFFFFFFFFFFFFFFFFFFFFFFFF60
:10B10000FFFF5EDF7703BB6DFFFFFFFFFFFFFFFF6A
:10B11000FFFFFFFFFFFFFFFFFFFFFFFFFFFFFFFF3F
:10B12000FFFFFFFFFFFFFFFFFFFFFFFFFFFFFFFF2F
:10B13000FFFFFFFFFFFF7C9E5703DDBEFFFFFFFF0A
:10B14000FFFFFFFFFFFFFFFFFFFFFFFFFFFFFFFF0F
:10B15000FFFFFFFFFFFFFFFFFFFFFFFFFFFFFFFFFF
:10B16000FFFFFFFFFFFFFFFFFFFFFFFFFFFF7FD797
:10B170001EBF1EBFFEBEFEBEFEB6DEAEBEAEBEA68D
:10B180009E9E7E967E967D8E5D863D863D7E1D765C
:10B190001D76FD6DFD65DD5DDD55BC4DBC4DBC45D1
:10B1A0009C3D9C355C1D7C1D7D769FDFFFFFBFEFC6
:10B1B0009FE7FFFFFFFFFFFFFFFFFFFFFFFFFFFF17
:10B1C0005ED73EC79EE7FFFFFFFFFFFFFFFFFFFFCA
:10B1D000DFF77EDF9EE7BFF79EE73DCF9CAE1B8E7D
:10B1E0009A6D3955D93C782C371CF60BB60375038C
:10B1F0003503350335031503B60B5ED7FFFFFFFF9D
:10B20000FFFFFFFFFFFFFFFFFFFFFFFFFFFFFFFF4E
:10B21000FFFFFFFFFFFFFFFFFFFFFFFFFFFFFFFF3E
:10B22000FFFFFFFFFFFFFFFFFFFFFFFFFFFF5A5D75
:10B23000B7039EE7FFFFFFFFFFFFFFFFFFFFFFFFDB
:10B24000FFFFFFFFFFFFFFFFFFFFFFFFFFFFFFFF0E
:10B25000FFFFFFFFFFFFFFFFFFFFFFFFFFFFFFFFFE
:10B26000581C992CFFFFFFFFFFFFFFFFFFFFFFFFB1
:10B27000FFFFFFFFFFFFFFFFFFFFFFFFFFFFFFFFDE
:10B28000FFFFFFFFFFFFFFFFFFFFFFFFFFFFFFFFCE
:10B29000FFFFFFFFFFFF7FDFFEB6FEBEFEBEFEB676
:10B2A000DEB6DEAEBEAEBEA69E9E9E9E7E967E8E16
:10B2B0005D8E5D863D7E3D7E1D761D6EFD65FD6568
:10B2C000DD5DDD55BD4DBC4D9C457C355C253D6649
:10B2D0009FDFFFFFFFFFFFFFFFFFFFFFFFFFFFFFFE
:10B2E000FFFFFFFFFFFFFFFFFFFFFFFFFFFFFFFF6E
:10B2F000FFFFFFFFFFFFFFFFFFFFFFFFBFEF3ECF9F
:10B300007C9EBB6D3A55F944F93CF944194D3955C9
:10B310005A5D9A6DBA75DB7DFB85FB85DB85BA7559
:10B3200059659844F854DFF7FFFFFFFFFFFFFFFF69
:10B33000FFFFFFFFFFFFFFFFFFFFFFFFFFFFFFFF1D
:10B34000FFFFFFFFFFFFFFFFFFFFFFFFFFFFFFFF0D
:10B35000FFFFFFFFFFFFFFFF5EDF7703DB75FFFFF0
:10B36000FFFFFFFFFFFFFFFFFFFFFFFFFFFFFFFFED
:10B37000FFFFFFFFFFFFFFFFFFFFFFFFFFFFFFFFDD
:10B38000FFFFFFFFFFFFFFFFBDAE5703BDAEFFFF97
:10B39000FFFFFFFFFFFFFFFFFFFFFFFFFFFFFFFFBD
:10B3A000FFFFFFFFFFFFFFFFFFFFFFFFFFFFFFFFAD
:10B3B000FFFFFFFFFFFFFFFFFFFFFFFFFFFF9FE715
:10B3C000DEB6FEB6FEB6FEB6DEAEDEAEBEAEBEA6E5
:10B3D0009E9E9E9E7D967E965D8E5D863D863D7E82
:10B3E0001D761D76FD6DFD65DD5DDD5DBD55BC4DDC
:10B3F0009C457C2DBC4D1EB7FFFFFFFFFFFFFFFFED
:10B40000FFFFFFFFFFFFFFFFFFFFFFFFFFFFFFFF4C
:10B41000FFFFFFFFFFFFFFFFFFFFFFFFFFFF9EE7B5
:10B42000FDBE5C96FB7DDB75FB7D3C8E9DA6FDBE67
:10B430003ECF5EDF7EDF5ED71DCFFDBE9CAE5C9E45
:10B440001B8EBA7D7A6D395DF94CB8449834B613C9
:10B45000F854FFFFFFFFFFFFFFFFFFFFFFFFFFFFAE
:10B46000FFFFFFFFFFFFFFFFFFFFFFFFFFFFFFFFEC
:10B47000FFFFFFFFFFFFFFFFFFFFFFFFFFFFFFFFDC
:10B48000FFFFFFFF3A4DD80BBFEFFFFFFFFFFFFFAE
:10B49000FFFFFFFFFFFFFFFFFFFFFFFFFFFFFFFFBC
:10B4A000FFFFFFFFFFFFFFFFFFFFFFFFFFFFFFFFAC
:10B4B000FFFFB934581CFFFFFFFFFFFFFFFFFFFF37
:10B4C000FFFFFFFFFFFFFFFF5DEFBAD63CE7FFFF87
:10B4D000FFFFFFFFFFFFFFFFFFFFFFFFFFFFFFFF7C
:10B4E000FFFFFFFFFFFFDFF7DEAEDEAEDEAEDEAE5C
:10B4F000DEAEBEAEBEA6BEA69E9E9E9E7E967E96EC
:10B500007D8E5D865D863D7E3D7E1D761D6EFD6D6C
:10B51000FD65DD5DDD55BC559C457C357D86DFF7E1
:10B52000FFFFFFFFFFFFFFFFFFFFFFFFFFFFFFFF2B
:10B53000FFFFFFFFFFFFFFFFFFFFFFFFFFFFFFFF1B
:10B54000FFFFFFFFFFFF9EE75ED77EDF9EE79FE7DF
:10B550007EDF3ECFBDAE1C867A65F944992C381447
:10B56000F703B703B70396037603760375037503F2
:10B57000750375037503750395033403FA85FFFF9F
:10B58000FFFFFFFFFFFFFFFFFFFFFFFFFFFFFFFFCB
:10B59000FFFFFFFFFFFFFFFFFFFFFFFFFFFFFFFFBB
:10B5A000FFFFFFFFFFFFFFFFFFFFFFFFFFFF1DCFBD
:10B5B00057033C96FFFFFFFFFFFFFFFFFFFFFFFF6B
:10B5C000FFFFFFFFFFFFFFFFFFFFFFFFFFFFFFFF8B
:10B5D000FFFFFFFFFFFFFFFFFFFF3ECF77033C961C
:10B5E000FFFFFFFFFFFFFFFF34AD494A59CEFFFFCA
:10B5F0009EF7A63920088110F39CFFFFFFFFFFFF95
:10B60000FFFFFFFFFFFFFFFFFFFFFFFFFFFFFFFF4A
:10B61000FEB6BEA6BEAEBEAEBEAEBEA6BEA69E9ECA
:10B620009E9E9E9E7E967E967D8E5D8E5D863D7EE6
:10B630003D7E1D761D76FD6DFD65DD5DDD5DDD55B7
:10B640009C3DDC553EC7FFFFFFFFFFFFFFFFFFFFF5
:10B65000FFFFFFFFFFFFFFFFFFFFFFFFFFFFFFFFFA
:10B66000FFFFFFFFFFFFFFFFFFFFFFFFFFFFFFFFEA
:10B670007EDFDDAE1C7E3A4DB9243804D803B80312
:10B68000B703B703D703D703D703D703D703F7030A
:10B69000D703D703D603D603B603B603B603B60360
:10B6A000B6039603750375031DCFFFFFFFFFFFFF72
:10B6B000FFFFFFFFFFFFFFFFFFFFFFFFFFFFFFFF9A
:10B6C000FFFFFFFFFFFFFFFFFFFFFFFFFFFFFFFF8A
:10B6D000FFFFFFFFFFFFFFFFFFFFB92C581CFFFF1D
:10B6E000FFFFFFFFFFFFFFFFFFFFFFFFFFFFFFFF6A
:10B6F000FFFFFFFFFFFFFFFFFFFFFFFFFFFFFFFF5A
:10B70000FFFFFFFF7A65B703BFEFFFFFFFFFFFFFFC
:10B71000FFFF89520000B29CFFFFFFFF494AE7414B
:10B720002429A2183CE7FFFFFFFFFFFFFFFFFFFFF9
:10B73000FFFFFFFFFFFFFFFF3ECF9E9EBEA6BEA600
:10B740009EA69E9E9E9E9E9E9E9E7E967E967E9689
:10B750007D8E5D8E5D863D7E3D7E1D761D761D6EE9
:10B76000FD65FD65DD5DBD557C3D5D7EBFEFFFFF89
:10B77000FFFFFFFFFFFFFFFFFFFFFFFFFFFFFFFFD9
:10B78000FFFFFFFFFFFFFFFFFFFFFFFFFFFFFFFFC9
:10B79000FFFF9EDFBDA6BB5DDA2459041804F80341
:10B7A00018041804180418041804F803F803F8031C
:10B7B000F703F703F703F703F703D703D703D6031A
:10B7C000D603B603B603B603B603B60395039503D3
:10B7D0005503372CDFFFFFFFFFFFFFFFFFFFFFFFDA
:10B7E000FFFFBEF7B6BDAA5AE7418A523CE7FFFF0A
:10B7F000FFFFFFFFFFFFFFFFFFFFBAD6BAD6FFFF35
:10B80000FFFFFFFF9CA65703FDBEFFFFFFFFFFFFEB
:10B81000FFFFFFFFFFFFFFFFFFFFFFFFFFFFFFFF38
:10B82000FFFFFFFFFFFFFFFFFFFFFFFFDFF7D80373
:10B830005A5DFFFFFFFFFFFFFFFFFFFFC639200834
:10B8400038CEFFFFFFFF518C96B56D730000D7BD5A
:10B85000FFFFFFFFFFFFFFFFFFFFFFFFFFFFFFFFF8
:10B86000BFEF7E969E9E9E9E9E9E9E9E9E9E9E9EAE
:10B870007E967E967E967E8E5D8E5D865D863D7E14
:10B880003D7E1D761D761D6EFD6DFD65DD5DBD5534
:10B890009C45BE9EFFFFFFFFFFFFFFFFFFFFFFFF77
:10B8A000FFFFFFFFFFFFFFFFFFFFFFFFFFFFFFFFA8
:10B8B000FFFFFFFFFFFF7EDF7D8E5B3D9A0C59048B
:10B8C0003904590459045904590439043904180431
:10B8D00018041804F803F803F803F703F703F70351
:10B8E000F703D703D703D703D603D603B603B603AC
:10B8F000B603B603B6039503950395031403BA7D07
:10B90000FFFFFFFFFFFFFFFFFFFFFFFF10840000AF
:10B91000A2188531863959CEFFFF34AD8E733CE7CE
:10B92000DFFF75AD61100C63FFFFFFFFFFFFDFF767
:10B93000F80B3A55FFFFFFFFFFFFFFFFFFFFFFFF81
:10B94000FFFFFFFFFFFFFFFFFFFFFFFFFFFFFFFF07
:10B95000FFFFFFFFFFFF9CA65703FDC6FFFFFFFF92
:10B96000FFFFFFFF1BE7E3202008B6B53CE7E741F8
:10B97000C639DBDE9AD600008D73FFFFFFFFFFFFA5
:10B98000FFFFFFFFFFFFFFFFFFFFDEAE5D8E7E9636
:10B990007E967E967E967E967E967E967E8E5D8E38
:10B9A0005D8E5D863D863D7E3D7E1D761D761D6EDF
:10B9B000FD6DFD65DD65BD55BC551EBFFFFFFFFF7D
:10B9C000FFFFFFFFFFFFFFFFFFFFFFFFFFFFFFFF87
:10B9D000FFFFFFFFFFFFFFFFFFFF9FE79D969B45D8
:10B9E000BA047A047904990499047904790459040D
:10B9F0005904390439041804180418041804F80305
:10BA0000F803F803F703F703F703F703D703D703A4
:10BA1000D703D603D603B603B603B603B603B603FD
:10BA2000950395039503750375035ED7FFFFFFFF2D
:10BA3000FFFFFFFFFFFFDBDEB6B55DEFFFFFF7BDEA
:10BA40006952E74161100000284AE7410000C3182D
:10BA5000F7BDFFFFFFFFFFFFFFFF7B65D703BFEFD2
:10BA6000FFFFFFFFFFFFFFFFFFFFFFFFFFFFFFFFE6
:10BA7000FFFFFFFFFFFFFFFFFFFFFFFFFFFFFFFFD6
:10BA8000FA443814FFFFFFFFFFFFFFFFD7BD442933
:10BA90008110A2187194B6B5000041108952FBDEE6
:10BAA0000C63200875ADFFFFFFFFFFFFFFFFFFFFE7
:10BAB000FFFF5ED73D867D8E7E8E7E8E7E8E7E8E55
:10BAC0007E8E7D8E5D8E5D8E5D865D863D7E3D7E4D
:10BAD0003D7E1D761D761D6EFD6DFD65FD65BD55BA
:10BAE000DC5D7ED7FFFFFFFFFFFFFFFFFFFFFFFFD4
:10BAF000FFFFFFFFFFFFFFFFFFFFFFFFFFFFFFFF56
:10BB00001EB7DC55FB0C9A049A049A049A049A0412
:10BB10009A049904790479045904590439043904BC
:10BB2000180418041804F803F803F803F803F703DB
:10BB3000F703F703F703D703D703D603D603D603D8
:10BB4000B603B603B603B6039603950395039503B0
:10BB500095033403D84CFFFFFFFFFFFFFFFFFFFFFC
:10BB6000FFFFFFFFFFFFFFFFFFFF718C0000A21828
:10BB7000C218A21882180842242924290742FFFF6C
:10BB8000FFFFFFFF1DC777037CA6FFFFFFFFFFFF3F
:10BB9000FFFFFFFFFFFFFFFFFFFFFFFFFFFFFFFFB5
:10BBA000FFFFFFFFFFFFFFFFBFEFB703BB75FFFF07
:10BBB000FFFFFFFFFFFFEF8300002008AA5A7194E8
:10BBC00038CE6D73A218400845298D73811041103D
:10BBD00018C6FFFFFFFFFFFFFFFFFFFF7D963D86BB
:10BBE0005D865D8E5D8E5D8E5D865D865D865D8625
:10BBF0003D863D7E3D7E3D7E3D7E1D761D761D6EE5
:10BC0000FD6DFD65FD65BD55FD659FDFFFFFFFFF18
:10BC1000FFFFFFFFFFFFFFFFFFFFFFFFFFFFFFFF34
:10BC2000FFFFFFFFBFEF9D8E7B2DBB04BA04DA043C
:10BC3000BA047A04FA145B3D9904990479047904EE
:10BC4000590459045904390439043904F803B70371
:10BC5000B703B703B703B703D703D703F703F70354
:10BC6000D703D703D603D603B603B603B603B6038A
:10BC7000B603960395039503950395037503340363
:10BC8000DDC6FFFFFFFFFFFFFFFFFFFF5CEF6D73F0
:10BC900075ADFFFF5DEF55ADC739C2188531C218CC
:10BCA0008531E320EB62695234AD9EF7FFFFFFFF61
:10BCB0003814FA44FFFFFFFFFFFFFFFFFFFFFFFF06
:10BCC000FFFFFFFFFFFFFFFFFFFFFFFFFFFFFFFF84
:10BCD000FFFF7CA677031DC7FFFFFFFFFFFFFFFFEE
:10BCE0001CE76952C21892949AD696B5DFFFA21843
:10BCF000C21861108110C218A218B6B5FFFFFFFF6D
:10BD0000FFFFFFFF3EC71D763D7E3D863D863D869B
:10BD10005D863D863D863D7E3D7E3D7E3D7E3D7E13
:10BD20001D761D761D761D6EFD6DFD65FD65BD558F
:10BD3000FC659FE7FFFFFFFFFFFFFFFFFFFFFFFF28
:10BD4000FFFFFFFFFFFFFFFFFFFF9FDF5D763B155C
:10BD5000DB04DB04FB04DB049A04BA04FC65BFE7E4
:10BD6000DB5D590499047904790459045904590490
:10BD700039043804FA441B86BDAE7C9EFB7D7A5D97
:10BD8000D93C581CD7039603B703D703D703D60370
:10BD9000D603B603B603B603B603B60395039503FD
:10BDA00095039503950395033403973CFFFFFFFF2D
:10BDB000FFFFFFFF7DEF284AE7410008D29C96B5C0
:10BDC000C318653103212429E320C218E7418218F2
:10BDD000EB6261108E73FFFFFFFF9B6DD703BFEF18
:10BDE000FFFFFFFFFFFFFFFFFFFFFFFFFFFFFFFF63
:10BDF000FFFFFFFFFFFFFFFFFFFFFFFF3A4D18149C
:10BE0000FFFFFFFFFFFFFFFFFFFFFFFFFFFF5DEFF4
:10BE10009EF7FFFF34A5DFFFC74181108531E32086
:10BE20006110E741FFFFFFFFFFFFFFFFFFFF5D86A0
:10BE30001D763D7E3D7E3D7E3D7E3D7E3D7E3D7E52
:10BE40003D7E3D7E1D7E1D761D761D761D6EFD6D33
:10BE5000FD65FD65DD65BD55DD5D9FDFFFFFFFFF16
:10BE6000FFFFFFFFFFFFFFFFFFFFFFFFFFFFFFFFE2
:10BE7000BFE75D763B0DFB04FB041B05FB04BA0426
:10BE8000BA04DC5D5ED7FFFF9FE79904790479046B
:10BE90007904790459045904390439041804F8035D
:10BEA00059145A5DFDBEFFFFFFFFFFFFDFF71DCFF7
:10BEB0001B8EB83496039603D603D603B603B60397
:10BEC000B603B603B603950395039503950395034F
:10BED000750375033403DDC6FFFFFFFFFFFF518CC1
:10BEE000284AFFFF96B5C639284A40086110C21893
:10BEF00004296D73A21824290321242900008E73BC
:10BF0000FFFFFFFFFDBE7703BDAEFFFFFFFFFFFF9B
:10BF1000FFFFFFFFFFFFFFFFFFFFFFFFFFFFFFFF31
:10BF2000FFFFFFFFDFF7F80B5A5DFFFFFFFFFFFF8B
:10BF3000FFFFFFFFFFFFFFFFFFFFFFFF38C6E3200C
:10BF4000EB62284A20080F8413A500008A52FFFFE5
:10BF5000FFFFFFFFFFFF5ECFFD651D761D761D769F
:10BF60001D761D761D761D761D761D761D761D7639
:10BF70001D6E1D6EFD6DFD65FD65FD65DD5DBD55CF
:10BF8000BC557ED7FFFFFFFFFFFFFFFFFFFFFFFF57
:10BF9000FFFFFFFFFFFFDFF79D865C15FB041B051E
:10BFA0001B051B05DB04DA04BC4D5EC7FFFFFFFF6A
:10BFB000FFFF1C7659049904790479045904590443
:10BFC00059043904390418041804F803B703B703F3
:10BFD000992C7C9EFFFFFFFFFFFFFFFFFFFFDDBEF1
:10BFE000D84476039603B603B603B603B6039603A6
:10BFF0009503950395039503950375037503140342
:10C00000D74CFFFFFFFFFFFF75B5E320BAD6FFFF58
:10C01000EF832008695285318110853104216952EE
:10C0200034AD3CE7BEF717C6BEF7FFFFFFFFDFF7F3
:10C03000F8037A65FFFFFFFFFFFFFFFFFFFFFFFF32
:10C04000FFFFFFFFFFFFFFFFFFFFFFFFFFFF1EC719
:10C0500077039DA6FFFFFFFFFFFFFFFFFFFFFFFF2F
:10C06000FFFFFFFFFFFFDBDE0B63A21881108218CA
:10C070000742EF8300003084FFFFFFFFFFFFFFFF59
:10C080007D8EFD651D6E1D6E1D6E1D761D761D76E9
:10C090001D761D6E1D6E1D6EFD6DFD6DFD65FD65D4
:10C0A000FD65DD5DDD5DDD559C4D3EBFFFFFFFFFA6
:10C0B000FFFFFFFFFFFFFFFFFFFFFFFFFFFF1EA7C9
:10C0C0009C25FB041B053B051B05DB04DB04BC4571
:10C0D0003EBFFFFFFFFFFFFFFFFFDFF7FA1479040A
:10C0E0007904790479045904590439043904380469
:10C0F00018041804F803F803F803B7039703B93CCE
:10C100003ED7FFFFFFFFFFFFFFFFFFFF5C9ED60B49
:10C110007503B603B603B60396039503950395031B
:10C120009503950375037503540354035EDFFFFF06
:10C13000FFFFFFFF7194C639494AE3202008D39CD2
:10C14000BEF77194284ACF7BD39CFFFFFFFFFFFF10
:10C15000FFFFFFFFFFFFFFFFFFFF1A45581CFFFF18
:10C16000FFFFFFFFFFFFFFFFFFFFFFFFFFFFFFFFDF
:10C17000FFFFFFFFFFFFFFFF1C8697039EE7FFFF08
:10C18000FFFFFFFFFFFFFFFFFFFFFFFFFFFFFFFFBF
:10C19000FFFF3CE70321A21881109194718C0000ED
:10C1A00075ADFFFFFFFFFFFF9FDFDD5DFD65FD65F7
:10C1B000FD6DFD6DFD6DFD6DFD6DFD6DFD6DFD6D2F
:10C1C000FD65FD65FD65FD65DD5DDD5DDD5DDD5507
:10C1D0009C45BD9EFFFFFFFFFFFFFFFFFFFFFFFF2F
:10C1E000FFFFFFFFBFE73D561C053C053C053B0537
:10C1F000FB04DB049C3D1EB7FFFFFFFFFFFFFFFFBB
:10C20000FFFFFFFFDDA6590499047904790479043E
:10C210005904590439043904180418041804F8039B
:10C22000F803F803F803F7039703D70BBCAEFFFF3F
:10C23000FFFFFFFFFFFFFFFF3ED737245503B60385
:10C24000B60395039503950395039503950375032D
:10C2500075037403F302997DFFFFFFFFFFFFFFFFEC
:10C26000DEF77DEFDBDEA2183084FFFFFFFFE74142
:10C270002008EB5AFFFFFFFFFFFFFFFFFFFFFFFF5D
:10C28000FFFFFFFF3C9697037EDFFFFFFFFFFFFFEF
:10C29000FFFFFFFFFFFFFFFFFFFFFFFFFFFFFFFFAE
:10C2A000FFFFFA44581CFFFFFFFFFFFFFFFFFFFFE8
:10C2B000FFFFFFFFFFFFFFFFFFFFFFFFF7BD40088E
:10C2C000C320A21824296D7338CEBEF7FFFFFFFFED
:10C2D000FFFFBEA6BC4DDD5DFD65FD65FD65FD6531
:10C2E000FD65FD65FD65FD65FD65DD65DD5DDD5DAE
:10C2F000DD5DDD5DDD55DC559C453D76FFFFFFFFD7
:10C30000FFFFFFFFFFFFFFFFFFFFFFFF1EB77C1DCB
:10C310001C055C053C051B05FB047C2DFEA6FFFFF0
:10C32000FFFFFFFFFFFFFFFFFFFFFFFFFFFF5B3D83
:10C3300059047904590439041904F803F803F8037B
:10C34000D803F80318041804F803F803F803F703F4
:10C35000F703F703B703B603DDBEFFFFFFFFFFFFE1
:10C36000FFFFFFFF9EE737245503B60395039503B0
:10C3700095039503950375037503750374033403DF
:10C380001624FFFFFFFFFFFFFFFFFFFFFFFFFFFF81
:10C39000FBDE5DEFFFFFFFFFD7BDA6399AD6FFFF9B
:10C3A000FFFFFFFFFFFFFFFFFFFFFFFFFFFF3ECF8E
:10C3B00077039DA6FFFFFFFFFFFFFFFFFFFFFFFFCC
:10C3C000FFFFFFFFFFFFFFFFFFFFFFFF180C5A5D9E
:10C3D000FFFFFFFFFFFFFFFFFFFFFFFFFFFFFFFF6D
:10C3E000FFFFFFFFFFFF9EF765316110C218A21823
:10C3F00020086D73BEF7FFFFFFFFFFFF1D6EBD55E9
:10C40000DD5DDD5DDD5DDD5DDD5DDD5DDD5DDD5D5C
:10C41000DD5DDD5DDD5DDD5DDD55DD55BD55BC4DB5
:10C42000BC4DBC4D9FE7FFFFFFFFFFFFFFFFFFFF7E
:10C43000FFFFFFFF9D863C053C055C051C05FB04DA
:10C440007C25DD9EFFFFFFFFFFFFFFFFFFFFFFFFDC
:10C45000FFFFFFFFFFFF5ECF590439045904991411
:10C460003A3DBB5D1C7E3C861C86BB65FA3C1804CD
:10C47000B703F803F803F803F703F703F703F70329
:10C48000B7031714BFEFFFFFFFFFFFFFFFFFFFFF23
:10C490007EDFD613750395039503950395039503E6
:10C4A000750375037503740354033403FDC6FFFF5E
:10C4B000FFFFFFFFFFFFFFFFFFFFFFFFFFFFFFFF8C
:10C4C000FFFFFFFFFFFFFFFFFFFFFFFFFFFFFFFF7C
:10C4D000FFFFFFFFFFFFFFFFDFF7F8039B65FFFF95
:10C4E000FFFFFFFFFFFFFFFFFFFFFFFFFFFFFFFF5C
:10C4F000FFFFFFFF7EDF97035C96FFFFFFFFFFFF5D
:10C50000FFFFFFFFFFFFFFFFFFFFFFFFFFFFFFFF3B
:10C51000FFFFD7BDC32061104008611000008D737C
:10C52000FFFFFFFF7FD79C45BC4DBD55BD55DD5579
:10C53000DD55DD55DD55DD55DD55DD55DD55BD558B
:10C54000BD55BC55BC4DBC4DBC4D7C35BD9EFFFFA3
:10C55000FFFFFFFFFFFFFFFFFFFFFFF73D5E1C0533
:10C560005C053C05FB047C1DBD8EDFF7FFFFFFFF74
:10C57000FFFFFFFFFFFFFFFFFFFFFFFFFFFFFFFFCB
:10C58000BB5DBA241C761EBFBFEFFFFFFFFFFFFF9E
:10C59000FFFFFFFFFFFFFFFF5ED77A65D703F803BA
:10C5A000F803F703F703F703F703D70376039A6D4E
:10C5B000FFFFFFFFFFFFFFFFFFFFFFFFDDBE550394
:10C5C000950395039503950395037503750374030C
:10C5D00074037403F3027975FFFFFFFFFFFFFFFF92
:10C5E000FFFFFFFFFFFFFFFFFFFFFFFFFFFFFFFF5B
:10C5F000FFFFFFFFFFFFFFFFFFFFFFFFFFFFFFFF4B
:10C60000FFFFFFFFB934992CFFFFFFFFFFFFFFFF84
:10C61000FFFFFFFFFFFFFFFFFFFFFFFFFFFFBDAEBD
:10C6200077031DC7FFFFFFFFFFFFFFFFFFFFFFFFB8
:10C63000FFFFFFFFFFFFFFFFFFFFFFFFFFFF3CE7E5
:10C6400058CEB294284A042175B5FFFFFFFFDE9E45
:10C650007C3DBC4DBC4DBC4DBC4DBC4DBC4DBC4DE2
:10C66000BC4DBC4DBC4DBC4DBC4DBC4DBC4DBC4D82
:10C67000BC459C3DBC45BFEFFFFFFFFFFFFFFFFF39
:10C68000FFFFDFF7FC453C053C051B055C159D865F
:10C69000DFEFFFFFFFFFFFFFFFFFFFFFFFFFFFFFDA
:10C6A000FFFFFFFFFFFFFFFFDFFF1EC7FFF7FFFFDB
:10C6B000FFFFFFFFFFFFFFFFFFFFFFFFFFFFFFFF8A
:10C6C000FFFFFFFFFFFF7C9ED703F703F703F7038E
:10C6D000F703F703D703B603D6037EE7FFFFFFFF99
:10C6E000FFFFFFFFFFFFFFFF9975340395039503DD
:10C6F000950395037503750374037403740334037E
:10C70000362CFFFFFFFFFFFFFFFFFFFFFFFFFFFFD5
:10C71000FFFFFFFFFFFFFFFFFFFFFFFFFFFFFFFF29
:10C72000FFFFFFFFFFFFFFFFFFFFFFFFFFFF9B6D0F
:10C73000F803DFF7FFFFFFFFFFFFFFFFFFFFFFFF34
:10C74000FFFFFFFFFFFFFFFFFB7DB703BFEFFFFF13
:10C75000FFFFFFFFFFFFFFFFFFFFFFFFFFFFFFFFE9
:10C76000FFFFFFFFFFFFFFFFFFFFFFFFFFFFFFFFD9
:10C77000BEF7FFFFFFFFFFFF1D6E7C359C45BC45EC
:10C78000BC45BC4DBC4DBC4DBC4DBC4DBC4DBC4D69
:10C79000BC45BC45BC45BC459C459C3D7C2D5D7E57
:10C7A000FFFFFFFFFFFFFFFFFFFFFFFFFC4D1C052B
:10C7B0005C057C1D9D7EBFEFFFFFFFFFFFFFFFFFBE
:10C7C000FFFFFFFFFFFFFFFFFFFFFFFFFFFFFFFF79
:10C7D000FFFFFFFFFFFFFFFFFFFFFFFFFFFFFFFF69
:10C7E000FFFFFFFFFFFFFFFFFFFFFFFFFFFFFFFF59
:10C7F000FFFFDB759703F703F703F703D703D703AF
:10C80000D7035603DB7DFFFFFFFFFFFFFFFFFFFFA7
:10C81000FFFFDFF7161C550395039503750375039A
:10C820007503740374037403540374035EDFFFFF22
:10C83000FFFFFFFFFFFFFFFFFFFFFFFFFFFFFFFF08
:10C84000FFFFFFFFFFFFFFFFFFFFFFFFFFFFFFFFF8
:10C85000FFFFFFFFFFFFFFFF7C9E97035ED7FFFFF9
:10C86000FFFFFFFFFFFFFFFFFFFFFFFFFFFFFFFFD8
:10C87000FFFF3A553814FFFFFFFFFFFFFFFFFFFFE9
:10C88000FFFFFFFFFFFFFFFFFFFFFFFFFFFFFFFFB8
:10C89000FFFFFFFFFFFFFFFFFFFFFFFFFFFFFFFFA8
:10C8A000BFEF9C3D7C359C3D9C3D9C3D9C3D9C450B
:10C8B0009C459C459C459C459C3D9C3D9C3D9C3D90
:10C8C0009C3D9C3D9C355C251EAFFFFFFFFFFFFF9D
:10C8D000FFFFFFFF7D6E1C055C051B051EAFFFFF04
:10C8E000FFFFFFFFFFFFFFFFFFFFFFFFFFFFFFFF58
:10C8F000FFFFFFFFFFFFFFFFFFFFFFFFFFFFFFFF48
:10C90000FFFFDFF7FFFFFFFFFFFFFFFFFFFFFFFF5F
:10C91000FFFFFFFFFFFFFFFFFFFFFFFFBFEF180C51
:10C92000D703F703F703D703D703D7039603B83C1E
:10C93000FFFFFFFFFFFFFFFFFFFFFFFFFFFFFB8D7D
:10C94000340395039503750375037403740374032B
:10C950007403740313035BA6FFFFFFFFFFFFFFFFDA
:10C96000FFFFFFFFFFFFFFFFFFFFFFFFFFFFFFFFD7
:10C97000FFFFFFFFFFFFFFFFFFFFFFFFFFFFFFFFC7
:10C98000FFFF1DC77703BDB6FFFFFFFFFFFFFFFFE0
:10C99000FFFFFFFFFFFFFFFFFFFFFFFF992CD93CC9
:10C9A000FFFFFFFFFFFFFFFFFFFFFFFFFFFFFFFF97
:10C9B000FFFFFFFFFFFFFFFFFFFFFFFFFFFFFFFF87
:10C9C000FFFFFFFFFFFFFFFFFFFF5EC75C257C351A
:10C9D0009C359C359C359C3D9C3D9C3D9C3D9C3DA7
:10C9E0009C3D9C3D9C3D9C359C357C357C357C2D0F
:10C9F0007C257ED7FFFFFFFFFFFFFFFF7ECF3C05BB
:10CA00003C053C051B05DC3DFFFFFFFFFFFFFFFF73
:10CA1000FFFFFFFFFFFFFFFFFFFFFFFFFFFFFFFF26
:10CA2000FFFFFFFF9EDF1C7E7B4DFA2CBA1CDA2431
:10CA30003A453C8EBFEFFFFFFFFFFFFFFFFFFFFF09
:10CA4000FFFFFFFFFFFFFFFF394D9603F703D703FB
:10CA5000D703D703D60396035724FFFFFFFFFFFF3B
:10CA6000FFFFFFFFFFFFFFFF9EE7B50B7503750399
:10CA7000750375037403740374037403740313035D
:10CA8000596DFFFFFFFFFFFFFFFFFFFFFFFFFFFFEE
:10CA9000FFFFFFFFFFFFFFFFFFFFFFFFFFFFFFFFA6
:10CAA000FFFFFFFFFFFFFFFFFFFFFFFF9EE7B70353
:10CAB0001C8EFFFFFFFFFFFFFFFFFFFFFFFFFFFFDA
:10CAC000FFFFFFFFFFFF180C7A65FFFFFFFFFFFF6F
:10CAD000FFFFFFFFFFFFFFFFFFFFFFFFFFFFFFFF66
:10CAE000FFFFFFFFFFFFFFFFFFFFFFFFFFFFFFFF56
:10CAF000FFFFFFFFDE9E3C157C257C2D7C2D7C2DD1
:10CB00007C2D9C2D9C357C357C359C359C2D7C2D3D
:10CB10007C2D7C2D7C2D7C257C257C1D9FDFFFFFC3
:10CB2000FFFFFFFFFFFF9D7EFB043C053B053B0530
:10CB30001B057ECFFFFFFFFFFFFFFFFFFFFFFFFF94
:10CB4000FFFFFFFFFFFFFFFFFFFFFFFFFFFFBB5DDB
:10CB5000F80339043904390439041804D803792452
:10CB60003ECFFFFFFFFFFFFFFFFFFFFFFFFFFFFFC6
:10CB7000FFFF1B869603F703D703D703D703D6031C
:10CB800096035724FFFFFFFFFFFFFFFFFFFFFFFF9D
:10CB9000FFFFFFFF973C34037503750375037403B0
:10CBA00074037403740374033403773CFFFFFFFFC3
:10CBB000FFFFFFFFFFFFFFFFFFFFFFFFFFFFFFFF85
:10CBC000FFFFFFFFFFFFFFFFFFFFFFFFFFFFFFFF75
:10CBD000FFFFFFFFFFFFDFFF180C7B65FFFFFFFF7D
:10CBE000FFFFFFFFFFFFFFFFFFFFFFFFFFFF9FEFC5
:10CBF000B703FB85FFFFFFFFFFFFFFFFFFFFFFFF07
:10CC0000FFFFFFFFFFFFFFFFFFFFFFFFFFFFFFFF34
:10CC1000FFFFFFFFFFFFFFFFFFFFFFFFFFFF5D665F
:10CC20003C057C157C1D7C1D7C257C257C257C257C
:10CC30007C257C257C257C257C257C257C1D7C1DFC
:10CC40007C157C0D3C055EC7FFFFFFFFFFFFFFFF6C
:10CC5000BD86DB043B053B051B05DB04FEA6FFFF91
:10CC6000FFFFFFFFFFFFFFFFFFFFFFFFFFFFFFFFD4
:10CC7000FFFFFFFFFFFFBFE7990C59047904590438
:10CC80005904590439043904D803B92CFFFFFFFFB4
:10CC9000FFFFFFFFFFFFFFFFFFFFFFFF9CA69603C5
:10CCA000D703D703D703D603D6037503D844FFFFB2
:10CCB000FFFFFFFFFFFFFFFFFFFFFFFFFFFF997574
:10CCC00034037503750374037403740374037403EA
:10CCD00074033403D51BDFF7FFFFFFFFFFFFFFFFE8
:10CCE000FFFFFFFFFFFFFFFFFFFFFFFFFFFFFFFF54
:10CCF000FFFFFFFFFFFFFFFFFFFFFFFFFFFFFFFF44
:10CD0000FFFF7924FA44FFFFFFFFFFFFFFFFFFFF54
:10CD1000FFFFFFFFFFFFFFFF5ED797037C9EFFFF34
:10CD2000FFFFFFFFFFFFFFFFFFFFFFFFFFFFFFFF13
:10CD3000FFFFFFFFFFFFFFFFFFFFFFFFFFFFFFFF03
:10CD4000FFFFFFFFFFFFFFFFFC3D3C055C055C05AF
:10CD50007C0D7C0D7C157C157C157C157C157C155B
:10CD60007C157C157C0D7C0D7C055C055C051C052B
:10CD70007D6EFFFFFFFFFFFFFFFFDFEFFC4D1B0599
:10CD8000DB04DB04BA043EBFFFFFFFFFFFFFFFFF32
:10CD9000FFFFFFFFFFFFFFFFFFFFFFFFFFFFFFFFA3
:10CDA0005C8E19047904590459045904390439046E
:10CDB00018041804F8033ECFFFFFFFFFFFFFFFFF3B
:10CDC000FFFFFFFFFFFFBDB6B703D703D703D703AE
:10CDD000D603D60355039A75FFFFFFFFFFFFFFFF42
:10CDE000FFFFFFFFFFFFFFFF1B9614037503750393
:10CDF000740374037403740374037403540374039B
:10CE00005EDFFFFFFFFFFFFFFFFFFFFFFFFFFFFFF3
:10CE1000FFFFFFFFFFFFFFFFFFFFFFFFFFFFFFFF22
:10CE2000FFFFFFFFFFFFFFFFFFFFFFFFD93C992C34
:10CE3000FFFFFFFFFFFFFFFFFFFFFFFFFFFFFFFF02
:10CE4000FFFF1EC79703DDB6FFFFFFFFFFFFFFFFDA
:10CE5000FFFFFFFFFFFFFFFFFFFFFFFFFFFFFFFFE2
:10CE6000FFFFFFFFFFFFFFFFFFFFFFFFFFFFFFFFD2
:10CE7000FFFF9C1D3C055C055C055C055C055C05D5
:10CE80005C055C055C055C055C055C055C055C059A
:10CE90005C055C055C055C053C053B053EBFFFFF92
:10CEA000FFFFFFFFFFFFFFFF7ED7DD9E7D865D76E4
:10CEB000DFEFFFFFFFFFFFFFFFFFFFFFFFFFFFFFB2
:10CEC000FFFFFFFFFFFFFFFFFFFFFA2439045904B4
:10CED0005904590439043904380418041804B703F0
:10CEE0007C9EFFFFFFFFFFFFFFFFFFFFFFFFFFFF36
:10CEF0009CAE9603D703D703D603D603B6037503B8
:10CF0000DDBEFFFFFFFFFFFFFFFFFFFFFFFFFFFF94
:10CF1000FFFF5BA634037503740374037403740387
:10CF200074037403740354033403DCBEFFFFFFFF78
:10CF3000FFFFFFFFFFFFFFFFFFFFFFFFFFFFFFFF01
:10CF4000FFFFFFFFFFFFFFFFFFFFFFFFFFFFFFFFF1
:10CF5000FFFFFFFFFFFF5A553814FFFFFFFFFFFFE2
:10CF6000FFFFFFFFFFFFFFFFFFFFFFFFBDB69703C0
:10CF70001EC7FFFFFFFFFFFFFFFFFFFFFFFFFFFFDA
:10CF8000FFFFFFFFFFFFFFFFFFFFFFFFFFFFFFFFB1
:10CF9000FFFFFFFFFFFFFFFFFFFFBFE75C0D3B054C
:10CFA0003C053C053C055C055C055C055C055C05D9
:10CFB0005C055C055C055C055C053C053C053C05C9
:10CFC0003C053C051B051B055D767ED7FFFFFFFF7B
:10CFD000FFFFFFFFFFFFFFFFFFFFFFFFFFFFFFFF61
:10CFE000FFFFFFFFFFFFFFFFFFFFFFFFFFFFFFFF51
:10CFF000FFFFFDB6390459045904590439043904B2
:10D000003904180418041804B703DB7DFFFFFFFF81
:10D01000FFFFFFFFFFFFFFFFFFFF3C967603D703F5
:10D02000D603D603D6039603371CDFF7FFFFFFFFB7
:10D03000FFFFFFFFFFFFFFFFFFFFFFFF5BA61403E4
:10D040007503740374037403740374037403740327
:10D05000740313035BA6FFFFFFFFFFFFFFFFFFFF4C
:10D06000FFFFFFFFFFFFFFFFFFFFFFFFFFFFFFFFD0
:10D07000FFFFFFFFFFFFFFFFFFFFFFFFFFFFFFFFC0
:10D080009B6DF803DFF7FFFFFFFFFFFFFFFFFFFFD1
:10D09000FFFFFFFFFFFF7CA697035ED7FFFFFFFFA9
:10D0A000FFFFFFFFFFFFFFFFFFFFFFFFFFFFFFFF90
:10D0B000FFFFFFFFFFFFFFFFFFFFFFFFFFFFFFFF80
:10D0C000FFFFFFFF9ED73B053B053B053B053C05AE
:10D0D0003C053C053C053C053C053C053C053C0548
:10D0E0003C053C053C053C051B055B153B053B052C
:10D0F0001B05DB041B059C351C669D8EDDA6DD9E95
:10D100007D867D86FFFFFFFFFFFFFFFFFFFFFFFF25
:10D11000FFFFFFFFFFFFFFFFFFFFFFFF7B4D190436
:10D12000590459043904390439041804180418043A
:10D130001804B703DB75FFFFFFFFFFFFFFFFFFFFD3
:10D14000FFFFFFFF7A657603D703D603D603B60346
:10D150005503BA7DFFFFFFFFFFFFFFFFFFFFFFFF4C
:10D16000FFFFFFFFFFFF1B96140374037403740398
:10D170007403740374037403740374031303FA8D48
:10D18000FFFFFFFFFFFFFFFFFFFFFFFFFFFFFFFFAF
:10D19000FFFFFFFFFFFFFFFFFFFFFFFFFFFFFFFF9F
:10D1A000FFFFFFFFFFFFFFFFFFFFDB7DD803BFEFA8
:10D1B000FFFFFFFFFFFFFFFFFFFFFFFFFFFFFFFF7F
:10D1C0005C9E97037EDFFFFFFFFFFFFFFFFFFFFF78
:10D1D000FFFFFFFFFFFFFFFFFFFFFFFFFFFFFFFF5F
:10D1E000FFFFFFFFFFFFFFFFFFFFFFFFFFFF5ECF20
:10D1F000FB041B051B053B053B053B053B053B05B0
:10D200003B053B053B053B053B053B053B051B053E
:10D210001B05DC457B1D1B051B051B051B05FB04B6
:10D22000DB04BB04BA04BA04BA045A043C6EFFFF20
:10D23000FFFFFFFFFFFFFFFFFFFFFFFFFFFFFFFFFE
:10D24000FFFFFFFF9EDF7904590459045904390494
:10D2500039041804180418041804F803B7033C969A
:10D26000FFFFFFFFFFFFFFFFFFFFFFFFFFFF782430
:10D270009603D603D603B6039603D60B7EE7FFFFCD
:10D28000FFFFFFFFFFFFFFFFFFFFFFFFFFFFFFFFAE
:10D2900079751403740374037403740374037403BF
:10D2A0007403740374031303997DFFFFFFFFFFFFF3
:10D2B000FFFFFFFFFFFFFFFFFFFFFFFFFFFFFFFF7E
:10D2C000FFFFFFFFFFFFFFFFFFFFFFFFFFFFFFFF6E
:10D2D000FFFFFFFF1C8EB7039FE7FFFFFFFFFFFF6E
:10D2E000FFFFFFFFFFFFFFFFFFFF3C96B7037EE757
:10D2F000FFFFFFFFFFFFFFFFFFFFFFFFFFFFFFFF3E
:10D30000FFFFFFFFFFFFFFFFFFFFFFFFFFFFFFFF2D
:10D31000FFFFFFFFFFFFFFFF3EC7FB041B051B05D1
:10D320001B051B051B051B051B051B051B051B05FD
:10D330001B051B051B05FB04FB047D7EBC3DFB049C
:10D340001B05FB04FB04FB04FB04FB04FB04DB04E4
:10D35000DB04DA04DA0CBFE7FFFFFFFFFFFFFFFF8C
:10D36000FFFFFFFFFFFFFFFFFFFFFFFFFFFF1C7E31
:10D370001804590459043904390418041804180409
:10D380001804F803F803B703DDB6FFFFFFFFFFFF44
:10D39000FFFFFFFFFFFF1DCFB603B603D603D60383
:10D3A000B60355039A6DFFFFFFFFFFFFFFFFFFFF6F
:10D3B000FFFFFFFFFFFFFFFFFFFFB84C34037403C5
:10D3C00074037403740374037403740374037403A5
:10D3D00013037975FFFFFFFFFFFFFFFFFFFFFFFF55
:10D3E000FFFFFFFFFFFFFFFFFFFFFFFFFFFFFFFF4D
:10D3F000FFFFFFFFFFFFFFFFFFFFFFFFFFFF3C9669
:10D40000B7037EE7FFFFFFFFFFFFFFFFFFFFFFFF09
:10D41000FFFFFFFF1C8EB7039EE7FFFFFFFFFFFF2D
:10D42000FFFFFFFFFFFFFFFFFFFFFFFFFFFFFFFF0C
:10D43000FFFFFFFFFFFFFFFFFFFFFFFFFFFFFFFFFC
:10D44000FFFF3EBFDB04FB04FB04FB04FB041B05E6
:10D450001B051B051B051B051B051B051B05FB04ED
:10D46000FB04FDA61C5EDB04FB04FB04FB04FB04C5
:10D47000FB04FB04DB04DA04DA04DA047A04FC6556
:10D48000FFFFFFFFFFFFFFFFFFFFFFFFFFFFFFFFAC
:10D49000FFFFFFFFFFFFFFFFBA1C390459043904E7
:10D4A00039041804180418041804F803F803F803DE
:10D4B000F7035EDFFFFFFFFFFFFFFFFFFFFFFFFF41
:10D4C0009A6D7603D603D603B6039603F6139EEF42
:10D4D000FFFFFFFFFFFFFFFFFFFFFFFFFFFFFFFF5C
:10D4E000FFFFDFF7F61B5403740374037403740324
:10D4F000740374037403740374031303596DFFFFFF
:10D50000FFFFFFFFFFFFFFFFFFFFFFFFFFFFFFFF2B
:10D51000FFFFFFFFFFFFFFFFFFFFFFFFFFFFFFFF1B
:10D52000FFFFFFFFFFFFFFFF5C96B7037EDFFFFFFC
:10D53000FFFFFFFFFFFFFFFFFFFFFFFFFFFF1C8E4F
:10D54000B7039EE7FFFFFFFFFFFFFFFFFFFFFFFFA8
:10D55000FFFFFFFFFFFFFFFFFFFFFFFFFFFFFFFFDB
:10D56000FFFFFFFFFFFFFFFFFFFFFFFF3EBFBA040C
:10D57000FB04FB04FB04FB04FB04FB04FB04FB04B3
:10D58000FB04FB04FB04FB04DB043EBF9D8EBA04DA
:10D59000FB04FB04FB04FB04DB04DA04DA04DA0416
:10D5A000DA04BA04BA049A045ED7FFFFFFFFFFFF54
:10D5B000FFFFFFFFFFFFFFFFFFFFFFFFFFFFFFFF7B
:10D5C000DDAE1804390439043904180418041804A9
:10D5D0001804F803F803F803B703B934FFFFFFFF9B
:10D5E000FFFFFFFFFFFFFFFF9EE7F70BB603D6032A
:10D5F000D603B60355033B96FFFFFFFFFFFFFFFF78
:10D60000FFFFFFFFFFFFFFFFFFFFFFFFFDC634032C
:10D610007403740374037403740374037403740352
:10D62000740374031303596DFFFFFFFFFFFFFFFF38
:10D63000FFFFFFFFFFFFFFFFFFFFFFFFFFFFFFFFFA
:10D64000FFFFFFFFFFFFFFFFFFFFFFFFFFFFFFFFEA
:10D65000FFFF5C96B7037EDFFFFFFFFFFFFFFFFFCB
:10D66000FFFFFFFFFFFFFFFF3C8EB7037EE7FFFFDB
:10D67000FFFFFFFFFFFFFFFFFFFFFFFFFFFFFFFFBA
:10D68000FFFFFFFFFFFFFFFFFFFFFFFFFFFFFFFFAA
:10D69000FFFFFFFFFFFF3EBFBA04DB04DB04FB0418
:10D6A000FB04FB04FB04FB04FB04FB04FB04DB04A2
:10D6B000BA041EAF7ECFBA04DB04DB04DB04DA0459
:10D6C000DA04DA04DA04DA04BA04BA04BA047A042A
:10D6D0009B4DFFFFFFFFFFFFFFFFFFFFFFFFFFFF70
:10D6E000FFFFFFFFFFFFFFFFFFFF3A45F80339048D
:10D6F000390418041804180418041804F803F8036B
:10D70000F80397037CA6FFFFFFFFFFFFFFFFFFFF6C
:10D71000FFFF9A6D7603D603D603B6035503B844CC
:10D72000FFFFFFFFFFFFFFFFFFFFFFFFFFFFFFFF09
:10D73000FFFFFFFFFFFF7975130374037403740386
:10D740007403740374037403740374037403130382
:10D750007975FFFFFFFFFFFFFFFFFFFFFFFFFFFFE9
:10D76000FFFFFFFFFFFFFFFFFFFFFFFFFFFFFFFFC9
:10D77000FFFFFFFFFFFFFFFFFFFFFFFF3C96B70329
:10D780007EE7FFFFFFFFFFFFFFFFFFFFFFFFFFFF42
:10D79000FFFF5C9697037EDFFFFFFFFFFFFFFFFFAA
:10D7A000FFFFFFFFFFFFFFFFFFFFFFFFFFFFFFFF89
:10D7B000FFFFFFFFFFFFFFFFFFFFFFFFFFFFFFFF79
:10D7C0005ECFBA04DA04DA04DA04DA04DA04DA043A
:10D7D000DB04DB04DB04DB049A049D8EFFFF3B1DAE
:10D7E000BA04DA04DA04DA04DA04DA04BA04BA04A9
:10D7F000BA04BA04BA04BA0479041EBFFFFFFFFFDB
:10D80000FFFFFFFFFFFFFFFFFFFFFFFFFFFFFFFF28
:10D81000FFFF5ED7380439043904180418041804CB
:10D820001804F803F803F803F803B703982CFFFF74
:10D83000FFFFFFFFFFFFFFFFFFFF3ECFB603B60373
:10D84000D603B6039603D60B7EDFFFFFFFFFFFFF75
:10D85000FFFFFFFFFFFFFFFFFFFFFFFFFFFFFFFFD8
:10D86000F61B3403740374037403740374037403A6
:10D8700074037403740374031303997DFFFFFFFFA4
:10D88000FFFFFFFFFFFFFFFFFFFFFFFFFFFFFFFFA8
:10D89000FFFFFFFFFFFFFFFFFFFFFFFFFFFFFFFF98
:10D8A000FFFFFFFFFFFF1C8EB7039EE7FFFFFFFF99
:10D8B000FFFFFFFFFFFFFFFFFFFFFFFF7DA69703B7
:10D8C0005ED7FFFFFFFFFFFFFFFFFFFFFFFFFFFF31
:10D8D0009EF78D731CE7DBDE8952EF83DFFFFFFFCE
:10D8E000FFFFFFFFFFFFFFFFFFFF7ED7BA04BA0471
:10D8F000BA04BA04DA04DA04DA04DA04DA04DA0478
:10D900007A041C66FFFF3C767A04DA04BA04BA048F
:10D91000BA04BA04BA04BA04BA04BA04BA04BA0417
:10D9200079045B35FFFFFFFFFFFFFFFFFFFFFFFFF6
:10D93000FFFFFFFFFFFFFFFFFFFFFFFFDB75F803A8
:10D9400039041804180418041804F803F803F80339
:10D95000F803F803B703DDBEFFFFFFFFFFFFFFFF84
:10D96000FFFFFFFF98347603D603D603B603750393
:10D970009CAEFFFFFFFFFFFFFFFFFFFFFFFFFFFF6B
:10D98000FFFFFFFFFFFFFFFF9CAE13037403740351
:10D9900074037403740374037403740374037403CF
:10D9A00074031303DA8DFFFFFFFFFFFFFFFFFFFF8D
:10D9B000FFFFFFFF75AD59CEFFFFFFFFFFFFFFFF2A
:10D9C000FFFFFFFFFFFFFFFFFFFFFFFFFFFFFFFF67
:10D9D000FB7DD703BFEFFFFFFFFFFFFFFFFFFFFF51
:10D9E000FFFFFFFFFFFFBDB697031EC7FFFFFFFF4F
:10D9F000FFFFFFFFFFFFFFFFFFFFEF83EF7BDFFF77
:10DA00000B63B6BDEF8334ADFFFFFFFFFFFFFFFFEA
:10DA1000FFFFFFFF9FE7DA0CBA04BA04BA04BA04A6
:10DA2000BA04BA04BA04BA049A045B2DFFFF7EDF7D
:10DA3000BA04BA04BA04BA04BA04BA04BA04BA04F6
:10DA4000BA04BA049A049A049A045904DDAEFFFF9A
:10DA5000FFFFFFFFFFFFFFFFFFFFFFFFFFFFFFFFD6
:10DA6000FFFFFFFFDFF779141804180418041804E7
:10DA70001804F803F803F803F803F80397039A6D02
:10DA8000FFFFFFFFFFFFFFFFFFFFFFFF9A6D760322
:10DA9000D603D603B6035503BA75FFFFFFFFFFFF9A
:10DAA000FFFFFFFFFFFFFFFFFFFFFFFFFFFFFFFF86
:10DAB000FFFF773C1403740374037403740374034B
:10DAC00074037403740374037403740313033B9E9D
:10DAD000FFFFFFFFFFFFFFFFFFFFFFFFFFFF38CE4E
:10DAE000284AB6B5FFFFFFFFFFFFFFFFFFFFFFFF65
:10DAF000FFFFFFFFFFFFFFFFFFFF9B6DF803DFF757
:10DB0000FFFFFFFFFFFFFFFFFFFFFFFFFFFFFFFF25
:10DB1000FDC69703DDB6FFFFFFFFFFFFFFFFFFFF1F
:10DB2000FFFFFFFF2C6B5DEFFFFF8A52FFFF18C660
:10DB30001084FFFFFFFFFFFFFFFFFFFFFFFFDFF787
:10DB4000FA1C9A04BA04BA04BA04BA04BA04BA04AD
:10DB50009A04BA047ED7FFFFDC5D7A04BA04BA04E3
:10DB6000BA04BA04BA049A049A049A049A049A0465
:10DB70009A0459041A25FFFFFFFFFFFFFFFFFFFF75
:10DB8000FFFFFFFFFFFFFFFFFFFFFFFFFFFF9DA660
:10DB9000D8031804180418041804F803F803F80349
:10DBA000F803F8039703B934FFFFFFFFFFFFFFFF00
:10DBB000FFFFFFFF3B967603B603D603B60355037C
:10DBC000F94CFFFFFFFFFFFFFFFFFFFFFFFFFFFF1E
:10DBD000FFFFFFFFFFFFFFFFFFFFDCBE3403540327
:10DBE000740374037403740374037403740374037D
:10DBF0007403740354033403BCBEFFFFFFFFFFFF35
:10DC0000FFFFFFFFFFFFFFFFFFFF7DEF4C6B9294D5
:10DC1000DADE5DEFDFFFFFFFFFFFFFFFFFFFFFFF2C
:10DC2000FFFFFFFF5A553814FFFFFFFFFFFFFFFF05
:10DC3000FFFFFFFFFFFFFFFFFFFF5ED797037C9E05
:10DC4000FFFFFFFFFFFFFFFFFFFFFFFFFFFFCE7B99
:10DC500096B5BAD6AA5A9EF7AA5A96B5FFFFFFFF05
:10DC6000FFFFFFFFFFFFFFFFFFFF5B3579049A0413
:10DC70009A049A049A049A04BA0459045C86FFFF31
:10DC80007EDF9A049A049A049A049A049A049A04E5
:10DC90009A049A049A0499049904990439049D9E5B
:10DCA000FFFFFFFFFFFFFFFFFFFFFFFFFFFFFFFF84
:10DCB000FFFFFFFFFFFFFFFFFA3CD8031804180423
:10DCC0001804F803F803F803F803F803B703581C23
:10DCD0009EE7FFFFFFFFFFFFFFFFFFFF7CA696030E
:10DCE000B603D603B6035503983CDFF7FFFFFFFFEB
:10DCF000FFFFFFFFFFFFFFFFFFFFFFFFFFFFFFFF34
:10DD0000FFFFFFFF5634140374037403740374039A
:10DD1000740374037403740374037403740354036B
:10DD200054033DD7FFFFFFFFFFFFFFFFFFFFFFFF94
:10DD3000FFFFFFFFFBDE6D73E7410B638A52BAD62C
:10DD4000FFFFFFFFFFFFFFFFFFFFFFFFFFFFF93CAC
:10DD5000992CFFFFFFFFFFFFFFFFFFFFFFFFFFFF0C
:10DD6000FFFFFFFF9FE7B703FB85FFFFFFFFFFFFFD
:10DD7000FFFFFFFFFFFFFFFF1CE7EB62284A18C60B
:10DD80007DEF55ADFFFFFFFFFFFFFFFFFFFFFFFF31
:10DD9000FFFFFFFFBB5D590499049A049A049A049B
:10DDA0009A0479041A2DFFFFFFFF1C7659049A0488
:10DDB0009A049A049A049904990499049904790498
:10DDC000790479045904DA1CDFF7FFFFFFFFFFFF36
:10DDD000FFFFFFFFFFFFFFFFFFFFFFFFFFFFFFFF53
:10DDE0003ECFF80318041804F803F803F803F80307
:10DDF000F803F803B703381C5ED7FFFFFFFFFFFFF0
:10DE0000FFFFFFFF5C9E9603B603D603D6035503C0
:10DE1000572CBFEFFFFFFFFFFFFFFFFFFFFFFFFFDD
:10DE2000FFFFFFFFFFFFFFFFFFFFFFFF3B9E13030F
:10DE3000740374037403740374037403740374032A
:10DE400074037403740374035403B513BFF7FFFF23
:10DE5000FFFFFFFFFFFFFFFFFFFFFFFF1084284AC8
:10DE600034A5FFFFFFFFDFFFFFFFFFFFFFFFFFFF07
:10DE7000FFFFFFFFFFFFFFFF7924FA44FFFFFFFFD3
:10DE8000FFFFFFFFFFFFFFFFFFFFFFFFFFFFFFFFA2
:10DE9000180C7A65FFFFFFFFFFFFFFFFFFFFFFFF8B
:10DEA000FFFFFFFFFFFFFFFFFFFF7DEFFFFFFFFF14
:10DEB000FFFFFFFFFFFFFFFFFFFFFFFFFFFF3C86AE
:10DEC0003904790479047904790499045904DDAE9C
:10DED000FFFFFFFFFA1C790499049904790479047F
:10DEE00079047904790479047904790479041904AA
:10DEF0005C8EFFFFFFFFFFFFFFFFFFFFFFFFFFFF46
:10DF0000FFFFFFFFFFFFFFFFFFFF9B65B803180444
:10DF1000F803F803F803F803F803F8039703581C11
:10DF20005ED7FFFFFFFFFFFFFFFFFFFFFB859603AD
:10DF3000B603D603D6035503572C9EE7FFFFFFFF1A
:10DF4000FFFFFFFFFFFFFFFFFFFFFFFFFFFFFFFFE1
:10DF5000FFFFFFFF9EEFB5133403740374037403D4
:10DF600074037403740374037403740374037403F9
:10DF7000740334035634FFFFFFFFFFFFFFFFFFFF73
:10DF8000FFFFFFFF7DEF9294BEF7FFFFFFFFFFFF54
:10DF9000FFFFFFFFFFFFFFFFFFFFFFFFFFFFFFFF91
:10DFA000FFFF180C7B65FFFFFFFFFFFFFFFFFFFF79
:10DFB000FFFFFFFFFFFFFFFFFFFF992CD93CFFFF93
:10DFC000FFFFFFFFFFFFFFFFFFFFFFFFFFFFFFFF61
:10DFD00075AD89528A52AA5275B5FFFFFFFFFFFF48
:10DFE000FFFFFFFFFFFFFFFFFDB63904790479044F
:10DFF0007904790439041A2DFFFFFFFF3EC7590445
:10E000007904790479047904790479047904790428
:10E0100079045904590439049914DFEFFFFFFFFF15
:10E02000FFFFFFFFFFFFFFFFFFFFFFFFFFFFFFFF00
:10E03000FFFFBFEF380CF803F803F803F803F80309
:10E04000F803F703970398347EDFFFFFFFFFFFFF1E
:10E05000FFFFBFEF395D7603B603D603D603550342
:10E0600077349EEFFFFFFFFFFFFFFFFFFFFFFFFF84
:10E07000FFFFFFFFFFFFFFFFFFFFFFFFFFFFD85482
:10E080001303740374037403740374037403740339
:10E090007403740374037403740374031303386503
:10E0A000FFFFFFFFFFFFFFFFFFFFFFFFFFFFB6B513
:10E0B000D39CFFFFFFFFFFFFFFFFFFFFFFFFFFFFFF
:10E0C000FFFFFFFFFFFFFFFFFFFF9EE7B7031C8E71
:10E0D000FFFFFFFFFFFFFFFFFFFFFFFFFFFFFFFF50
:10E0E000FFFFFFFF3A4D5814FFFFFFFFFFFFFFFF49
:10E0F000FFFFFFFFFFFFFFFF75B58A52BAD6DFFFB4
:10E10000FBDEAA5A79CEFFFFFFFFFFFFFFFFFFFFF5
:10E11000FFFF9EE77904590479047904790419040E
:10E120009D9EFFFFFFFF5C8E19047904790479043A
:10E1300079045904590459045904590459045904D7
:10E14000F8031C7EFFFFFFFFFFFFFFFFFFFFFFFF46
:10E15000FFFFFFFFFFFFFFFFFFFFFFFF5C96B7031F
:10E16000F803F803F803F803F803D70397033A55C5
:10E17000DFF7FFFFFFFFFFFFFFFFDDBE5724760342
:10E18000B603D603B6035503B844BFF7FFFFFFFF3E
:10E19000FFFFFFFFFFFFFFFFFFFFFFFFFFFFFFFF8F
:10E1A000FFFFFFFFFFFF3B9E130354037403740341
:10E1B00074037403740374037403740374037403A7
:10E1C00074037403740313033B9EFFFFFFFFFFFF01
:10E1D000FFFFFFFFFFFFFFFF508C9294FFFFFFFF49
:10E1E000FFFFFFFFFFFFFFFFFFFFFFFFFFFFFFFF3F
:10E1F000FFFFFFFF1EC77703BDAEFFFFFFFFFFFF5F
:10E20000FFFFFFFFFFFFFFFFFFFFFFFFFFFFFB7DA4
:10E21000D703BFEFFFFFFFFFFFFFFFFFFFFFFFFF82
:10E22000FFFF4D6BFBDEFFFFFFFFFFFFD6BD308C16
:10E23000FFFFFFFFFFFFFFFFFFFFFFFFFFFFFA34BE
:10E2400039045904590439049914DFF7FFFFFFFF1B
:10E25000BB5D19045904590459045904590459045B
:10E2600059045904590459043904790CBFEFFFFFCC
:10E27000FFFFFFFFFFFFFFFFFFFFFFFFFFFFFFFFAE
:10E28000FFFFFFFFFFFFB92CD703F803F803F803E4
:10E29000F803B703D7031B8EFFFFFFFFFFFFFFFF4E
:10E2A0009EE77A6596039603D603D603B603550315
:10E2B000395DFFFFFFFFFFFFFFFFFFFFFFFFFFFFD6
:10E2C000FFFFFFFFFFFFFFFFFFFFFFFFFFFF1DCF70
:10E2D00054035403740374037403740374037403C6
:10E2E0007403740374037403740374037403540396
:10E2F00054033DD7FFFFFFFFFFFFFFFFFFFFFFFFBF
:10E30000FFFF6D73284AAA5A4D6B7194D6BD9EF7D4
:10E31000FFFFFFFFFFFFFFFFFFFFFFFFFFFF7C9EF1
:10E3200097035ED7FFFFFFFFFFFFFFFFFFFFFFFF2A
:10E33000FFFFFFFFFFFFFFFFBDAE77031EC7FFFF1D
:10E34000FFFFFFFFFFFFFFFFFFFFFFFF8D73DBDE20
:10E35000FFFFFFFFFFFFF3A4718CFFFFFFFFFFFF35
:10E36000FFFFFFFFFFFFFFFFFB75F8035904590490
:10E370001804BB65FFFFFFFFFFFF3A45190459046E
:10E3800059045904590459045904590439043904E5
:10E390003904F803DB75FFFFFFFFFFFFFFFFFFFFFF
:10E3A000FFFFFFFFFFFFFFFFFFFFFFFFFFFFFDC6B8
:10E3B000D703F803F803F803D7039703B9341DCF45
:10E3C000FFFFFFFFFFFFBFEFFB8517147603B603C8
:10E3D000D603D60396037503DB85FFFFFFFFFFFF20
:10E3E000FFFFFFFFFFFFFFFFFFFFFFFFFFFFFFFF3D
:10E3F000FFFFFFFFFFFF9EEFF52314037403740379
:10E400007403740374037403740374037403740354
:10E41000740374037403740334031624FFFFFFFFB3
:10E42000FFFFFFFFFFFFFFFFFFFF9EF7CB5ABEF787
:10E430001CE7D7BD718C0C639AD6FFFFFFFFFFFF6F
:10E44000FFFFFFFFFFFFFFFF9B6DF803DFF7FFFFFD
:10E45000FFFFFFFFFFFFFFFFFFFFFFFFFFFFFFFFCC
:10E46000FFFF5EDF97035C96FFFFFFFFFFFFFFFFED
:10E47000FFFFFFFFFFFFD6BDAA5A79CEFBDED39C7C
:10E48000284A3CE7FFFFFFFFFFFFFFFFFFFFFFFF03
:10E49000FFFFFDBEF80339043904F803BDAEFFFFEA
:10E4A000FFFFFFFF1A3D1804390439043904390409
:10E4B000390439043904390439041904380C9EE745
:10E4C000FFFFFFFFFFFFFFFFFFFFFFFFFFFFFFFF5C
:10E4D000FFFFFFFFFFFFFFFF5A5DB703F803F703DE
:10E4E0009703F70BFB85FFFFFFFFFFFF7EDFDB7D61
:10E4F000371C7603B603D603D603D6037503F61B83
:10E50000BCB6FFFFFFFFFFFFFFFFFFFFFFFFFFFFA7
:10E51000FFFFFFFFFFFFFFFFFFFFFFFFFFFFFFFF0B
:10E52000773C130374037403740374037403740358
:10E530007403740374037403740374037403740323
:10E5400074031303596DFFFFFFFFFFFFFFFFFFFF82
:10E55000FFFFFFFF9EF796B5FFFFFFFFFFFFFFFFE7
:10E56000FFFFFFFFFFFFFFFFFFFFFFFFFFFFFFFFBB
:10E57000FFFFD934992CFFFFFFFFFFFFFFFFFFFFD5
:10E58000FFFFFFFFFFFFFFFFFFFFFFFFFFFF180C75
:10E590005A5DFFFFFFFFFFFFFFFFFFFFFFFFFFFFD2
:10E5A000FFFF75B5CA5AAA5ACF7B9DF7BEF7BEF7D3
:10E5B000FFFFFFFFFFFFFFFFFFFFFFFFDFF79914E4
:10E5C00018041804590C9EE7FFFFFFFFFFFF3A45B0
:10E5D000F803390439043904390439043904380496
:10E5E00018043804D8039B65FFFFFFFFFFFFFFFF00
:10E5F000FFFFFFFFFFFFFFFFFFFFFFFFFFFFFFFF2B
:10E600009EE7180CD703B703F7039A6DBFEFFFFF20
:10E61000DFF7BCAE3955F70B7603B603D703D60345
:10E62000D603B6035503D84C7EE7FFFFFFFFFFFF7D
:10E63000FFFFFFFFFFFFFFFFFFFFFFFFFFFFFFFFEA
:10E64000FFFFFFFFFFFFFFFFF854F30274037403A3
:10E650007403740374037403740374037403740302
:10E660007403740374037403740374031303BCBE50
:10E67000FFFFFFFFFFFFFFFFFFFFFFFFFFFFFBDECF
:10E680005DEFFFFFFFFFFFFFFFFFFFFFFFFFFFFF4C
:10E69000FFFFFFFFFFFFFFFFFFFFDFF7F8037B65D3
:10E6A000FFFFFFFFFFFFFFFFFFFFFFFFFFFFFFFF7A
:10E6B000FFFFFFFFFFFFFFFFF944591CFFFFFFFFB4
:10E6C000FFFFFFFFFFFFFFFFFFFFFFFFFFFFFFFF5A
:10E6D000FFFF59CEAE7B494A9AD6FFFFFFFFFFFFEF
:10E6E000FFFFFFFFFFFFFFFF9B65D803F803B92C77
:10E6F000FFFFFFFFFFFFFFFF9B65D803180418040F
:10E700001804180418041804180418041804180429
:10E710007EDFFFFFFFFFFFFFFFFFFFFFFFFFFFFFAA
:10E72000FFFFFFFFFFFFFFFFFFFF1B869703381C64
:10E730007A65DDBE5ED77C9E3A55371C96039603FC
:10E74000B603D703D603D603D6037503B60B1B8EC9
:10E75000FFFFFFFFFFFFFFFFFFFFFFFFFFFFFFFFC9
:10E76000FFFFFFFFFFFFFFFFFFFFFFFFFFFFFFFFB9
:10E770001865F3027403740374037403740374035D
:10E7800074037403740374037403740374037403D1
:10E79000740374033403D51BDFF7FFFFFFFFFFFF94
:10E7A000FFFFFFFFFFFFFFFF34AD494ACB5A0F8445
:10E7B000B6BD5DEFFFFFFFFFFFFFFFFFFFFFFFFFA6
:10E7C000FFFFFFFF3ECF77037CA6FFFFFFFFFFFFAA
:10E7D000FFFFFFFFFFFFFFFFFFFFFFFFFFFFFFFF49
:10E7E000FFFF1C86B7039EE7FFFFFFFFFFFFFFFF52
:10E7F000FFFFFFFFFFFFFFFFD7BD494A0C6334ADAA
:10E800007DEFFFFFFFFFFFFFFFFFFFFFFFFFFFFFAA
:10E81000FFFFFDC6D803D8033A4DFFFFFFFFFFFF00
:10E82000FFFF9DA6D8031804180418041804180440
:10E83000180418041804B8035A55FFFFFFFFFFFF20
:10E84000FFFFFFFFFFFFFFFFFFFFFFFFFFFFFFFFD8
:10E85000FFFFFFFF7824B703982CF9445824D7030F
:10E8600096039603B703D703D703D703D603D6037C
:10E8700096037503D84C5ED7FFFFFFFFFFFFFFFF36
:10E88000FFFFFFFFFFFFFFFFFFFFFFFFFFFFFFFF98
:10E89000FFFFFFFFFFFFFFFF3865F3025403740320
:10E8A00074037403740374037403740374037403B0
:10E8B0007403740374037403740374037403F30222
:10E8C000596DFFFFFFFFFFFFFFFFFFFFFFFFFFFF90
:10E8D000FFFFFFFFFFFF9AD6D39C4C6B69529AD67D
:10E8E000FFFFFFFFFFFFFFFFFFFFFFFFFFFF3C9664
:10E8F00097037EDFFFFFFFFFFFFFFFFFFFFFFFFF2D
:10E90000FFFFFFFFFFFFFFFFFFFFFFFF1DC77703B5
:10E910009DAEFFFFFFFFFFFFFFFFFFFFFFFFFFFFBA
:10E920005DEF284A9AD6FFFFFFFFFFFFFFFFFFFFC3
:10E93000FFFFFFFFFFFFFFFFFFFFFFFFFFFFB92C00
:10E9400097039B65FFFFFFFFFFFFFFFFBFEF38143B
:10E95000F803180418041804180418041804F80319
:10E96000D7033ECFFFFFFFFFFFFFFFFFFFFFFFFFCC
:10E97000FFFFFFFFFFFFFFFFFFFFFFFFBDB6970396
:10E98000F703D703B703D703D703D703D703D703B7
:10E99000D703D703D603B603550337247CA6FFFF5E
:10E9A000FFFFFFFFFFFFFFFFFFFFFFFFFFFFFFFF77
:10E9B000FFFFFFFFFFFFFFFFFFFFFFFFFFFFFFFF67
:10E9C000F85CF30254037403740374037403740354
:10E9D000740374037403740374037403740374037F
:10E9E000740374037403540334031DCFFFFFFFFF4C
:10E9F000FFFFFFFFFFFFFFFFFFFF7DEF8E7318C6D6
:10EA0000FFFFFFFFFFFFBEF7DFFFFFFFFFFFFFFF7F
:10EA1000FFFFFFFFFFFFFFFF1A4D3814FFFFFFFF4F
:10EA2000FFFFFFFFFFFFFFFFFFFFFFFFFFFFFFFFF6
:10EA3000FFFFFFFFFFFFDFF7F80B5A5DFFFFFFFF50
:10EA4000FFFFFFFFFFFFFFFFFFFFFBDE0C63FFFF8A
:10EA5000FFFFFFFFFFFF18C638C6FFFFFFFFFFFFE6
:10EA6000FFFFFFFFFFFFFFFF5C965603BB6DFFFF3D
:10EA7000FFFFFFFFFFFFFFFF1C869703F803F8036C
:10EA8000F803F803F803F803B7031A45FFFFFFFF85
:10EA9000FFFFFFFFFFFFFFFFFFFFFFFFFFFFFFFF86
:10EAA000FFFFFFFFFFFF194D9603F703F703F7037F
:10EAB000D703D703D703D703D703D603B60375030A
:10EAC000D60BDA7DDFF7FFFFFFFFFFFFFFFFFFFF42
:10EAD000FFFFFFFFFFFFFFFFFFFFFFFFFFFFFFFF46
:10EAE000FFFFFFFFFFFFBFEF9744F30274037403C0
:10EAF000740374037403740374037403740374035E
:10EB0000740374037403740374037403740374034D
:10EB10001303973CFFFFFFFFFFFFFFFFFFFFFFFF18
:10EB2000FFFFFFFF4C6B71947DEF7194284AF3A4B3
:10EB3000FFFFFFFFFFFFFFFFFFFFFFFFFFFFFFFFE5
:10EB4000DFF7F80B7A5DFFFFFFFFFFFFFFFFFFFF1F
:10EB5000FFFFFFFFFFFFFFFFFFFFFFFFFFFFFFFFC5
:10EB6000FFFF1A4D1814FFFFFFFFFFFFFFFFFFFF1E
:10EB7000FFFFFFFFFFFF2C6BF3A479CE518C8A526D
:10EB80008A5218C6FFFFFFFFFFFFFFFFFFFFFFFFD7
:10EB9000FFFFBFF7F8037A5DFFFFFFFFFFFFFFFFF7
:10EBA000FFFFFFFFB934B703F803F803F803F803D6
:10EBB000F803B703FDBEFFFFFFFFFFFFFFFFFFFFEF
:10EBC000FFFFFFFFFFFFFFFFFFFFFFFFFFFF7EDFF6
:10EBD000D703D703F703D703D703D703D703D70345
:10EBE000D703B6037603D60B7A6D7EE7FFFFFFFFF0
:10EBF000FFFFFFFFFFFFFFFFFFFFFFFFFFFFFFFF25
:10EC0000FFFFFFFFFFFFFFFFFFFFFFFFFFFF5EDFD5
:10EC1000162C1303740374037403740374037403D2
:10EC2000740374037403740374037403740374032C
:10EC30007403740374037403740313039CB6FFFF1B
:10EC4000FFFFFFFFFFFFFFFFFFFFFFFF79CE8D7389
:10EC5000FFFF14A58A52FBDECB5ADBDEFFFFFFFF6E
:10EC6000FFFFFFFFFFFFFFFFFFFFFDBE7703BDAE0E
:10EC7000FFFFFFFFFFFFFFFFFFFFFFFFFFFFFFFFA4
:10EC8000FFFFFFFFFFFFFFFFFFFFFFFF7CA67703F4
:10EC90001ECFFFFFFFFFFFFFFFFFFFFFFFFFFFFF95
:10ECA0005DEF4C6BCB5A518CBAD6FFFFD7BDDADE85
:10ECB000FFFFFFFFFFFFFFFFFFFFFFFFFFFFBB6D3A
:10ECC000F93CFFFFFFFFFFFFFFFFFFFFFFFF7EDFBE
:10ECD0003814B703F803F803F803B703D934FFFF78
:10ECE000FFFFFFFFFFFFFFFFFFFFFFFFFFFFFFFF34
:10ECF000FFFFFFFFFFFFFFFFDB7D9603D703D70377
:10ED0000D703D703D703D60396037503F60B7A6DA3
:10ED10005EDFFFFFFFFFFFFFFFFFFFFFFFFFFFFFC4
:10ED2000FFFFFFFFFFFFFFFFFFFFFFFFFFFFFFFFF3
:10ED3000FFFFFFFFFFFF9CB69513140374037403DA
:10ED4000740374037403740374037403740374030B
:10ED500074037403740374037403740374037403FB
:10ED600074031403362CFFFFFFFFFFFFFFFFFFFFBD
:10ED7000FFFFFFFFFFFFDBDECB5A14A507429EF724
:10ED8000FFFF2C6BDBDEFFFFFFFFFFFFFFFFFFFF3F
:10ED9000FFFFFFFFBB6DB703BFEFFFFFFFFFFFFFED
:10EDA000FFFFFFFFFFFFFFFFFFFFFFFFFFFFFFFF73
:10EDB000FFFFFFFFFFFF9FEFB703BB75FFFFFFFFE5
:10EDC000FFFFFFFFFFFFFFFFFFFFFFFFFFFFFFFF53
:10EDD000FFFFFFFFFFFFD6BDEF7BFFFFFFFFFFFF42
:10EDE000FFFFFFFFFFFFFFFF9EE7F944FFFFFFFF6D
:10EDF000FFFFFFFFFFFFFFFFFFFF3ECF381C970322
:10EE0000F703F703B7039CAEFFFFFFFFFFFFFFFF12
:10EE1000FFFFFFFFFFFFFFFFFFFFFFFFFFFFFFFF02
:10EE2000FFFF371CB603D703D703D703B603760318
:10EE300076033724DB859EE7FFFFFFFFFFFFFFFF21
:10EE4000FFFFFFFFFFFFFFFFFFFFFFFFFFFFFFFFD2
:10EE5000FFFFFFFFFFFFFFFFFFFFFFFFFFFF997DAA
:10EE6000340334037403740374037403740374036A
:10EE700074037403740374037403740374037403DA
:10EE800074037403740374037403740313039CAE58
:10EE9000FFFFFFFFFFFFFFFFFFFFFFFFFFFFFFFF82
:10EEA000FFFFB6B52C63DBDE3CE7718C4D6BFFFFDB
:10EEB000FFFFFFFFFFFFFFFFFFFFFFFFFFFF381414
:10EEC000FA44FFFFFFFFFFFFFFFFFFFFFFFFFFFF12
:10EED000FFFFFFFFFFFFFFFFFFFFFFFFFFFFFFFF42
:10EEE000FFFFF93C381CFFFFFFFFFFFFFFFFFFFFA5
:10EEF000FFFFFFFFFFFFFFFFFFFFFFFFFFFFDFFF42
:10EF000013A524295DEFFFFFFFFFFFFFFFFFFFFFBA
:10EF1000FFFFFFFF5C9E5ED7FFFFFFFFFFFFFFFFCE
:10EF2000FFFFFFFFFFFF9EE7F94497039703581C7D
:10EF3000DFF7FFFFFFFFFFFFFFFFFFFFFFFFFFFF09
:10EF4000FFFFFFFFFFFF9EEF7CA6B83CB603D70391
:10EF5000B60376037603D60B19559CAEDFFFFFFF91
:10EF6000FFFFFFFFFFFFFFFFFFFFFFFFFFFFFFFFB1
:10EF7000FFFFFFFFFFFFFFFFFFFFFFFFFFFFFFFFA1
:10EF8000FFFFFFFF3DD7773C130354037403740363
:10EF900074037403740374037403740374037403B9
:10EFA00074037403740374037403740374037403A9
:10EFB000740374031303773CFFFFFFFFFFFFFFFFA2
:10EFC000FFFFFFFFFFFFFFFFBEF7D7BDFFFFFFFF04
:10EFD000FFFF10844C6B9DF7FFFFFFFFFFFFFFFF5C
:10EFE000FFFFFFFFFFFF1DC777037CA6FFFFFFFFAB
:10EFF000FFFFFFFFFFFFFFFFFFFFFFFFFFFFFFFF21
:10F00000FFFFFFFFFFFFFFFFFFFFFFFF7CA6570390
:10F010001DC7FFFFFFFFFFFFFFFFFFFFFFFFFFFF1A
:10F02000FFFFFFFF7DEF7194494AAE7B108410848F
:10F03000FFFFFFFFFFFFFFFFFFFFFFFFFFFFBFF728
:10F040007EDFFFFFFFFFFFFFFFFFFFFFFFFFFFFF71
:10F05000FFFFFFFF7CA6782C960337145A655C9E51
:10F06000FDC65ED75EDF5ED7FDC69CA6DB7DF9449C
:10F07000F70B56035503760396031714F94C5C9E61
:10F080009EE7FFFFFFFFFFFFFFFFFFFFFFFFFFFF09
:10F09000FFFFFFFFFFFFFFFFFFFFFFFFFFFFFFFF80
:10F0A000FFFFFFFFFFFFFFFFFFFFFFFFFA8D750B65
:10F0B00014037403740374037403740374037403F8
:10F0C0007403740374037403740374037403740388
:10F0D00074037403740374037403740354033403D8
:10F0E000FDC6FFFFFFFFFFFFFFFFFFFFFFFFFFFF6B
:10F0F000DFFF2C6B8A52CA5ADFFFFFFFFFFFFFFFC3
:10F10000FFFFFFFFFFFFFFFFFFFFFFFFFFFFFFFF0F
:10F110009B65B703BFEFFFFFFFFFFFFFFFFFFFFF91
:10F12000FFFFFFFFFFFFFFFFFFFFFFFFFFFFFFFFEF
:10F13000FFFFFFFFFFFFBFF7D8035A5DFFFFFFFF91
:10F14000FFFFFFFFFFFFFFFFFFFFFFFF96B5084236
:10F15000CF7BFBDEFFFFDFFF508CFFFFFFFFFFFFDA
:10F16000FFFFFFFFFFFFFFFFFFFFFFFFFFFFFFFFAF
:10F17000FFFFFFFFFFFFFFFFFFFFFFFFFFFFFFFF9F
:10F18000FFFFBDB63A551714960376037603960330
:10F1900076035503350335035603D6035724F94C3C
:10F1A000DB7DDDBEBFEFFFFFFFFFFFFFFFFFFFFFC8
:10F1B000FFFF3CE79ACE518C718CFFFFFFFFFFFFF2
:10F1C000FFFFFFFFFFFFFFFFFFFFFFFFFFFFFFFF4F
:10F1D000FFFFFDC6773C14035403740374037403E8
:10F1E0007403740374037403740374037403740367
:10F1F0007403740374037403740374037403740357
:10F20000740374037403F3023865FFFFFFFFFFFF0D
:10F21000FFFFFFFFFFFFFFFFFFFF55AD0F84FFFF65
:10F220008E73B29CB294AE7BFBDEFFFFFFFFFFFF4D
:10F23000FFFFFFFFFFFFFFFFDFF7F80B3A55FFFF70
:10F24000FFFFFFFFFFFFFFFFFFFFFFFFFFFFFFFFCE
:10F25000FFFFFFFFFFFFFFFFFFFFFFFFFFFFFFFFBE
:10F26000FFFF7A5DD703BFEFFFFFFFFFFFFFFFFF49
:10F27000FFFFFFFFFFFFFBDE3CE7FFFFFFFFFFFF9E
:10F28000FFFFDBDE75ADFFFFFFFFFFFFFFFFFFFFAF
:10F29000FFFFFFFFFFFFFFFFFFFFFFFFFFFFFFFF7E
:10F2A000FFFFFFFFFFFFFFFFFFFFFFFFFFFFFFFF6E
:10F2B000FFFF7EDFDDBE7C9E1B8EFB851B8E5C9E72
:10F2C0009CAEFDC67EE7DFFFFFFFFFFFFFFFFFFFF6
:10F2D000FFFFDFFF5DEFBEF7FFFF9294CF7BDFFF05
:10F2E00096B5694AFFFFFFFFFFFFFFFFFFFFFFFF2C
:10F2F000FFFFFFFFFFFFFFFF7EE738655403340386
:10F300007403740374037403740374037403740345
:10F310007403740374037403740374037403740335
:10F320007403740374037403740374037403340365
:10F33000D51BBFF7FFFFFFFFFFFFFFFFFFFFFFFF33
:10F34000FFFF9EF70B63DFFFFFFF494A2C6310842A
:10F3500014A5BEF7FFFFFFFFFFFFFFFFFFFFFFFF4B
:10F36000FFFF9CA65703FDBEFFFFFFFFFFFFFFFF50
:10F37000FFFFFFFFFFFFFFFFFFFFFFFFFFFFFFFF9D
:10F38000FFFFFFFFFFFFFFFFFFFFFFFF3ECF570322
:10F390003C96FFFFFFFFFFFFFFFFFFFFFFFFFFFFA9
:10F3A000FFFFFFFFFFFFFFFFDFFF9294084234AD36
:10F3B000FFFFFFFFFFFFFFFFFFFFFFFFFFFFFFFF5D
:10F3C000FFFFFFFFFFFFFFFFFFFFFFFFFFFFFFFF4D
:10F3D000FFFFFFFFFFFFFFFFFFFFFFFFFFFFFFFF3D
:10F3E000FFFFFFFFFFFFFFFFFFFFFFFFFFFFFFFF2D
:10F3F000FFFFFFFFFFFFDFFF79CE18C618BE7ACEF2
:10F40000DFFFFFFF75ADCB5A96B555ADAA52F7BDDC
:10F41000FFFFFFFFFFFFFFFFFFFFFFFFFFFF9EEF6D
:10F42000997D950B140374037403740374037403BC
:10F430007403740374037403740374037403740314
:10F440007403740374037403740374037403740304
:10F4500074037403740354031303BCB6FFFFFFFF6C
:10F46000FFFFFFFFFFFFFFFFFFFFFFFF3CE707423C
:10F47000718C518CD39CFFFFFFFFFFFFFFFFFFFF4D
:10F48000FFFFFFFFFFFFFFFFFFFFFFFFB934581C27
:10F49000FFFFFFFFFFFFFFFFFFFFFFFFFFFFFFFF7C
:10F4A000FFFFFFFFFFFFFFFFFFFFFFFFFFFFFFFF6C
:10F4B000FFFFFFFFFFFFFFFF992C581CFFFFFFFF1F
:10F4C000FFFFFFFFFFFFFFFFFFFFFFFFFFFFFFFF4C
:10F4D00075B5494A24295DEFFFFFFFFFFFFFFFFFDE
:10F4E000FFFFFFFFFFFFFFFFFFFFFFFFFFFFFFFF2C
:10F4F000FFFFFFFFFFFFFFFFFFFFFFFFFFFFFFFF1C
:10F50000FFFFFFFFFFFFFFFFFFFFFFFFFFFFBEF754
:10F51000FFFFFFFFBEF759CE59CE96B5D39CFFFF34
:10F52000BEF7663155ADBEF71CE77DEFFFFFFFFF6D
:10F53000AA52D7BDFFFFEF7B2C63FFFFFFFFFFFF4A
:10F54000FFFFFFFF9EEF9A7DB5131403540374036E
:10F5500074037403740374037403740374037403F3
:10F5600074037403740374037403740374037403E3
:10F5700074037403740374037403740374037403D3
:10F58000F302596DFFFFFFFFFFFFFFFFFFFFFFFFCC
:10F59000FFFFFFFF9EF7FBDE7DF7719465316D7312
:10F5A000DBDEFFFFFFFFFFFFFFFFFFFFFFFFFFFFB0
:10F5B000FFFFFFFF3ECF57033C8EFFFFFFFFFFFF24
:10F5C000FFFFFFFFFFFFFFFFFFFFFFFFFFFFFFFF4B
:10F5D000FFFFFFFFFFFFFFFFFFFFFFFFFFFFFFFF3B
:10F5E000FFFF9DAE5703BDB6FFFFFFFFFFFFFFFF0D
:10F5F000FFFFFFFFFFFFFFFFD29C6952BAD6B29C0C
:10F60000B294FFFFFFFF3CE7FFFFFFFFFFFFFFFF9D
:10F61000FFFFFFFFFFFFFFFFFFFFFFFFFFFFFFFFFA
:10F62000FFFFFFFFFFFFFFFFFFFFFFFFFFFFFFFFEA
:10F63000FFFFFFFFBFF7CF7B8A52DFF7FFFF34A545
:10F64000694ABEF71CE78629FBDEFFFFAE73518CCB
:10F650009ACED39C694ABEF7FFFF4D6B8E6B59CE95
:10F6600096B5BAD6FFFFFFFFFFFF9EE79A7DB51361
:10F670001403540375037403740374037403740351
:10F6800074037403740374037403740374037403C2
:10F6900074037403740374037403740374037403B2
:10F6A00074037403740374031303563CFFFFFFFFDA
:10F6B000FFFFFFFFFFFFFFFFFFFFFFFFFFFFCF7B0E
:10F6C00014A5FFFFFFFFDFFFB29C284A38C6FFFFEB
:10F6D000FFFFFFFFFFFFFFFFFFFFFFFFFFFF3A55A9
:10F6E000D703BFEFFFFFFFFFFFFFFFFFFFFFFFFF9E
:10F6F000FFFFFFFFFFFFFFFFFFFFFFFFFFFFFFFF1A
:10F70000FFFFFFFFFFFFFFFFFFFFFFFFFFFF381CB3
:10F71000B934FFFFFFFFFFFFFFFFFFFFFFFFFFFF0A
:10F72000FFFF7DEFFFFFFFFFDFFF4D6B96B5CA5A6E
:10F730009294FFFFFFFFFFFFFFFFFFFFFFFFFFFFB1
:10F74000FFFFFFFFFFFFFFFFFFFFFFFFFFFFFFFFC9
:10F75000FFFFFFFFFFFFFFFFFFFFFFFFFFFFFFFFB9
:10F7600075ADE739DFFFFFFFD7BDE739FBDEBAD65E
:10F77000C73918C6FFFFFFFFFFFFFFFF3CE7652902
:10F78000DBDEFFFF9EF779CE7DEFFFFFFFFFFFFF80
:10F790003DD7596DB51314035403750374037403F3
:10F7A00074037403740374037403740374037403A1
:10F7B0007403740374037403740374037403740391
:10F7C0007403740374037403740374037403740381
:10F7D0003403B51B7EE7FFFFFFFFFFFFFFFFFFFFC7
:10F7E000FFFFFFFFFFFF79CECB5AFFFF38CE14A5F6
:10F7F000FFFFFFFFDFFF9EF7FFFFFFFFFFFFFFFFA2
:10F80000FFFFFFFFFFFF7EDF7703BB75FFFFFFFFFB
:10F81000FFFFFFFFFFFFFFFFFFFFFFFFFFFFFFFFF8
:10F82000FFFFFFFFFFFFFFFFFFFFFFFFFFFFFFFFE8
:10F83000FFFFFFFFFFFFFFFF5C9E5703FDBEFFFFC3
:10F84000FFFFFFFFFFFFFFFFFFFFFFFFFFFFFFFFC8
:10F85000FFFF9EF7CA5A8631F7BDD7BDB6BDFFFF81
:10F86000FFFFFFFFFFFFFFFFFFFFFFFFFFFFFFFFA8
:10F870009EE7FFFFFFFFFFFFFFFFFFFFFFFFFFFF11
:10F88000FFFFFFFFFFFFFFFFFFFF38C60842DFFF5C
:10F89000FFFFDFFF59C6BBD65DEF694AD39CFFFF70
:10F8A000FFFF9AD618C6F7BD18C6DFFFFFFFFFFFA0
:10F8B000FFFFFFFFDFF77CAEB74C75031403540363
:10F8C000750375037403740374037403740374037E
:10F8D0007403740374037403740374037403740370
:10F8E0007403740374037403740374037403740360
:10F8F000740374037403740334035403FDC6FFFFDD
:10F90000FFFFFFFFFFFFFFFFFFFFFFFFFFFFBEF750
:10F910008952FBDEFFFFAA5A59CEFFFFF3A47DEF09
:10F92000FFFFFFFFFFFFFFFFFFFFFFFFFFFFFFFFE7
:10F930007A5DB7039EE7FFFFFFFFFFFFFFFFFFFFBB
:10F94000FFFFFFFFFFFFFFFFFFFFFFFFFFFFFFFFC7
:10F95000FFFFFFFFFFFFFFFFFFFFFFFFFFFFFFFFB7
:10F96000FFFFFFFF381CB934FFFFFFFFFFFFFFFF62
:10F97000FFFFFFFFFFFFFFFFFFFF96B5E741718C21
:10F98000FFFF7DEF0842BAD6FFFFFFFFFFFFFFFF3B
:10F99000FFFFFFFFFFFFFFFFFFFF7EDFFA853ED780
:10F9A000FFFFFFFFFFFFFFFFFFFFFFFFFFFFFFFF67
:10F9B000FFFFFFFFF7C5A631DFFFFFFFFFFF5DEF92
:10F9C0009AD679CE308459CEFFFFDFFF1CE79EF731
:10F9D000FFFFFFFFFFFFFFFFDFFFDDBE596DF61BDF
:10F9E00034033403750375037503740374037403DC
:10F9F000740374037403740374037403740374034F
:10FA0000740374037403740374037403740374033E
:10FA1000740374037403740374037403740374032E
:10FA2000340334039CB6FFFFFFFFFFFFFFFFFFFF20
:10FA3000FFFFFFFFFFFFDFFF5DEFAA520F84518C36
:10FA4000D39CFFFFF7C5CB5ABEFFFFFFFFFFFFFFB1
:10FA5000FFFFFFFFFFFFFFFF7EDF7703BB6DFFFFB1
:10FA6000FFFFFFFFFFFFFFFFFFFFFFFFFFFFFFFFA6
:10FA7000FFFFFFFFFFFFFFFFFFFFFFFFFFFFFFFF96
:10FA8000FFFFFFFFFFFFFFFFFFFFFFFFFFFF7C9E6A
:10FA90003703BDB6FFFFFFFFFFFFFFFFFFFFFFFFC5
:10FAA000FFFFFFFFF7C5BAD6FFFFFFFFAA5A38CE08
:10FAB000FFFF5DEF9EF7FFFFFFFFFFFFFFFFFFFF71
:10FAC000FFFFFFFFFFFF1DCF572C596D5EDFFFFFCC
:10FAD000FFFFFFFFFFFFFFFFFFFFFFFFFFFF3CE711
:10FAE000B6B5DFFFFFFFFFFF1CE71CE77DEFFFFF61
:10FAF000FFFFFFFFFFFFFFFFFFFFFFFF9EEF9CAE3B
:10FB0000596D1624540314035403750375037503C8
:10FB1000740374037403740374037403740374032D
:10FB2000740374037403740374037403740374031D
:10FB3000740374037403740374037403740374030D
:10FB40007403740374037403340334037BA6FFFF4C
:10FB5000FFFFFFFFFFFFFFFFFFFFFFFFFFFFFFFFB5
:10FB60003CE76D73FFFF9294E320F39CBEF7AA5A23
:10FB7000DBDEFFFFFFFFFFFFFFFFFFFFFFFFFFFFDA
:10FB8000FFFF3A55B7039FEFFFFFFFFFFFFFFFFFA8
:10FB9000FFFFFFFFFFFFFFFFFFFFFFFFFFFFFFFF75
:10FBA000FFFFFFFFFFFFFFFFFFFFFFFFFFFFFFFF65
:10FBB000FFFFFFFFFFFFFFFFFFFF78245824FFFF39
:10FBC000FFFFFFFFFFFFFFFFFFFFFFFFFFFFFFFF45
:10FBD000FFFFFFFF7194F3A4BAD6308CC7391084AD
:10FBE000FFFFFFFFFFFFFFFFFFFFFFFFFFFFFFFF25
:10FBF000FFFF5EDFD6135503D84C3B963ED7FFFF81
:10FC0000FFFFFFFFFFFFFFFFFFFFFFFFFFFFFFFF04
:10FC1000FFFFFFFFFFFFFFFFFFFFFFFFDFF75EDFDD
:10FC20009CAE9A75973CB50B3403340354037503AB
:10FC30007503750375037403740374037403740309
:10FC400074037403740374037403740374037403FC
:10FC500074037403740374037403740374037403EC
:10FC600074037403740374037403740374037403DC
:10FC7000340334035BA6FFFFFFFFFFFFFFFFFFFF1F
:10FC8000FFFFFFFFFFFFFFFFFFFFFFFF8D7334A5A7
:10FC9000FFFF3CE74D6B8531B29CFFFFFFFFFFFF8D
:10FCA000FFFFFFFFFFFFFFFFFFFF1ECF5703FB7D9F
:10FCB000FFFFFFFFFFFFFFFFFFFFFFFFFFFFFFFF54
:10FCC000FFFFFFFFFFFFFFFFFFFFFFFFFFFFFFFF44
:10FCD000FFFFFFFFFFFFFFFFFFFFFFFFFFFFFFFF34
:10FCE000FFFFFFFFDDB636033C8EFFFFFFFFFFFF88
:10FCF000FFFFFFFFFFFFFFFFFFFFFFFF96B585310F
:10FD0000AE7BAE73B6BDAA5ABAD6FFFFFFFFFFFFA8
:10FD1000FFFFFFFFFFFFFFFFFFFFFFFFFFFF9EE76C
:10FD20005734F402550395033724D84C7A751B9643
:10FD30007CAEBCBEFDC6FDC6FDC6BCBE7CAE3B9661
:10FD4000BA7D395D973C161C9503340334033403A4
:10FD500075037503750375037503750374037403E5
:10FD600074037403740374037403740374037403DB
:10FD700074037403740374037403740374037403CB
:10FD800074037403740374037403740374037403BB
:10FD900074037403740374031403540B9CB6FFFFC1
:10FDA000FFFFFFFFFFFFFFFFFFFFFFFFFFFFFFFF63
:10FDB000FFFFFFFFFFFF5DEF89529EF7FFFFFFFF91
:10FDC00038C6BEF7FFFFFFFFFFFFFFFFFFFFFFFF8C
:10FDD000FFFFFFFF99341814DFF7FFFFFFFFFFFF5E
:10FDE000FFFFFFFFFFFFFFFFFFFFFFFFFFFFFFFF23
:10FDF000FFFFFFFFFFFFFFFFFFFFFFFFFFFFFFFF13
:10FE0000FFFFFFFFFFFFFFFFFFFFFFFFFFFFFFFF02
:10FE10001A45B7039EE7FFFFFFFFFFFFFFFFFFFF4E
:10FE2000FFFFFFFFFFFF55AD1084DBDEFFFFEF8319
:10FE300075B5FFFF38C617C6FFFFFFFFFFFFFFFFC7
:10FE4000FFFFFFFFFFFFFFFFFFFFDFF7D84C34038B
:10FE500075037503550334033403550355037503C4
:10FE60007503550355033403340334033403540337
:10FE700055037503750375037503750375037503E2
:10FE800075037403740374037403740374037403B9
:10FE900074037403740374037403740374037403AA
:10FEA000740374037403740374037403740374039A
:10FEB000740374037403740374037403740374038A
:10FEC0001303D51BFDC6FFFFFFFFFFFFFFFFFFFF73
:10FED000FFFFFFFFFFFFFFFFFFFF718C34AD9EF7B9
:10FEE000FFFF14A5518CFFFFFFFFFFFFFFFFFFFF88
:10FEF000FFFFFFFFFFFFFFFFFFFFFFFF7C9E3603BB
:10FF00009CA6FFFFFFFFFFFFFFFFFFFFFFFFFFFFBD
:10FF1000FFFFFFFFFFFFFFFFFFFFFFFFFFFFFFFFF1
:10FF2000FFFFFFFFFFFFFFFFFFFFFFFFFFFFFFFFE1
:10FF3000FFFFFFFFFFFFFFFFFFFF7EDF97033A5545
:10FF4000FFFFFFFFFFFFFFFFFFFFFFFFFFFFFFFFC1
:10FF5000FFFFFFFFFFFF96B5AE7B59CE4D6BAA5A50
:10FF600018C67DEFFFFFFFFFFFFFFFFFFFFFFFFF53
:10FF7000FFFFFFFFFFFFFFFF9A7555037503950312
:10FF800095039503950395039503950395039503B1
:10FF900095039503950395039503950375037503E1
:10FFA0007503750375037503740374037403740395
:10FFB0007403740374037403740374037403740389
:10FFC0007403740374037403740374037403740379
:10FFD0007403740374037403740374037403740369
:10FFE0007403740374035403F302763C7EE7FFFF4B
:10FFF000FFFFFFFFFFFFFFFFFFFFFFFFFFFFFFFF11
:020000040801F1
:10000000BEFFFFFFD7BD6D73AA5ACF7B17C6EB5A51
:10001000DBDEFFFFFFFFFFFFFFFFFFFFFFFFFFFF35
:10002000FFFFFFFFBFEFD80BD93CFFFFFFFFFFFF34
:10003000FFFFFFFFFFFFFFFFFFFFFFFFFFFFFFFFD0
:10004000FFFFFFFFFFFFFFFFFFFFFFFFFFFFFFFFC0
:10005000FFFFFFFFFFFFFFFFFFFFFFFFFFFFFFFFB0
:10006000FFFFFFFFFFFF1C863603BDAEFFFFFFFF54
:10007000FFFFFFFFFFFFFFFFFFFFFFFFFFFFDBDED5
:1000800044292C6BCE7B18C6FFFF96B54529D7BDFA
:10009000FFFFFFFFFFFFFFFFFFFFFFFFFFFFFFFF70
:1000A000FFFFFFFF9CAEB613340395039503950342
:1000B00095039503950395039503950375037503C0
:1000C0007503750375037503750375037503740371
:1000D0007403740374037403740374037403740368
:1000E0007403740374037403740374037403740358
:1000F0007403740374037403740374037403740348
:100100007403740374037403740374037403340377
:1001100034037975FFFFFFFFFFFFFFFFFFFFFFFFC6
:10012000FFFFFFFFFFFFFFFFFFFFF7C5CA5AFFFFFB
:10013000FFFF9EF796B51084484A96B5FFFFFFFF74
:10014000FFFFFFFFFFFFFFFFFFFFFFFFFFFF3A552E
:1001500097035EDFFFFFFFFFFFFFFFFFFFFFFFFFD4
:10016000FFFFFFFFFFFFFFFFFFFFFFFFFFFFFFFF9F
:10017000FFFFFFFFFFFFFFFFFFFFFFFFFFFFFFFF8F
:10018000FFFFFFFFFFFFFFFFFFFFFFFFFFFFFFFF7F
:10019000FFFF992CF80BBFEFFFFFFFFFFFFFFFFFF3
:1001A000FFFFFFFFFFFFFFFFFBDEB2941CE7FFFF37
:1001B000FFFFB29CAA5A79CEAA52F7BDFFFFFFFFFC
:1001C000FFFFFFFFFFFFFFFFFFFFFFFFFFFFFFFF3F
:1001D0007EE7D84C340355039503950395037503C7
:1001E000750375037503750375037503750375034F
:1001F0007503740374037403740374037403740346
:100200007403740374037403740374037403740336
:100210007403740374037403740374037403740326
:100220007403740374037403740374037403740316
:10023000740374035403F302D523BCB6FFFFFFFF1E
:10024000FFFFFFFFFFFFFFFFFFFFFFFFFFFFFFFFBE
:100250009EF7DBDEFFFF718C484A7DEFFFFFFFFF5B
:10026000FFFFDFFFFFFFFFFFFFFFFFFFFFFFFFFFBE
:10027000FFFFFFFFFFFF9DAE36031C86FFFFFFFF62
:10028000FFFFFFFFFFFFFFFFFFFFFFFFFFFFFFFF7E
:10029000FFFFFFFFFFFFFFFFFFFFFFFFFFFFFFFF6E
:1002A000FFFFFFFFFFFFFFFFFFFFFFFFFFFFFFFF5E
:1002B000FFFFFFFFFFFFFFFFFFFFFFFF5ED777039B
:1002C0001A4DFFFFFFFFFFFFFFFFFFFFFFFFFFFFD5
:1002D000FFFFFFFFFFFFFFFFFFFFB2944529AE7B4B
:1002E000FFFF3CE7694A79CEFFFFFFFFFFFFFFFFFB
:1002F000FFFFFFFFFFFFFFFFFFFFFFFFFFFF3B9E33
:10030000D51B140375037503750375037503750316
:100310007503750375037403740374037403740322
:100320007403740374037403740374037403740315
:100330007403740374037403740374037403740305
:1003400074037403740374037403740374037403F5
:1003500074037403740374037403540313033403A6
:10036000596DBFF7FFFFFFFFFFFFFFFFFFFFFFFF1D
:10037000FFFFFFFFFFFFFFFFFFFF7DEF494A18C6AA
:10038000FFFFF39C07421CE7FFFFFFFFFFFFFFFF9C
:10039000FFFFFFFFFFFFFFFFFFFFFFFFFFFF9EE7E6
:1003A000D70BB934FFFFFFFFFFFFFFFFFFFFFFFF8A
:1003B000FFFFFFFFFFFFFFFFFFFFFFFFFFFFFFFF4D
:1003C000FFFFFFFFFFFFFFFFFFFFFFFFFFFFFFFF3D
:1003D000FFFFFFFFFFFFFFFFFFFFFFFFFFFFFFFF2D
:1003E000FFFFFFFFFFFFFFFF3C8E36035C96FFFF22
:1003F000FFFFFFFFFFFFFFFFFFFFFFFFFFFFFFFF0D
:10040000FFFF308CAA5ADFFF71946D73FFFF3CE74A
:100410005DEFFFFFFFFFFFFFFFFFFFFFFFFFFFFF9E
:10042000FFFFFFFFFFFFFFFFFFFFBEEF7975750BBB
:100430001403550375037503740374037403740381
:1004400074037403740374037403740374037403F4
:1004500074037403740374037403740374037403E4
:1004600074037403740374037403740374037403D4
:1004700074037403740374037403740374037403C4
:10048000540313031303974C1DCFFFFFFFFFFFFF20
:10049000FFFFFFFFFFFFFFFFFFFFFFFFFFFFFFFF6C
:1004A000FFFFFFFFFFFFFBDEE74199D6FFFF75B5BA
:1004B000E739BAD6FFFFFFFFFFFFFFFFFFFFFFFF98
:1004C000FFFFFFFFFFFFFFFFD93C97037EDFFFFF2A
:1004D000FFFFFFFFFFFFFFFFFFFFFFFFFFFFFFFF2C
:1004E000FFFFFFFFFFFFFFFFFFFFFFFFFFFFFFFF1C
:1004F000FFFFFFFFFFFFFFFFFFFFFFFFFFFFFFFF0C
:10050000FFFFFFFFFFFFFFFFFFFFFFFFFFFFFFFFFB
:10051000FFFFFFFF1A4D77033ECFFFFFFFFFFFFFF7
:10052000FFFFFFFFFFFFFFFFFFFFFFFF14A5EB62D1
:10053000DFFFFFFF1084F7BDFFFFDADE2C6B718C4D
:10054000DFFFFFFFFFFFFFFFFFFFFFFFFFFFFFFFDB
:10055000FFFFFFFFFFFFFFFF5ED718657403130364
:1005600054037403740374037403740374037403F3
:1005700074037403740374037403740374037403C3
:1005800074037403740374037403740374037403B3
:1005900074037403740374037403740374037403A3
:1005A000740374037403540313031303763C9CB65F
:1005B000FFFFFFFFFFFFFFFFFFFFFFFFFFFFFFFF4B
:1005C000FFFFFFFFFFFFFFFFDFFFAE73308CB6B50D
:1005D0007DEFBAD689521CE7FFFF38CEDADEFFFF87
:1005E000FFFFFFFFFFFFFFFFFFFFFFFFFFFFFFFF1B
:1005F000DB7D36039CA6FFFFFFFFFFFFFFFFFFFF32
:10060000FFFFFFFFFFFFFFFFFFFFFFFFFFFFFFFFFA
:10061000FFFFFFFFFFFFFFFFFFFFFFFFFFFFFFFFEA
:10062000FFFFFFFFFFFFFFFFFFFFFFFFFFFFFFFFDA
:10063000FFFFFFFFFFFFFFFFFFFFFFFFFFFFBFEF1A
:10064000181C181CBFEFFFFFFFFFFFFFFFFFFFFF9E
:10065000FFFFFFFFFFFFFFFF13A5EB629EF7FFFF0A
:10066000FFFFFFFF8A52B6BD71948E73DFFFFFFF5D
:10067000FFFFFFFFFFFFFFFFFFFFFFFFFFFFFFFF8A
:10068000FFFFFFFFFFFF3DD75975B513130313039A
:1006900054037403740374037403740374037403C2
:1006A0007403740374037403740374037403740392
:1006B0007403740374037403740374037403740382
:1006C0007403740374037403740354033403F30254
:1006D0005403B74CBCBEFFFFFFFFFFFFFFFFFFFF50
:1006E000FFFFFFFFFFFFFFFFFFFFFFFFFFFFFFFF1A
:1006F000FBDEFFFFAE7303211084CB5A6D730842FB
:1007000045313CE7FFFFFFFFFFFFFFFFFFFFFFFF5C
:10071000FFFFFFFFFFFFFFFFBDAE57037A65FFFF3F
:10072000FFFFFFFFFFFFFFFFFFFFFFFFFFFFFFFFD9
:10073000FFFFFFFFFFFFFFFFFFFFFFFFFFFFFFFFC9
:10074000FFFFFFFFFFFFFFFFFFFFFFFFFFFFFFFFB9
:10075000FFFFFFFFFFFFFFFFFFFFFFFFFFFFFFFFA9
:10076000FFFFFFFFFFFFFFFFFFFF3ECF7703D944EF
:10077000FFFFFFFFFFFFFFFFFFFFFFFFFFFFFFFF89
:10078000FFFFFFFF92947194FFFF1CE79EF74D6BF4
:10079000B6B5FFFF8A5279D6FFFFFFFFFFFFFFFFCD
:1007A000FFFFFFFFFFFFFFFFFFFFFFFFFFFFFFFF59
:1007B000FFFFFFFFBEEF1B9E77445403F3021303BA
:1007C00054035403740374037403740374037403B1
:1007D0007403740374037403740374037403740361
:1007E0007403740374037403740374037403540371
:1007F0003403F3023403162C997D3DD7FFFFFFFF2E
:10080000FFFFFFFFFFFFFFFFFFFFFFFFFFFFFFFFF8
:10081000FFFFFFFFFFFFFFFFFFFFCE7B508CFFFFBF
:10082000AE7B9294FFFFBADE95B50F841CE7FFFF05
:10083000FFFFFFFFFFFFFFFFFFFFFFFFFFFFFFFFC8
:100840005ED797039934FFFFFFFFFFFFFFFFFFFF16
:10085000FFFFFFFFFFFFFFFFFFFFFFFFFFFFFFFFA8
:10086000FFFFFFFFFFFFFFFFFFFFFFFFFFFFFFFF98
:10087000FFFFFFFFFFFFFFFFFFFFFFFFFFFFFFFF88
:10088000FFFFFFFFFFFFFFFFFFFFFFFFFFFFFFFF78
:10089000FFFFFFFFFFFF9DA637037A65FFFFFFFF06
:1008A000FFFFFFFFFFFFFFFFFFFFFFFFFFFFFFFF58
:1008B000BEF7FFFFEB62BAD63CE707423CE7F39C8A
:1008C0007DEFF3A4508CFFFFFFFFFFFFFFFFFFFF53
:1008D000FFFFFFFFFFFFFFFFFFFFFFFFFFFFFFFF28
:1008E000FFFFFFFF5DDFFA95974CB5133403F3026A
:1008F0001303340354035403540374037403740341
:10090000740374037403740374037403540354036F
:10091000340313031303130374033634797DDCC6E5
:10092000FFFFFFFFFFFFFFFFFFFFFFFFFFFFFFFFD7
:10093000FFFFFFFFFFFFFFFFFFFFFFFFFFFFFFFFC7
:10094000FFFFFFFF9EF7084238C6FFFFCB5AB29465
:10095000FFFFFFFFFFFFFFFFFFFFFFFFFFFFFFFFA7
:10096000FFFFFFFFFFFFFFFFBFEF181CF8139EE71D
:10097000FFFFFFFFFFFFFFFFFFFFFFFFFFFFFFFF87
:10098000FFFFFFFFFFFFFFFFFFFFFFFFFFFFFFFF77
:10099000FFFFFFFFFFFFFFFFFFFFFFFFFFFFFFFF67
:1009A000FFFFFFFFFFFFFFFFFFFFFFFFFFFFFFFF57
:1009B000FFFFFFFFFFFFFFFFFFFFFFFFFFFFFFFF47
:1009C000FFFFFB7D3603FB85FFFFFFFFFFFFFFFF00
:1009D000FFFFFFFFFFFFFFFFFFFFFFFFFFFF2C6B8E
:1009E000B6B5FFFFD29CEF7BFFFFFFFF9EF7AE7B0C
:1009F000484A1CE7FFFFFFFFFFFFFFFFFFFFFFFF6E
:100A0000FFFFFFFFFFFFFFFFFFFFFFFFFFFFFFFFF6
:100A1000FFFFFFFF9EEFBCBEBA85D854162CB5135E
:100A200054033403130313031303130313031303B4
:100A30001303130313035403940BF523974479759D
:100A40007BAE5EDFFFFFFFFFFFFFFFFFFFFFFFFF4C
:100A5000FFFFFFFFFFFFFFFFFFFFFFFFFFFFFFFFA6
:100A6000FFFFFFFFFFFFFFFF6D73BAD6FFFFFFFF22
:100A70009AD607429EF7BEF78952F7C5FFFFFFFFE0
:100A8000FFFFFFFFFFFFFFFFFFFFFFFFFFFFFFFF76
:100A9000DFF7993497033ECFFFFFFFFFFFFFFFFF14
:100AA000FFFFFFFFFFFFFFFFFFFFFFFFFFFFFFFF56
:100AB000FFFFFFFFFFFFFFFFFFFFFFFFFFFFFFFF46
:100AC000FFFFFFFFFFFFFFFFFFFFFFFFFFFFFFFF36
:100AD000FFFFFFFFFFFFFFFFFFFFFFFFFFFFFFFF26
:100AE000FFFFFFFFFFFFFFFFFFFFFFFFFFFF7A6535
:100AF00036035C96FFFFFFFFFFFFFFFFFFFFFFFFD7
:100B0000FFFFFFFFFFFFFFFFFBDE8952B29C2C6B54
:100B1000D29CFFFFFFFFFFFF8D738E73CB5A18C669
:100B2000FFFFFFFFFFFFFFFFFFFFFFFFFFFFFFFFD5
:100B3000FFFFFFFFFFFFFFFFFFFFFFFFFFFFFFFFC5
:100B4000FFFFFFFFFFFFFFFF9EEF3DD7BCBE5BA691
:100B50001B96DA8DBA85BA85DA85FA955BA69CB6BE
:100B60001DCF7EE7DFFFFFFFFFFFFFFFFFFFFFFF60
:100B7000FFFFFFFFFFFFFFFFFFFFFFFFFFFFFFFF85
:100B8000FFFFFFFFFFFFFFFFFFFFFFFFFFFFFFFF75
:100B9000FFFF96B5284ADFFFFFFFFFFF7194108427
:100BA000FFFFBEF77DEFFFFFFFFFFFFFFFFFFFFF30
:100BB000FFFFFFFFFFFFFFFFFFFFF9445703BDB635
:100BC000FFFFFFFFFFFFFFFFFFFFFFFFFFFFFFFF35
:100BD000FFFFFFFFFFFFFFFFFFFFFFFFFFFFFFFF25
:100BE000FFFFFFFFFFFFFFFFFFFFFFFFFFFFFFFF15
:100BF000FFFFFFFFFFFFFFFFFFFFFFFFFFFFFFFF05
:100C0000FFFFFFFFFFFFFFFFFFFFFFFFFFFFFFFFF4
:100C1000FFFFFFFFFFFFFFFFFFFF1A5557037C9EFB
:100C2000FFFFFFFFFFFFFFFFFFFFFFFFFFFFFFFFD4
:100C3000FFFFFFFF5DEF518C34A5FFFFFFFFFFFFBC
:100C4000B2940C63FFFF5DEFFBDEFFFFFFFFFFFFD2
:100C5000FFFFFFFFFFFFFFFFFFFFFFFFFFFFFFFFA4
:100C6000FFFFFFFFFFFFFFFFFFFFFFFFFFFFFFFF94
:100C7000FFFFFFFFFFFFFFFFFFFFFFFFFFFFFFFF84
:100C8000FFFFFFFFFFFFFFFFFFFFFFFFFFFFFFFF74
:100C9000FFFFFFFFFFFFFFFFFFFFFFFFFFFFFFFF64
:100CA000FFFFFFFFFFFFFFFFFFFFFFFFFFFFFFFF54
:100CB000FFFFFFFFFFFFFFFFFFFFFFFFFFFF1084AE
:100CC0006D73FFFFFFFF96B56D6BFFFFFFFFFFFF2B
:100CD000FFFFFFFFFFFFFFFFFFFFFFFFFFFFFFFF24
:100CE000FFFF3A5537037C9EFFFFFFFFFFFFFFFF2B
:100CF000FFFFFFFFFFFFFFFFFFFFFFFFFFFFFFFF04
:100D0000FFFFFFFFFFFFFFFFFFFFFFFFFFFFFFFFF3
:100D1000FFFFFFFFFFFFFFFFFFFFFFFFFFFFFFFFE3
:100D2000FFFFFFFFFFFFFFFFFFFFFFFFFFFFFFFFD3
:100D3000FFFFFFFFFFFFFFFFFFFFFFFFFFFFFFFFC3
:100D4000FFFFFFFFFFFFF94457037CA6FFFFFFFFF4
:100D5000FFFFFFFFFFFFFFFFFFFFFFFFFFFFFFFFA3
:100D6000FFFFFFFFFFFFFFFF9AD6E7419EF7FFFF60
:100D7000FFFFFFFFFFFFFFFFFFFF3CE7FFFFFFFF5E
:100D8000FFFFFFFFFFFFFFFFFFFFFFFFFFFFFFFF73
:100D9000FFFFFFFFFFFFFFFFFFFFFFFFFFFFFFFF63
:100DA000FFFFFFFFFFFFFFFFFFFFFFFFFFFFFFFF53
:100DB000FFFFFFFFFFFFFFFFFFFFFFFFFFFFFFFF43
:100DC000FFFFFFFFFFFFFFFFFFFFFFFFFFFFFFFF33
:100DD000FFFFFFFFFFFFFFFFFFFF79D6484ABEF787
:100DE000FFFFFFFFFFFFFFFFFFFFEB62CF7BF3A4DF
:100DF0006952BAD6FFFFFFFFFFFFFFFFFFFFFFFFB4
:100E0000FFFFFFFFFFFFFFFFFFFF3A5536033C9652
:100E1000FFFFFFFFFFFFFFFFFFFFFFFFFFFFFFFFE2
:100E2000FFFFFFFFFFFFFFFFFFFFFFFFFFFFFFFFD2
:100E3000FFFFFFFFFFFFFFFFFFFFFFFFFFFFFFFFC2
:100E4000FFFFFFFFFFFFFFFFFFFFFFFFFFFFFFFFB2
:100E5000FFFFFFFFFFFFFFFFFFFFFFFFFFFFFFFFA2
:100E6000FFFFFFFFFFFFFFFFFFFFFFFFFFFFFFFF92
:100E7000FFFFD94457035C9EFFFFFFFFFFFFFFFF0B
:100E8000FFFFFFFFFFFFFFFFFFFFFFFFFFFFFFFF72
:100E90009EF7284A17C6FFFFFFFFFFFFFFFFFFFF78
:100EA000FFFF7DEFE7410C6334A5FFFFFFFFFFFF6E
:100EB000FFFFFFFFFFFFFFFFFFFFFFFFFFFFFFFF42
:100EC000FFFFFFFFFFFFFFFFFFFFFFFFFFFFFFFF32
:100ED000FFFFFFFFFFFFFFFFFFFFFFFFFFFFFFFF22
:100EE000FFFFFFFFFFFFFFFFFFFFFFFFFFFFFFFF12
:100EF000FFFFFFFFFFFFFFFFFFFFFFFFFFFFDFFF22
:100F0000FFFFFFFF59CE821814A5FFFFFFFFFFFF71
:100F1000FFFFFFFFDFFF508CEF833CE7FFFFFFFF8A
:100F2000FFFFFFFFFFFFFFFFFFFFFFFFFFFFFFFFD1
:100F3000FFFF1A5536033C8EFFFFFFFFFFFFFFFF49
:100F4000FFFFFFFFFFFFFFFFFFFFFFFFFFFFFFFFB1
:100F5000FFFFFFFFFFFFFFFFFFFFFFFFFFFFFFFFA1
:100F6000FFFFFFFFFFFFFFFFFFFFFFFFFFFFFFFF91
:100F7000FFFFFFFFFFFFFFFFFFFFFFFFFFFFFFFF81
:100F8000FFFFFFFFFFFFFFFFFFFFFFFFFFFFFFFF71
:100F9000FFFFFFFFFFFFFFFFFFFFFFFFFFFF1A4DF8
:100FA00036031C8EFFFFFFFFFFFFFFFFFFFFFFFF6A
:100FB000FFFFFFFFFFFFFFFFFFFF9EF718C6FFFFCA
:100FC000FFFFFFFFFFFFFFFFFFFFFFFF7194719423
:100FD000FBDE8D73AE7BFFFFFFFFFFFFFFFFFFFF19
:100FE000FFFFFFFFFFFFFFFFFFFFFFFFFFFFFFFF11
:100FF000FFFFFFFFFFFFFFFFFFFFFFFFFFFFFFFF01
:10100000FFFFFFFFFFFFFFFFFFFFFFFFFFFFFFFFF0
:10101000FFFFFFFFFFFFFFFFFFFFFFFFFFFFFFFFE0
:10102000FFFFBEF7DFFF18C6452938C6FFFFDBDE2E
:101030008E73EB62BEF7FFFFFFFFFFFFFFFFFFFFB7
:10104000FFFFFFFFFFFFFFFFFFFFFFFFFFFFFFFFB0
:10105000FFFFFFFFFFFFFFFFDFF7D94457035C9659
:10106000FFFFFFFFFFFFFFFFFFFFFFFFFFFFFFFF90
:10107000FFFFFFFFFFFFFFFFFFFFFFFFFFFFFFFF80
:10108000FFFFFFFFFFFFFFFFFFFFFFFFFFFFFFFF70
:10109000FFFFFFFFFFFFFFFFFFFFFFFFFFFFFFFF60
:1010A000FFFFFFFFFFFFFFFFFFFFFFFFFFFFFFFF50
:1010B000FFFFFFFFFFFFFFFFFFFFFFFFFFFFFFFF40
:1010C000FFFFFFFFFFFFFFFFFFFF5A5D3603BB750A
:1010D000FFFFFFFFFFFFFFFFFFFFFFFFFFFFFFFF20
:1010E000FFFFFFFFFFFFFFFFFFFFFFFFFFFFFFFF10
:1010F000FFFFFFFFFFFFA639B6BDFFFFFFFFE74180
:10110000FFFF7194695291949AD6FFFFFFFFFFFF92
:10111000FFFFFFFFFFFFFFFFFFFFFFFFFFFFFFFFDF
:10112000FFFFFFFFFFFFFFFFFFFFFFFFFFFFFFFFCF
:10113000FFFFFFFFFFFFFFFFFFFFFFFFFFFFFFFFBF
:10114000FFFFFFFFFFFFFFFFFFFFFFFF38C6AE738C
:101150009EF7C639494A38C6DFFFB2941084F39C23
:10116000FFFFFFFFFFFFFFFFFFFFFFFFFFFFFFFF8F
:10117000FFFFFFFFFFFFFFFFFFFFFFFFFFFFFFFF7F
:101180009EE7792C77037CA6FFFFFFFFFFFFFFFFA1
:10119000FFFFFFFFFFFFFFFFFFFFFFFFFFFFFFFF5F
:1011A000FFFFFFFFFFFFFFFFFFFFFFFFFFFFFFFF4F
:1011B000FFFFFFFFFFFFFFFFFFFFFFFFFFFFFFFF3F
:1011C000FFFFFFFFFFFFFFFFFFFFFFFFFFFFFFFF2F
:1011D000FFFFFFFFFFFFFFFFFFFFFFFFFFFFFFFF1F
:1011E000FFFFFFFFFFFFFFFFFFFFFFFFFFFFFFFF0F
:1011F000FFFFFFFFFFFFBB7536031A55DFF7FFFF49
:10120000FFFFFFFFFFFFFFFFFFFFFFFFFFFFFFFFEE
:10121000FFFFFFFFFFFFFFFFFFFFFFFFFFFF75B5B2
:101220006952AE736D73EB62EF7BFFFFCA5A9AD6B9
:10123000F3A40B6314A559CEF3A4FBDEDFFFFFFF7D
:10124000FFFFFFFFFFFFFFFFFFFFFFFFFFFFFFFFAE
:10125000FFFFFFFFFFFFFFFFFFFFFFFFFFFFFFFF9E
:10126000FFFFFFFFFFFFFFFF5DEF18C6F7BDBEF7F3
:101270008E73BEF7FFFFBEF76952FFFF7194508C6B
:101280002C6BF7BDB294FBDE484A9EF7FFFFFFFFD1
:10129000FFFFFFFFFFFFFFFFFFFFFFFFFFFFFFFF5E
:1012A000FFFFFFFFFFFFFFFF1EC7F813B703DDB609
:1012B000FFFFFFFFFFFFFFFFFFFFFFFFFFFFFFFF3E
:1012C000FFFFFFFFFFFFFFFFFFFFFFFFFFFFFFFF2E
:1012D000FFFFFFFFFFFFFFFFFFFFFFFFFFFFFFFF1E
:1012E000FFFFFFFFFFFFFFFFFFFFFFFFFFFFFFFF0E
:1012F000FFFFFFFFFFFFFFFFFFFFFFFFFFFFFFFFFE
:10130000FFFFFFFFFFFFFFFFFFFFFFFFFFFFFFFFED
:10131000FFFFFFFFFFFFFFFFFFFFFFFFFFFFFFFFDD
:10132000FFFF5C965703582C5ED7FFFFFFFFFFFFC0
:10133000FFFFFFFFFFFFFFFFFFFFFFFFFFFFFFFFBD
:10134000FFFFFFFFFFFFDFFF484A9AD6FFFF59CE9E
:10135000B6B5FFFF18C6A639DBDEFFFFFFFFBEF7FD
:101360009AD6308CE741AA5AAE7B1CE718C6D7BD87
:1013700079D6BEF7FFFFFFFFFFFFFFFFDFFFFFFF95
:10138000FFFFFFFFDFFFFFFFFFFFFFFFFFFFD6BDF8
:10139000EB620C636D7375ADFFFFCB5A17C6FFFF91
:1013A000FFFF8E7396B55DEFCB5A5DEFCA5A494A7F
:1013B000FFFF34AD1CE7FFFFFFFFFFFFFFFFFFFF55
:1013C000FFFFFFFFFFFFFFFFFFFFFFFFFFFFFFFF2D
:1013D0007C9E9703181C3ECFFFFFFFFFFFFFFFFF20
:1013E000FFFFFFFFFFFFFFFFFFFFFFFFFFFFFFFF0D
:1013F000FFFFFFFFFFFFFFFFFFFFFFFFFFFFFFFFFD
:10140000FFFFFFFFFFFFFFFFFFFFFFFFFFFFFFFFEC
:10141000FFFFFFFFFFFFFFFFFFFFFFFFFFFFFFFFDC
:10142000FFFFFFFFFFFFFFFFFFFFFFFFFFFFFFFFCC
:10143000FFFFFFFFFFFFFFFFFFFFFFFFFFFFFFFFBC
:10144000FFFFFFFFFFFFFFFFFFFFFFFFFFFFFDBEEF
:10145000D80BB7039DAEFFFFFFFFFFFFFFFFFFFFAE
:10146000FFFFFFFFFFFFFFFFFFFFFFFFFFFFFFFF8C
:10147000BEF796B5FFFFFFFFFFFFFFFFFFFFCF7B2C
:101480006D6B8D73EB6296B5FFFFFFFFFFFFEB5AAD
:10149000BADE79D679D6E741508CCE7B895218C610
:1014A000FFFF9DF7AE7B0C630C63F7BDFFFF54ADF0
:1014B000B294FFFFFFFFFFFF718C8E73FFFFFFFFF2
:1014C000FFFFFFFFF39CCF7BFFFFFFFFB6B56D7300
:1014D000FFFF8E7334A55DEFCF7BDFFFFFFFFFFFC4
:1014E000FFFFFFFFFFFFFFFFFFFFFFFFFFFFFFFF0C
:1014F000FFFFFFFFFFFFFFFF9B6D3603D944BFEFE8
:10150000FFFFFFFFFFFFFFFFFFFFFFFFFFFFFFFFEB
:10151000FFFFFFFFFFFFFFFFFFFFFFFFFFFFFFFFDB
:10152000FFFFFFFFFFFFFFFFFFFFFFFFFFFFFFFFCB
:10153000FFFFFFFFFFFFFFFFFFFFFFFFFFFFFFFFBB
:10154000FFFFFFFFFFFFFFFFFFFFFFFFFFFFFFFFAB
:10155000FFFFFFFFFFFFFFFFFFFFFFFFFFFFFFFF9B
:10156000FFFFFFFFFFFFFFFFFFFFFFFFFFFFFFFF8B
:10157000FFFFFFFFFFFFFFFFFFFF7EDFB93C3703E9
:101580007B6DDFF7FFFFFFFFFFFFFFFFFFFFFFFFA9
:10159000FFFFFFFFFFFFFFFFFFFFFFFFFFFFFFFF5B
:1015A000FFFFFFFFFFFF7DEF494AFFFFFFFFDBDE8D
:1015B00079CEFFFFFFFFDBDEEB5AFFFFFFFF18C610
:1015C0008E73FFFFFFFF55ADEB62FFFF0C63B29C14
:1015D0009EF79AD6284ADBDED6BD6D73FFFFFFFF6C
:1015E000FFFF59CECA5A14A5CE7B8D739EF75CEFD0
:1015F0006952FFFFFFFFDBDECA5AFFFFDBDE92947A
:10160000FFFFFFFFFFFFFFFFFFFFFFFFFFFFFFFFEA
:10161000FFFFFFFFFFFFFFFFFFFFFFFFFFFF5ED7A3
:1016200079345703BB75FFFFFFFFFFFFFFFFFFFF8D
:10163000FFFFFFFFFFFFFFFFFFFFFFFFFFFFFFFFBA
:10164000FFFFFFFFFFFFFFFFFFFFFFFFFFFFFFFFAA
:10165000FFFFFFFFFFFFFFFFFFFFFFFFFFFFFFFF9A
:10166000FFFFFFFFFFFFFFFFFFFFFFFFFFFFFFFF8A
:10167000FFFFFFFFFFFFFFFFFFFFFFFFFFFFFFFF7A
:10168000FFFFFFFFFFFFFFFFFFFFFFFFFFFFFFFF6A
:10169000FFFFFFFFFFFFFFFFFFFFFFFFFFFFFFFF5A
:1016A000FFFFFFFFFFFFFFFFBB75570358241DC758
:1016B000FFFFFFFFFFFFFFFFFFFFFFFFFFFFFFFF3A
:1016C000FFFFFFFFFFFFFFFFFFFFFFFFFFFFFFFF2A
:1016D000DBDE284AEF7BD7BDFFFFFFFFFFFFFFFFE9
:1016E00055ADCE7BFFFFFFFFD7BDA6390F84718CB0
:1016F0000B6396B53CE7AA5AFFFFFFFFFFFFF3A479
:10170000308CFBDE2C63FFFFFFFFFFFF9EF7C63927
:101710007194F7C55DEFFFFFFFFF8D73AE7B95B54D
:10172000AA5A14A5FFFFFFFFFFFFFFFFFFFFFFFF08
:10173000FFFFFFFFFFFFFFFFFFFFFFFFFFFFFFFFB9
:10174000FFFFFFFFFFFF3C8E9703F80BBDB6FFFFC7
:10175000FFFFFFFFFFFFFFFFFFFFFFFFFFFFFFFF99
:10176000FFFFFFFFFFFFFFFFFFFFFFFFFFFFFFFF89
:10177000FFFFFFFFFFFFFFFFFFFFFFFFFFFFFFFF79
:10178000FFFFFFFFFFFFFFFFFFFFFFFFFFFFFFFF69
:10179000FFFFFFFFFFFFFFFFFFFFFFFFFFFFFFFF59
:1017A000FFFFFFFFFFFFFFFFFFFFFFFFFFFFFFFF49
:1017B000FFFFFFFFFFFFFFFFFFFFFFFFFFFFFFFF39
:1017C000FFFFFFFFFFFFFFFFFFFFFFFFFFFFFFFF29
:1017D000FFFFFFFFDDBE181C7703BB75DFF7FFFFC0
:1017E000FFFFFFFFFFFFFFFFFFFFFFFFFFFFFFFF09
:1017F000FFFFFFFFFFFFFFFFFFFFFFFFBEF796B5F5
:10180000AE730C635DEFFFFFFFFFAE7314A5FFFF28
:10181000FFFFF3A48E7318C6C739D39CFFFF38CEE1
:101820000B63FFFFFFFFFFFFB6BDAE739EF7CB5A02
:10183000FFFFFFFFFFFFFFFFEB629EF7FFFF5DEF84
:1018400059CEDFFFBEF7508CCF7B18C6FFFFFFFFDE
:10185000FFFFFFFFFFFFFFFFFFFFFFFFFFFFFFFF98
:10186000FFFFFFFFFFFFFFFFFFFFFFFF5ED7B93C5A
:1018700036031A4D9EE7FFFFFFFFFFFFFFFFFFFF4D
:10188000FFFFFFFFFFFFFFFFFFFFFFFFFFFFFFFF68
:10189000FFFFFFFFFFFFFFFFFFFFFFFFFFFFFFFF58
:1018A000FFFFFFFFFFFFFFFFFFFFFFFFFFFFFFFF48
:1018B000FFFFFFFFFFFFFFFFFFFFFFFFFFFFFFFF38
:1018C000FFFFFFFFFFFFFFFFFFFFFFFFFFFFFFFF28
:1018D000FFFFFFFFFFFFFFFFFFFFFFFFFFFFFFFF18
:1018E000FFFFFFFFFFFFFFFFFFFFFFFFFFFFFFFF08
:1018F000FFFFFFFFFFFFFFFFFFFFFFFFFFFFFFFFF8
:10190000DFF77A655703381CBDAEFFFFFFFFFFFF0F
:10191000FFFFFFFFFFFFFFFFFFFFFFFFFFFFFFFFD7
:10192000FFFFFFFFFFFFFFFFFFFFFFFF9EF7DFFF50
:10193000FFFFFFFFCF7BBAD6FFFFFFFFEF7BD39CFC
:10194000FFFFBADE284ABEF77DEF494A7DEFFFFF71
:10195000FFFF8E73F3A4FFFFAA5A9DF77DEF1BE7ED
:10196000FFFFEF7B69524D6B0C63308CDFFFFFFF95
:10197000FFFFFFFFFFFFFFFFFFFFFFFFFFFFFFFF77
:10198000FFFFFFFFFFFFFFFFFFFFFFFFFFFFFFFF67
:10199000FFFFDFF7DB7D9703D80B7C9EFFFFFFFF88
:1019A000FFFFFFFFFFFFFFFFFFFFFFFFFFFFFFFF47
:1019B000FFFFFFFFFFFFFFFFFFFFFFFFFFFFFFFF37
:1019C000FFFFFFFFFFFFFFFFFFFFFFFFFFFFFFFF27
:1019D000FFFFFFFFFFFFFFFFFFFFFFFFFFFFFFFF17
:1019E000FFFFFFFFFFFFFFFFFFFFFFFFFFFFFFFF07
:1019F000FFFFFFFFFFFFFFFFFFFFFFFFFFFFFFFFF7
:101A0000FFFFFFFFFFFFFFFFFFFFFFFFFFFFFFFFE6
:101A1000FFFFFFFFFFFFFFFFFFFFFFFFFFFFFFFFD6
:101A2000FFFFFFFFFFFFFFFFFFFFFFFFFFFFFDBE09
:101A3000792C5603F9443ECFFFFFFFFFFFFFFFFF66
:101A4000FFFFFFFFFFFFFFFFFFFFFFFFFFFFFFFFA6
:101A5000FFFFFFFFFFFFFFFFFFFFFFFFFFFFFFFF96
:101A6000FFFFFFFFFFFF34AD59CEFFFFFFFF6D7398
:101A7000D39CFFFF55AD8A52B29CCE7B0C63BEF760
:101A8000FFFFEB62CA5A0C63CF7BDFFF1CE7F7BD99
:101A90003CE7FFFFFFFFFFFFFFFFFFFFFFFFFFFF31
:101AA000FFFFFFFFFFFFFFFFFFFFFFFFFFFFFFFF46
:101AB000FFFFFFFFFFFFFFFFFFFF7CA6181C570380
:101AC0005A5D9FE7FFFFFFFFFFFFFFFFFFFFFFFFE5
:101AD000FFFFFFFFFFFFFFFFFFFFFFFFFFFFFFFF16
:101AE000FFFFFFFFFFFFFFFFFFFFFFFFFFFFFFFF06
:101AF000FFFFFFFFFFFFFFFFFFFFFFFFFFFFFFFFF6
:101B0000FFFFFFFFFFFFFFFFFFFFFFFFFFFFFFFFE5
:101B1000FFFFFFFFFFFFFFFFFFFFFFFFFFFFFFFFD5
:101B2000FFFFFFFFFFFFFFFFFFFFFFFFFFFFFFFFC5
:101B3000FFFFFFFFFFFFFFFFFFFFFFFFFFFFFFFFB5
:101B4000FFFFFFFFFFFFFFFFFFFFFFFFFFFFFFFFA5
:101B5000FFFFFFFFFFFFFFFFFFFFFFFF1C8ED8030C
:101B600077035A657EDFFFFFFFFFFFFFFFFFFFFFE9
:101B7000FFFFFFFFFFFFFFFFFFFFFFFFFFFFFFFF75
:101B8000FFFFFFFFFFFFFFFFFFFFFFFFFFFFFFFF65
:101B9000FFFFFFFFFFFFFFFFDFFF3CE7FFFFFFFF50
:101BA000BADEF39C96B5FFFFFFFFFFFF9EF77DEFC8
:101BB000FFFFFFFFFFFFFFFFFFFFFFFFFFFFFFFF35
:101BC000FFFFFFFFFFFFFFFFFFFFFFFFFFFFFFFF25
:101BD000FFFFFFFFFFFFFFFFFFFFFFFFFFFFFFFF15
:101BE000DDB6993456039934FDBEFFFFFFFFFFFFBA
:101BF000FFFFFFFFFFFFFFFFFFFFFFFFFFFFFFFFF5
